:020000040800F2
:1000000000000110A1F50308292C0308691201085A
:10001000A5F60308A5F60308A5F6030800000000EE
:10002000000000000000000000000000693203082A
:100030006732030800000000653203088DDB00080A
:10004000A5F60308A5F60308A5F60308A5F6030818
:10005000A5F60308A5F603082DE5000859E60008F3
:100060001DE60008E1E50008A5E50008B9A70008BD
:10007000A9A7000899A7000889A7000879A7000880
:1000800065A7000851A70008A5F60308A5F6030810
:10009000A5F60308A5F60308A5F6030869E5000818
:1000A000A9D2000819D30008A5F6030829D300082F
:1000B00009D30008F9D20008E9D20008FDBF000802
:1000C00005C00008F1BF0008F9BF0008A5F6030845
:1000D000A5F6030841DE0008A1DD000801DD0008E7
:1000E000F1E40008A5F60308253C0308A5F603087B
:1000F000B9D20008A5F60308C9D200083DA7000838
:10010000A5F60308A5F60308D9D20008A5F603084A
:1001100061DC0008A5F603083DE7010821E70108B6
:1001200029A7000815A7000801A70008EDA60008E8
:10013000D9A60008A5F60308A5F60308A5F6030846
:10014000A5F60308A5F60308A5F603082B2C03085B
:10015000C5A60008B1A600089DA60008C1DB0008DE
:10016000E5BF0008EDBF0008A5F60308A5F60308E3
:10017000A5F60308A5F60308A5F60308A5F60308E7
:08018000A5F60308A5F603082B
:0801880038F103000100000042
:10019000020203007C1E0020781E002000000000E8
:1001A000000000000E020200741E0020801E0020CD
:1001B00000000000180600081D000100982400201F
:1001C00020250020000000001A0600082700040077
:1001D000B824002024250020000000001C06000890
:1001E00016000800342500204C25002000000000E7
:1001F000200600080A020A00A4260020B4260020D7
:1002000000000000280600082C001000042A00202E
:10021000F42900200000000009ED01082B00240053
:10022000382A0020142A002000000000D9EC010820
:10023000290050002C2900205C2A0020000000002A
:1002400000000000031233005F2D00202C2D002041
:10025000000000003406000825005A00782C002019
:10026000D22C00200000000000000000F6110C005D
:100270006C2C0020602C00200000000068060008A4
:1002800015007000802B0020F02B002000000000E3
:10029000000000002A006000C02A0020202B00205F
:1002A00000000000FD6C0208090201007E2F002002
:1002B000F82F0020000000007406000812200C0037
:1002C000A92F0020FC2F0020000000007606000867
:1002D0000C002400B62F0020083000200000000091
:1002E000C3110308000205002C300020C432002096
:1002F00000000000000000001E0004003430002058
:10030000CC3200200000000082060008030001003B
:1003100084340020E83800200000000000000000C5
:1003200003010A001C3900202839002000000000C9
:100330008606000822000C00B83C0020383D002052
:10034000000000009006000826000E00543D00202A
:10035000443D002000000000919902080B2010008D
:10036000DC390020643D0020000000009C060008ED
:100370001F000E00403F002014410020000000003C
:10038000AC06000805020100283F0020244100209F
:1003900000000000BA060008051006005E420020BA
:1003A0004443002000000000BC0600080E20EA00C4
:1003B0003E4100204C4300200000000075710308FE
:1003C000020103002B4100203844002000000000FF
:1003D00085110308010104000C4A0020F46100208B
:1003E0000000000000000000080209001C6100205D
:1003F000F861002000000000E9C2000806020C00BD
:100400009461002004620020000000005D8A000862
:1004100007020200C86100201062002000000000F6
:10042000C2060008FF010100EC61002014620020F8
:1004300000000000C406000802000C00A0610020BB
:10044000186200200000000000000000F701060014
:10045000106100202462002000000000C606000891
:1004600034001000C87000209871002000000000C7
:10047000B96C020818102C0054700020A8710020DC
:10048000000000006DF201080D00440080700020A3
:10049000D471002000000000C5930308FE0109008C
:1004A0004C6A0020187200200000000001C1000802
:1004B000FD012400B87F0020DC7F00200000000048
:1004C00061C2000806001600247C00200080002085
:1004D0000000000031700308FB010100607B002078
:1004E0001880002000000000C5C00008FC010900C1
:1004F0002C7A00201C8000200000000091C0000821
:100500000A10120024720020288000200000000041
:10051000CC06000801200800E081002000820020B5
:1005200000000000DE0600081A000800C481002058
:100530000882002000000000E60600081300040006
:10054000AC870020B887002000000000F0060008FB
:1005500010000300A8870020BC87002000000000D6
:10056000F40600082800100098870020C0870020AB
:1005700000000000FDF4020823001000888700201E
:10058000D08700200000000019F5020819000500BE
:1005900080870020E087002000000000F8060008A7
:1005A000F81101007C870020E8870020000000008F
:1005B000FE0600080001040078870020EC87002078
:1005C00000000000000700082F0011005C870020D9
:1005D000F0870020000000000407000804008000ED
:1005E000A4A50020E0AE00200000000000000000F4
:1005F000F90104001488002060AF00200000000012
:10060000D1C200081400020088B10020F0B100201F
:080610000000000016070008BD
:100618000000000020030000C40900001901282878
:1006280000004A01B400D6010000000000000000EC
:1006380000000000000000000000000000000000B2
:1006480000000000000000000000000000000000A2
:100658000000000000000000000000000000010091
:100668000000000000000000000000001000000072
:100678000001000546344259000000000100040151
:1006880001006C1600000000C800141E0100640080
:100698002C0128002B21231E640102000000010008
:1006A8000A01290000000000000001000000000508
:1006B80000000000200002010000013C000055007D
:1006C8000100000000300100005A00000000900105
:1006D8002C01C8006400E8036400040A00017E05D8
:1006E800EA05B4053200000008000000000105001A
:1006F8000000280100000400900100000000000034
:1007080000000000000000000000000000000300DE
:100718005001000007000000020000000000000077
:10072800000000000102030406070809FF0000009A
:1007380001010000B83D0408FC690408000000003D
:1007480000000000C83D0408D03D04080000000077
:1007580001200000D43D0408DC3D0408000000002E
:1007680001400000E03D0408246004080000000087
:1007780001200000EC3D0408F83D040800000000DA
:1007880004000000FC3D0408083E040800000000C6
:10079800040000000C3E04083C4F04080000000060
:1007A80001000000020100000000803F0000803FBF
:1007B8000000000000000000000000000000803F72
:1007C8000101D60121FF020800000000000000001E
:1007D800FFFFFFFF01010100D940020800000000EF
:1007E8003C020020586804080000000000000000D7
:1007F8000000000000000000FC6904080000000080
:10080800000000007C0600200400000004680408C2
:100818000C00000085E602086406002000000000C5
:10082800246704080C0000005DE602085806002052
:1008380000000000786804080800000000000000BC
:100848004C06002004000000686804080C00000042
:10085800C5DE020840060020000000000C670408FE
:1008680003000000D9E2020834060020000000005E
:100878007068040803000000D9E202082806002076
:1008880000000000106704080100000000000000DC
:100898000000000000000000000000000D00000043
:1008A8000000000000000000000000005868040874
:1008B8000000000000000000000000000000000030
:1008C800FC69040800000000000000007C0600200D
:1008D800040000009C6704080300000081E302088C
:1008E8001C06002008000000686804080C000000CE
:1008F800C5DE020840060020000000000C6704085E
:1009080003000000D9E202083406002000000000BD
:100918007068040803000000D9E2020828060020D5
:10092800000000001067040801000000000000003B
:100938000000000000000000000000000D000000A2
:1009480000000000000000000000000080680408AB
:10095800000000000000000000000000000000008F
:10096800FC69040800000000000000007C0600206C
:1009780004000000A467040803000000D9E202088C
:100988007006002000000000106704080100000045
:10099800000000000000000000000000000000004F
:1009A8000D00000000000000000000000000000032
:1009B800F02F002088136F1701000000F22F00208D
:1009C80088136F1700000000E466040800000000A8
:1009D800000000000000000000000000F4660408A9
:1009E8000800000000000000AC0200200400000025
:1009F800006704080800000000000000A0020020B2
:100A0800000000000C6704080400000099E40208D4
:100A1800000000000000000010670408010000004A
:100A280000000000000000000000000000000000BE
:100A38000D000000000000000000000000000000A1
:100A4800F42F002088136F1701000000203F0020BA
:100A580088136F17000000009DDE020800000000E8
:100A6800B8020020F62F002001000000B02504087D
:100A7800223F002001000000BC250408183F002088
:100A880002000000C42504089EA600200000000003
:100A9800000000009CA600200000000000000000EC
:100AA8009AA60020000000000000000098A6002080
:100AB800000000000000000096A6002000000000D2
:100AC8000000000094A600200000000000000000C4
:100AD800B40B002000000000000000001F2F0020C1
:100AE80002000000D0250408546704080000000034
:100AF800000000000000000000000000F466040888
:100B080008000000000000003C0300200400000072
:100B180000670408080000000000000030030020FF
:100B2800000000000C6704080400000071DE0208E1
:100B38000000000000000000106704080100000029
:100B4800000000000000000000000000000000009D
:100B58000D00000000000000000000000000000080
:100B680064670408000000000000000000000000A6
:100B780000000000746704080C00000005E6020885
:100B88006C03002004000000806704080C000000CB
:100B9800E1E5020860030020040000008C670408F7
:100BA8000C000000B5E40208540300200000000017
:100BB8009867040803000000A1E302084803002026
:100BC80008000000A467040803000000D9E2020836
:100BD80070060020000000001067040801000000F3
:100BE80000000000000000000000000000000000FD
:100BF8000D000000000000000000000000000000E0
:100C0800AC670408000000000000000000000000BD
:100C180000000000B467040804000000E9E40208CA
:100C28000000000000000000106704080100000038
:100C380000000000000000000000000000000000AC
:100C48000D0000000000000000000000000000008F
:100C58000C6804080000000000000000000000000C
:100C680000000000E04804080C000000000000003C
:100C7800CC030020040000001C68040808000000E1
:100C880000000000C00300200400000028680408D9
:100C98000800000000000000B40300200400000069
:100CA800306804080800000000000000A8030020C5
:100CB8000400000038680408080000000000000074
:100CC8009C0300200400000040680408080000009D
:100CD8000000000090030020040000004868040899
:100CE8000800000000000000840300200400000049
:100CF8005068040808000000000000007803002085
:100D08000400000010670408010000000000000053
:100D18000000000000000000000000000D000000BE
:100D280000000000000000000000000089DE02084A
:100D380000000000D80300200000000000000000B0
:100D4800500400200000000000000000F004002013
:100D58001E3F002004000000DC2504081C3F002082
:100D6800E0150C17000000001B3F002008000000E1
:100D7800BC2A04081A3F002005000000F0250408DA
:100D88000000000000000000400500202D202D2D4F
:100D9800202D2D2D2D202D2D2D00000000000000D0
:100DA800000000000000000000000000000000003B
:100DB8000102030401020304060708094C4604085B
:100DC800000000000000000095110308A086010043
:100DD8000400000000000000000000000000000007
:100DE80000000000000000000000000000000000FB
:100DF800487404089C4504080000000011450108D7
:100E08007D00000006000000000000000000000057
:100E180000000000000000000000000000000000CA
:100E280000000000406B0408000000000000000003
:100E3800390B0108E803000003000000000000006F
:100E4800000000000000000000000000000000009A
:100E58000000000000000000486B040800000000CB
:100E6800000000009571030810270000030000002F
:100E7800000000000000000000000000000000006A
:100E8800000000000000000000000000DC6804080A
:100E98000000000061EB01083DE70008204E00005B
:100EA8000500000000000000000000000000000035
:100EB800000000000000000000000000000000002A
:100EC800E04704080000000000000000F1120108DB
:100ED80010270000010000000000000000000000D2
:100EE80000000000000000000000000000000000FA
:100EF80000000000546B040800000000000000001F
:100F080009E70008E80300000500000000000000F1
:100F180000000000000000000000000000000000C9
:100F28000000000000000000606B040800000000E2
:100F380000000000E1130308204E00000300000039
:100F48000000000000000000000000000000000099
:100F5800000000000000000000000000706B0408A2
:100F68000000000000000000E9110308204E000006
:100F78000300000000000000000000000000000066
:100F88000000000000000000000000000000000059
:100F9800806B04080000000000000000A50F010895
:100FA800400D0300030000000000000000000000E6
:100FB8000000000000000000000000000000000029
:100FC80000000000184704080000000000000000AE
:100FD800359F0308102700000100000000000000F2
:100FE80000000000000000000000000000000000F9
:100FF8000000000000000000B845040800000000E0
:1010080000000000756002081027000003000000BF
:1010180000000000000000000000000000000000C8
:10102800000000000000000000000000906B0408B1
:10103800000000000000000091E30308A086010002
:101048000100000000000000000000000000000097
:101058000000000000000000000000000000000088
:10106800A84504080000000000000000B1E20308E1
:1010780050C3000001000000000000000000000054
:101088000000000000000000000000000000000058
:1010980000000000986B0408000000000000000039
:1010A80019DE0308A861000001000000000000002C
:1010B8000000000000000000000000000000000028
:1010C8000000000000000000A46B040800000000FD
:1010D8000000000013660208A0860100010000005D
:1010E80000000000000000000000000000000000F8
:1010F800000000000000000000000000E8470408AD
:10110800000000000000000045180108A00F0000C2
:1011180001000000000000000000000000000000C6
:1011280000000000000000000000000000000000B7
:101138004C480408000000000000000015CB02081D
:10114800102700000100000000000000000000005F
:101158000000000000000000000000000000000087
:1011680000000000804504080000000000000000A6
:10117800CDE902081A41000001000000000000004B
:101188000000000000000000000000000000000057
:101198000000000000000000B06B04080000000020
:1011A800000000004DB10108400D030000000000E0
:1011B8000000000000000000000000000000000027
:1011C800000000000000000000000000B86B0408E8
:1011D8000000000000000000E9B00108400D030015
:1011E80000000000000000000000000000000000F7
:1011F80000000000000000000000000000000000E7
:10120800C06B04080000000000000000C569020867
:10121800A08601000300000000000000000000009C
:1012280000000000000000000000000000000000B6
:101238000000000009024300020100C03209040056
:10124800000102020100052400100105240100012B
:10125800042402020524060001070582030800FF92
:1012680009040100020A000000070501024000000D
:101278000705810240000000FF00000000FFFF009A
:1012880000000000AA5505010000012D202D2D2089
:101298002D2D2D2D202D2D2D2D00000000000000BE
:1012A80000000000000000000000AA550B0100002B
:1012B800AA5507010000AA55090200000000000015
:1012C80001000000C012AA5503009F0020700020F2
:1012D800702D72000000000000000000E0180020DF
:1012E800FFFFFFFFFA0000000100000001000000FE
:1012F800AC670408000000000000000000000000C7
:1013080000000000136C0408040000006346020893
:101318000000000000000000106704080100000041
:1013280000000000000000000000000000000000B5
:101338000D00000000000000000000000000000098
:1013480056A600200100C4090000000054A6002091
:101358000100C4090000000052A600200100C409D1
:101368000000000050A600200100C4090000000091
:101378004CA600200100C409000000004EA6002071
:101388000100C409000000004AA600200100C409A9
:101398000000000048A600200100C4090000000069
:1013A8000000000000000000E00B0020E43E0020E8
:1013B8009CFF2C0100000000C40000200A0000006F
:1013C800E42A04081C2F0020E0150C170000000078
:1013D800C600002008000000BC2A0408C500002040
:1013E80005000000F02504081E2F00200200000060
:1013F800FC2A0408644200200100FF7F010000006D
:101408005D42002002000000082B04083241002041
:1014180003000000182B04083141002003000000DD
:10142800182B0408304200200000F40101000000DD
:101438002E4200200000F401010000002C42002090
:101448000000F401010000002A4200200000F4011D
:10145800010000002842002000FF0100484200204F
:10146800E803D0070A00000046420020006401009B
:101478000A000000424200200064010041420020AE
:101488000064010047420020006401000A000000D7
:1014980040420020006401000A000000454200208C
:1014A800006401000A0000004442002000640100BA
:1014B8000A00000043420020006401000A00000006
:1014C8003F42002000FF01000A0000003E420020C9
:1014D80000FF01000A0000003A4100200000F4016A
:1014E80001000000384100200000F4010100000064
:1014F800364100200000F4010100000034410020C2
:101508000000F401010000003A4200201400E80342
:101518000100000038420020E80330750100000097
:101528003742002000C801003642002000C80100F0
:101538003542002000C80100344200200064010048
:101548000A0000003342002000FF01000A000000EA
:101558005342002000C801005242002000C8010088
:101568005142002000C801005042002000C801007C
:101578004F42002000C801004E42002000C8010070
:101588004D42002000C801004C42002000C8010064
:101598004B42002000C80100406C04080000000015
:1015A800000000000000000000000000506C04086B
:1015B8000900000000000000840C00200400000066
:1015C800586C04080900000000000000780C002096
:1015D80004000000E46F0408090000000000000097
:1015E8006C0C0020040000009C680408090000003E
:1015F80000000000600C002004000000606C04087B
:101608000900000000000000540C00200400000045
:10161800686C04080900000000000000480C002065
:1016280004000000706C04080900000000000000BD
:101638003C0C002004000000786C0408090000003D
:1016480000000000300C00200400000010670408AF
:101658000100000000000000000000000000000081
:10166800000000000D000000000000000000000065
:1016780000000000786D0408000000000000000071
:101688000000000000000000FC69040800000000E1
:10169800000000007B0B002004000000986804088C
:1016A8000C000000C5460208D80C0020000000000D
:1016B800046804080C000000BD400208CC0C00209F
:1016C80000000000246704080C000000A140020884
:1016D800C00C002000000000786804080800000022
:1016E80000000000B40C0020040000006868040832
:1016F8000C000000ED3F0208A80C002000000000CC
:10170800846D040809000000000000009C0C002003
:10171800040000000C67040803000000D9E2020876
:10172800900C002000000000106704080100000071
:1017380000000000000000000000000000000000A1
:101748000D00000000000000000000000000000084
:101758008C6D04080000000000000000000000007C
:10176800000000009C6D04080C0000000000000050
:10177800F00C002000000000A46D04080A0000001E
:1017880000000000EE42002000000000B06D0408D8
:101798000A00000000000000F642002000000000DF
:1017A800B86D04080A00000000000000FE42002096
:1017B80000000000C06D04080800000000000000E0
:1017C800E40C00200000000010670408010000007D
:1017D8000000000000000000000000000000000001
:1017E8000D000000000000000000000000000000E4
:1017F800C86D0408000000000000000000000000A0
:1018080000000000DC6D04080C000000000000006F
:10181800080D002000000000EC6D04080400000022
:10182800CDE602080000000000000000F46D040886
:101838000C00000000000000FC0C0020000000006C
:10184800086E040804000000ADE60208000000006D
:1018580000000000106704080100000000000000FC
:101868000000000000000000000000000D00000063
:10187800000000000000000000000000106E0408D6
:101888000000000000000000000000000000000050
:10189800246E04080700000000000000440D00202A
:1018A80000000000306E040808000000000000007E
:1018B800380D0020000000003C6E040808000000FD
:1018C800000000002C0D002000000000486E0408F5
:1018D8000800000000000000200D002000000000AB
:1018E800546E04080800000000000000140D0020D9
:1018F800000000001067040801000000000000005C
:101908000000000000000000000000000D000000C2
:10191800000000000000000000000000606E0408E5
:101928000000000000000000BF0B002000000000C5
:101938006C6E04080B00000000000000BC0D0020C5
:1019480000000000746E04080B0000000000000096
:10195800B00D002000000000806E04080B0000009D
:1019680000000000A40D0020000000008C6E040898
:101978000B00000000000000980D0020000000008F
:10198800986E04080B000000000000008C0D002079
:1019980000000000A46E04080B0000000000000016
:1019A800800D002000000000AC6E04080B00000051
:1019B80000000000740D002000000000B86E04084C
:1019C80007000000000000006C0D0020000000006F
:1019D800C06E04080700000000000000640D00202D
:1019E80000000000CC6E04080B000000000000009E
:1019F800580D002000000000D86E04080800000000
:101A0800000000004C0D00200000000010670408D2
:101A180001000000000000000000000000000000BD
:101A2800000000000D0000000000000000000000A1
:101A380000000000E46E0408000000000000000040
:101A48000000000000000000F86E04080800000014
:101A580000000000EC0D002000000000046F0408E6
:101A68000800000000000000E00D00200000000059
:101A7800106F04080800000000000000D40D0020CA
:101A8800000000001C6F04080800000000000000AF
:101A9800C80D0020000000001067040801000000C5
:101AA800000000000000000000000000000000002E
:101AB8000D00000000000000000000000000000011
:101AC800246F04080000000000000000BC0B002088
:101AD80000000000346F04080B0000000000000044
:101AE800340E002000000000406F04080B000000C6
:101AF80000000000280E0020000000004C6F0408C1
:101B08000700000000000000200E00200000000078
:101B1800586F04080700000000000000180E00209D
:101B280000000000646F04080700000000000000C7
:101B3800100E002000000000706F0408080000006C
:101B480000000000040E002000000000786F040868
:101B58000800000000000000F80D00200000000050
:101B680010670408010000000000000000000000E9
:101B780000000000000000000D0000000000000050
:101B88000000000000000000806F04080000000052
:101B980000000000BC0B0020000000008C6F04084F
:101BA8000700000000000000800E00200000000078
:101BB800946F04080700000000000000780E002061
:101BC800000000009C6F04080700000000000000EF
:101BD800700E002000000000A46F04080700000039
:101BE80000000000680E002000000000AC6F040830
:101BF8000700000000000000600E00200000000048
:101C0800B46F04080700000000000000580E002010
:101C180000000000BC6F040807000000000000007E
:101C2800500E002000000000C46F040807000000E8
:101C380000000000480E002000000000CC6F0408DF
:101C48000700000000000000400E00200000000017
:101C580010670408010000000000000000000000F8
:101C680000000000000000000D000000000000005F
:101C780000000000000000000000000059DF02081A
:101C8800880E0020304100201B000000282B04088B
:101C98002F4100200A3201002E41002001FA0100E4
:101CA8002A41002000C8010028410020E803D0078D
:101CB8000100000046344259000000002940020893
:101CC80000000000640F0020C1E3020891E102084F
:101CD800401000206FDF020800000000E010002024
:101CE800F5DF0208C5DF02086C1100207DE002085C
:101CF800C1E002080C1200203C4200200103010050
:101D0800A1DF02087DDF02082413002025E0020875
:101D1800EDE60208B0130020F1E0020845E70208EA
:101D2800781400203242002001030100D46F040817
:101D3800000000000000000000000000000000009B
:101D4800E06F04080800000000000000981500205B
:101D580000000000E86F0408070000000000000011
:101D68009015002000000000F86F0408070000002C
:101D7800000000008815002000000000047004081E
:101D8800070000000000000080150020000000008F
:101D9800107004080C0000000000000074150020FA
:101DA800000000001C70040803000000D9E20208CB
:101DB80068150020000000001067040801000000FA
:101DC800000000000000000000000000000000000B
:101DD8000D000000000000000000000000000000EE
:101DE800247004080000000000000000000000004B
:101DF80000000000347004080A0000000000000021
:101E0800243E0408000000003C7004080A0000009A
:101E180000000000983D0408000000004470040819
:101E28000A000000000000005442002000000000EA
:101E38004C7004080A00000000000000A4150020EF
:101E48000000000010670408010000000000000006
:101E58000000000000000000000000000D0000006D
:101E6800000000000000000000000000547004089A
:101E7800000000000000000000000000000000005A
:101E88006870040803000000D9E20208B8150020B1
:101E9800000000007470040803000000D9E2020882
:101EA800C8000020000000007C7004080300000047
:101EB800D9E20208AC1500200000000010670408F1
:101EC8000100000000000000000000000000000009
:101ED800000000000D0000000000000000000000ED
:101EE80000000000847004080000000000000000EA
:101EF80000000000000000009070040807000000C7
:101F080091E7020814160020000000004874040835
:101F180003000000D9E202080816002000000000B3
:101F28009C70040803000000D9E20208FC15002098
:101F380000000000A470040803000000D9E20208B1
:101F4800F015002000000000AC7004080700000035
:101F580075E70208E8150020000000002068040862
:101F680003000000D9E20208DC1500200000000090
:101F7800B870040803000000D9E20208D015002058
:101F880000000000C470040803000000D9E2020841
:101F9800C4150020000000001067040801000000BC
:101FA8000000000000000000000000000000000029
:101FB8000D0000000000000000000000000000000C
:101FC80021DF0208E9DE02081C1600205DE1020894
:101FD80000000000D01600200000000000000000F3
:101FE8005C17002035E10208ADE70208D41700208D
:101FF800D07004080000000000000000000000008D
:1020080000000000D468040803000000D9E20208B8
:10201800D418002000000000DC7004080300000051
:10202800D9E20208C818002000000000E87004087F
:1020380003000000D9E20208BC18002000000000DC
:10204800F470040803000000D9E20208B018002068
:1020580000000000FC700408020000002DE80208DF
:1020680000000000000000000471040802000000E5
:102078002DE80208010000000000000010710408AB
:10208800020000002DE80208020000000000000025
:10209800000000000D00000000000000000000002B
:1020A8000000000001000000742E04080508040068
:1020B80000000000F0250408BC2A0408DC250408F8
:1020C80000000000A02E040805080A000000000017
:1020D800F0250408BC2A0408E42A040800000000CB
:1020E800040309041201000202020040830440575D
:1020F8000002010203010000F18C02081992020893
:102108006D8D0208BD8602083D890208CD86020849
:10211800E986020895860208858602080000000004
:102128000000000000600240106002400000000053
:10213800000B00000000200000000000000000006C
:10214800006002402860024000000000060C000009
:1021580000002000000000000000000000600240B5
:102168004060024000000000100D00000000200048
:1021780000000000000000000060024058600240BB
:1021880000000000160E0000000020000000000003
:102198000000000000600240706002400000000083
:1021A800200F0000000020000000000000000000D8
:1021B8000060024088600240000000002610000015
:1021C8000000200000000000000000000060024045
:1021D800A060024000000000301100000000200054
:1021E800000000000000000000600240B8600240EB
:1021F80000000000362F0000000020000000000052
:10220800000000000064024010640240000000006A
:10221800003800000000400000000000000000003E
:1022280000640240286402400000000006390000F3
:1022380000004000000000000000000000640240B0
:102248004064024000000000103A00000000400016
:1022580000000000000000000064024058640240D2
:1022680000000000163B00000000400000000000D5
:10227800000000000064024070640240000000009A
:10228800203C0000000040000000000000000000AA
:1022980000640240886402400000000026440000F8
:1022A8000000400000000000000000000064024040
:1022B800A06402400000000030450000000040001B
:1022C800000000000000000000640240B864024002
:1022D800000000003646000000004000000000003A
:1022E80000000000CD8B0208E9B6020839B60208E2
:1022F8000000000099B202088DB502080DB6020868
:10230800F5B4020800000000000000008DB20208C9
:102318009D2903089B290308992903089329030881
:10232800912903089729030895290308AD2903086B
:102338009F290308BD2A0308D12A0308A92A0308EC
:10234800952A0308812A0308010000000000803F45
:102358000000000000000000000000000000803FB6
:102368000000000000000000000000000000000065
:102378000000000000000000000000000000000055
:10238800000000000000803F000000000000000086
:10239800000000000000803F00010101685E0C00A1
:1023A80001000000981C0020000000000000000050
:1023B8000000000000000000000000000000000015
:1023C8000000000000000000000000000000000005
:1023D80000000000000000000000000000000000F5
:1023E80000000000000000000000000000000000E5
:1023F80000000000000000000000000000000000D5
:102408000000000000000000430000000000000081
:1024180000000000000000000000000000000000B4
:102428000000000000000000430000000000000061
:102438000000000000000000000000000000000094
:102448000000000000000000430000000000000041
:102458000000000000000000000000000000000074
:102468000000000000000000430000000000000021
:102478000000000000000000000000000000000054
:102488000000000000000000430000000000000001
:102498000000000000000000000000000000000034
:1024A80000000000000000004300000000000000E1
:1024B8000000000000000000000000000000000014
:1024C80000000000000000004300000000000000C1
:1024D80000000000000000000000000000000000F4
:1024E80000000000000000002BF9030807F90308AA
:1024F80000000000FB7604080F6C04085A51040819
:102508005A5104085A5104085A5104085A510408E7
:102518005A5104085A5104085A5104085A510408D7
:10252800FFFFFFFFFFFFFFFFFFFFFFFFFFFF0000B1
:102538000100415343494900000000000000000029
:102548000000000000000000000000000000000083
:10255800000041534349490000000000000000000A
:102568000000000000000000000000000000000063
:0825780000000000010000005A
:10800000002870B51EDB0928044620DD012303EBA0
:1080100083035B00B0FBF3F2092AF8D87BB10E4E64
:10802000B4FBF3F00928CCBF57223022A6FB03E5AE
:10803000024403FB1044EB0801F8012BF0D10023AC
:108040000B7070BD2D230B7040420131DBE73030E7
:1080500001F8010BF3E700BFCDCCCCCC884230B4A3
:108060004FF001042ED301FB04F4B0FBF4F58D4274
:10807000F9D284B1AAB901E0B0FBF4F5092DCCBF67
:10808000572230222A4404FB150003F8012BB4FBCD
:10809000F1F4002CF0D100221A7030BC7047B0FB14
:1080A000F4F5092DCCBF372230222A4404FB1500F9
:1080B00003F8012BB4FBF1F4002CF0D100221A706C
:1080C00030BC70470546002AEBD1D7E72DE9F047D1
:1080D00014461D46064600234FF47A722046294670
:1080E00037F08AF8DFF840814B4A4C4F88FB00316B
:1080F0000144C31782FB002EC3EB611188FB0128EA
:1081000087FB00278644464AC3EBEE2EC1EB011CD9
:1081100082FB0E29A0EB8C0C0744424A86F806C06D
:10812000C3EB27474FEAEE7C08EB010ACCEBA90C26
:1081300082FB07824FEAE1780CEB4C0CC8EB6A1823
:10814000AEEBCC0EC8EB0818DFF8E0C086F804E010
:10815000A1EB880171718CFB0010F917C1EBE212E1
:1081600040F2B55101FB1272C3EBE050B2F5896FDA
:108170004FEA80073CDA40F2DA239A4242DCB2F559
:10818000B77FB4BF4FF0000C4FF0010C4FEA4C0921
:10819000DFF89C8009EB0C0308EBC3031FFA8CFE8D
:1081A000D88A09EB0C0108EBC10116310B2301E061
:1081B00031F8020D824218DA013BF9D1CC44012397
:1081C00038F83C00B37007F2B2770132121ABE449D
:1081D000F270A6F800E0204629464FF47A72002398
:1081E00037F00AF83281BDE8F0870133DBB2E9E706
:1081F0004FF0030EF44640F29650DFF834804FF013
:108200000609CEE74FF0020EDFF82480F44640F274
:1082100029404FF00409C4E7C5B3A29107452EC217
:10822000ABAAAA2A73B06D1689888888792D0311A4
:10823000500A040803685A1C02601970704700BF96
:108240002DE9F047089C2578002B804689460CBF15
:108250004FF0200A4FF0300A661C35B3002A29DDA2
:10826000334601E0024698B113F8011B501E002965
:10827000F8D1971E60B13D46013D51464046C84782
:108280006B1C002BF8DC257827EAE770013055B12C
:10829000041B29464046C847301916F8015B002DDB
:1082A000F7D1BDE8F087BDE8F087002A04DC284656
:1082B000BDE8F0870020EBE7571EDCE783684268E3
:1082C000D0ED037A00EB83010133934281ED040A80
:1082D000836004BF0023836000EB830393ED047A83
:1082E000036870EE277A9A42C0ED037A77EEC77A78
:1082F000C0ED037A0CDA013307EE103AF8EEC76AE4
:10830000B7EE007A87EEA60A036030EE070A7047E0
:1083100007EE102AB8EEC77A87EE870A704700BFCB
:1083200090ED057A90ED004AD0ED066AD0ED014A55
:10833000D0ED047A90ED035AD0ED025AA4EE007A03
:10834000B0EE406AB0EE470AB0EE667AA6EE247A46
:1083500067EEC07AA0EE457AE6EE257A80ED057AE2
:10836000C0ED067A704700BFD0ED057A90ED013A76
:10837000D0ED003AD0ED064A90ED024A90ED077A32
:1083800090ED035A90ED086AD0ED045AC0ED067ADC
:10839000F0EE406A27EE830AC0ED056AA3EEA60A56
:1083A00080ED087AA4EE240AA5EE470AA5EEC60AD7
:1083B00080ED070A704700BFD0ED007A90ED017A9A
:1083C00030EE670AE7EE007AB0EE670AC0ED007A99
:1083D000704700BF704700BF0A44914214D030B4C8
:1083E0000139551E41F2210211F8014F082380EA9C
:1083F000042004044CBF82EA40004000013B80B2EC
:10840000F7D18D42F0D130BC70470378407840EA14
:10841000032010FB01F04FF4807190FBF1F000F3AA
:108420000F0000B270472DE9F04F654B654EB3F871
:108430000AC03468B3F8048087B04FEA0C2A05906C
:108440001889B4EB0A0A4FF000024FF0000565EB03
:10845000020BA0FB0A4500FB0B55E00940EA456012
:108460004FEA084407198E46D8884FEAE51141EBD8
:108470000208A0FB0A45CDE90278B3F8028000FBB0
:108480000B55200A40EA05604FEAC83410EB040897
:108490004FEA252141EB02099A89A2FB0A0102FB5E
:1084A0000B11C20D42EA412212F5FA604FEAE15384
:1084B00043F10001B0F5FA6FCDE9000171F100015F
:1084C000B4465EDA0524A2FB040104FB031100FBA1
:1084D00003F402FB0144DDE90267A0FB0201214431
:1084E0004D104FEA3004361B4FEA900444EA817481
:1084F00067EB05078D10B8EB040869EB0509DDE9AA
:10850000004531484FF0FF31844275EB0101CDE960
:10851000026723DA40F6AC5012184FF000014B41CD
:1085200002FB03F1A2FB022303EB4103D900D000BD
:10853000101A41EA527163EB0101341847EB01054F
:10854000CDE902450B24A2FB040104FB03114910F1
:108550004FEA3000B8EB000869EB01090AFB0BF3A6
:10856000DDE90001AAFB0AAB0BEB430B4FEADA7221
:1085700042EA4B02801A4FEAEB7361EB0301CDE94B
:108580000001DCF80410A1FB082301FB0933540DA2
:108590005D1544EAC324DDE90223A21A65EB030357
:1085A0001D46D30B059A43EA454302B11360BEF161
:1085B000000F02D0009BCEF8003007B0BDE8F08F6E
:1085C000E0B10020681E002024FAFFFF4FF4805322
:1085D00083827047012380F845307047BFF34F8F87
:1085E0000549064BCA6802F4E0621343CB60BFF34F
:1085F0004F8F00BFFDE700BF00ED00E00400FA056B
:1086000070B4037B04681F2B08D9203B20216268CB
:1086100001FA03F31A421CD170BC70472021226872
:1086200001FA03F31A42F7D0426914495C2000FBB7
:10863000021251685689CD680868296821F0010145
:108640002960828992B222EA06028281A36070BC0C
:108650007047426909495C2000FB02125168568943
:10866000CD680868296821F001012960828992B2E9
:1086700022EA06028281E36070BC70474C7C0020D5
:108680002B4B1978002951D02A4B30B41C6898889C
:1086900000226262A5899A80284380B20129A081C4
:1086A00043D09C6898896262A589284380B20229D8
:1086B000A0819A8139D01C69988A6262A589284371
:1086C00080B20329A0819A822FD09C69988B626224
:1086D000A589284380B20429A0819A8325D01C6AE9
:1086E000988C6262A589284380B20529A0819A846A
:1086F0001BD09C6A988D6262A589284380B20629A6
:10870000A0819A8511D01C6B988E6262A58928433E
:1087100080B20729A0819A8607D0986B998F426210
:108720008489214389B281819A8730BC704700BF18
:108730002C7F0020307F0020F0B5C400221892006A
:10874000AE498B585B689D8AADB2EEB2F7070A441A
:108750005CD4B70732D5BFF35F8F167EF6B2012E19
:1087600000F0C780A64D1A8BBFF35F8F221801EB74
:108770008202167E022E00F0D580221801EB8202C2
:10878000167E032E00F088809A8895F9086092B2D0
:1087900042F480629A80221801EB8202127E01323A
:1087A00096425BD1AA7A00266E72002A40F095802C
:1087B000204401EB800000234375F0BD77074ED4C1
:1087C00016F0400600F0C9808D4D1E8A95F908E02C
:1087D000176AF6B207F80E605FFA8EFE0EF1010C12
:1087E0004FFA8CFC177E85F808C00CF10302974203
:1087F000664600F01C81221801EB8202127E94452D
:10880000C9D10EF1020676B22E72C4E71E887C4DE5
:1088100026F400663604360C1E801E88B6B246F476
:1088200080661E80967E00272F72002E48D06E7ABA
:10883000002E42D0221801EB82020126127E6E72B7
:10884000022A00F0B980221801EB8202927D42F0E8
:1088500001021A82204401EB8000037EF0BD684DC6
:10886000967E0127AF72002E73D06E7A002E7BD1D8
:10887000221801EB8202527E002A00F0A3801A889F
:108880002E7A92B2013642F4007276B21A802E72BB
:108890001A88D205FCD47EE7927E002A3FF474AF9A
:1088A0006A7A002A3FF470AF9A8895F9086022F43A
:1088B00080621204120C9A806DE7D27DFF2AB9D033
:1088C000221801EB8202967D06F0FE061E82D37D01
:1088D000FF2BBFD0FF232B72BCE79A8822F4407293
:1088E00012042044120C01EB80009A80002343758F
:1088F000F0BD927E424D002A3FF435AF6A7A002ADD
:108900003FF431AF1A8822F480621204120C1A80EC
:10891000BFF35F8F1A8B1A88AE7292B242F4007264
:108920001A8031E7927E002A3FF427AF6A7A002A44
:108930003FF423AF1A8895F9086022F4806212048C
:10894000120C1A809A8822F480621204120C9A8007
:1089500021E76A7A002A8BD091E715F0800F284D25
:108960003AD195F9086016E7167ED2F820E01F8804
:10897000022E95F9086045D927F480673F043F0C23
:108980001F801F8AFFB20EF806701F88D2F820E001
:10899000BFB247F400771F80F2B21F8A561C76B22E
:1089A000FFB20EF806709F88961CBAB276B242F4F7
:1089B00080622E729A806BE71A8892B242F400624B
:1089C0001A8040E71A8895F9086092B242F48072E2
:1089D00001271A806F725BE795F90870B7F1FF3FC6
:1089E0002CD0D669F65D1E8292F818E001377AB273
:1089F000964516462A727FF4CEAEA3E72861002082
:108A0000681E0020BFB247F400771F801F8AFFB2A4
:108A10000EF80670F6B21F8AD2F820E0721C52B22D
:108A20000336FFB276B20EF802702E7230E79A88E3
:108A300022F480621204120C9A80DCE6D77D1F8239
:108A40002E72957E1DB9127E002A7FF403AF9A889C
:108A500022F480621204120C9A80FBE60023436029
:108A6000036083602A2343702B2303710123C371A6
:108A700083727047F8B50468C4F30D0405460E46CA
:108A800004B32F6820F022FE092840F08880454C6E
:108A9000236923F440732361236943F40073236142
:108AA000236943F0010323613E6020F00FFE236938
:108AB000092823F00103236171D12B6804332B6053
:108AC0000020F8BD384B394A93422BD902F5804239
:108AD000934226D902F5804293422AD902F5804278
:108AE000934228D902F58032934226D902F500320A
:108AF000934224D902F50032934222D902F5003282
:108B0000934220D902F5003293421ED902F5802209
:108B100093421CD9B3F1016F1BD3052003F052FD22
:108B2000FBE7082420F0D2FD092814D04FF0FF30D5
:108B3000F8BD1024F6E71824F4E72024F2E72824EF
:108B4000F0E73024EEE73824ECE74024EAE7482455
:108B5000E8E75824E6E7134F3B6923F440733B6191
:108B60003B6943F400733B613B6923F0F8033B61CD
:108B70003B6943F002031C433C613B6943F480338F
:108B80003B6120F0A3FD3B6923F002033B613B699D
:108B9000092823F0F8033B613FF473AFC6E76FF099
:108BA0000100F8BD003C024000400008FF3F000803
:108BB000F8B504460D468E180027B54201D120694C
:108BC000F8BDE368591CE160234415F8012B1A72C3
:108BD0000429F2D1206918B9A1682046FFF74AFF9D
:108BE0002061E760E9E700BF014B186805F0ECB9C8
:108BF000CC1F0020F8B5057B466903681F2D29D9D5
:108C0000A5F120045F682021A1400F422A4613D01D
:108C10001022A240D960DA605A68E240D10703D539
:108C2000012202FA04F4DC600446304605F058F9EB
:108C3000227B23681F2A20D9A2F1200008215A682C
:108C40008140114200D0D9600422596882400A4212
:108C500021D1F8BD20211C68A9400C422A460CD025
:108C60001022AA4099609A601A68EA40D207DBD5C0
:108C7000012202FA05F59D60D6E7082118689140A7
:108C8000014200D099600421186801FA02F2024200
:108C900003D09A60F8BDDA60F8BDF8BD08B504F0FD
:108CA000DDFA40B12D2282710022C2712021BDE87F
:108CB000084005F003BB08BD0E4B98420AD0A3F54F
:108CC0007843984211D003F5806398420FD04FF05B
:108CD000FF3070470022084B03EB02135A89013220
:108CE00092B25A81588980B270470122F3E702227A
:108CF000F1E700BF00300140ACB10020F0B587695A
:108D000083B0064617B13B68BA885A837069DFF8AA
:108D1000A4E08389C3244FF47A734FF0060C6D46A8
:108D20004FF6FF710EF1010E03E0013B9BB28B4247
:108D300020D002899207F8D5A3B283814FF47A73C9
:108D400002E0A3B28B4215D00289D20703F1FF34AF
:108D5000F7D5828992B20DB12A700135BCF1000FAE
:108D60000BD00CF1FF3CFF24BEF1000FE1D09EF8C8
:108D70000040D7E7FFF7A0FFB76917B13B68BA8893
:108D80001A839DF805009DF801509DF802109DF88A
:108D900003409DF804209DF8063041EA052143EA8E
:108DA000002342EA0422012031877287B38703B08F
:108DB000F0BD00BFB00A0408F8B584894FF6FF760D
:108DC0004FF47A7433B319B30F78013101E0B44230
:108DD00018D00589013CAD07A4B2F8D5BCB2848196
:108DE0004FF47A7402E0BCB2B4420BD00589ED07AF
:108DF00004F1FF37F7D58589ADB20AB1157001329C
:108E0000013BDFE7FFF758FF003018BF0120F8BD36
:108E1000FF27DEE70120F8BD08B540F2E93300E0A6
:108E2000A3B10289013B12F0020F9BB2F8D089B2C4
:108E3000818140F2E93300E043B10289013B12F045
:108E4000010F9BB2F8D08089C0B208BDFFF734FF94
:108E5000C0B208BD427A02B9704710B50446036833
:108E6000406804F10A0198470023637210BD00BFF7
:108E7000437A5A1C0344D2B242729972037A9342E3
:108E800000D802B9704710B504460368406804F181
:108E90000A0198470023637210BD00BF50B301233D
:108EA000302803FA01F122D0312820D032281ED0F8
:108EB00033281CD034281ED035281CD020281AD0A6
:108EC000212818D0102812D0112810D012280ED026
:108ED00013280CD014280ED015280CD0162801D039
:108EE000172806D111F0030018BF012070474A0768
:108EF00003D1002070478B07FBD00120704700BFD3
:108F0000302829D0312829D0322829D0332829D017
:108F1000342829D0352829D0202829D0212829D023
:108F2000102829D0112829D0122829D0132829D077
:108F3000142829D0152829D0162805D0172808BFAD
:108F40000F2302D0002070470E23114A03EB430386
:108F5000134493F86A0070470023F6E70123F4E70F
:108F60000223F2E70323F0E70423EEE70523ECE70F
:108F70000623EAE70723E8E70823E6E70923E4E70F
:108F80000A23E2E70B23E0E70C23DEE70D23DCE70F
:108F9000500A040870B5448806460D46C4F30B0415
:108FA00022460021284637F0E3FC3369094A934200
:108FB00009D3094A934206D2224628461946BDE8FB
:108FC000704037F0B0BC23B121462846BDE8704060
:108FD000184770BD180600081807000838B5054C7A
:108FE000054DAC4200D338BD61682046FFF7D2FF83
:108FF0001434F6E79001000818060008064B0749EC
:109000008B4202D30023184670471A88C2F30B0222
:109010009042F8D01433F3E79001000818060008D6
:10902000024A136823EA000010607047AC870020F2
:10903000F8B5174D2B78A52B28D16B78BE2B25D1F1
:10904000022229464FF6FF70FFF7C6F9114FAC1CFC
:1090500022884AB1A618BE4218D2052A16D921463E
:10906000FFF7BAF93446F3E721460222FFF7B4F9D5
:109070000222A118FFF7B0F90634074B641B1C80CD
:1090800041F60F53C31A58425841F8BD0020F8BDAD
:109090000040000800800008A42D00202DE9F04FBA
:1090A000DFF84C914D4F8BB00326A7EB0907182230
:1090B000002104A837F05CFC494BCDF810900597CF
:1090C0001A69002A04DA474A5A6002F188325A6063
:1090D00001228DF82420F322DA60434B434C1B8895
:1090E000ADF800300222694604A8FFF761FD0222B4
:1090F00069464FF6FF70FFF76FF9DFF8F8A080467A
:109100004FF0000B544539D30AAC002524F8245DF8
:109110000222214604A8FFF74BFD022221464046C9
:10912000FFF75AF940BAC043ADF80800022202A97D
:1091300004A8FFF73DFD079878B106ABC0F1040223
:109140002946184437F014FC089818B9069904A861
:10915000FFF790FC0023089007939DF82430089AAD
:1091600023B11F490B6943F000430B61013E2DD031
:10917000002A9CD1FFF75CFF50B32CE065888DF886
:109180000DB0C5F30B05AB1DADF808302388C3F354
:109190000B02ADF80A201B0B062202A904A88DF8C9
:1091A0000C30FFF705FD062202A94046FFF714F92F
:1091B000616880462A4604A8FFF7FAFC61684046C9
:1091C0002A46FFF709F9143480469BE7002AD1D0DC
:1091D000052003F0F7F90BB0BDE8F08F0080000820
:1091E000003C024023016745E80A0408900100089A
:1091F00000400008180600080378202B024600F102
:109200000100F9D0092BF7D02D2B2CD02B2B03BF2D
:109210005378B7EE000A0246B7EE000AA3F1300118
:10922000C8B209289FED467A10D8F2EE046A07EE1C
:10923000901AF8EEE77A12F8013FE7EE267AA3F1EA
:109240003001C8B20928B0EE677AF0D92E2B4CD085
:1092500003F0DF03452B0BD0F7EE007A67EE276AA9
:1092600020EE260A70475378BFEE000A0246D5E783
:1092700010B451782D2959D02B290ABF9178501C50
:10928000901C0024A1F13003092B53D8002303EBD9
:10929000830301EB430310F8011FA1F13002092AF7
:1092A000A3F13003F3D9B3F59A7F28BF4FF49A7333
:1092B000072B42D9DFED236A1A46F7EE007A083A07
:1092C000072A67EEA67AFAD803F007032BB1F2EE6D
:1092D000046A013B67EEA67AFBD124B3C7EE276A86
:1092E0005DF8044B20EE260A70475378A3F1300155
:1092F000C8B2092802F10102AAD8F2EE046AF0EE1F
:10930000665A07EE901AF8EEE77A12F8013F87EEF8
:10931000A66AA3F13001C8B2092866EEA56A37EE45
:10932000067AEED994E767EE276AD9E7901C917820
:109330000124A7E7F7EE007ACFE7F7EE007AC5E75A
:109340000000000020BCBE4CB5EEC00ADFED317A53
:10935000F1EE10FACCBF30EE270A30EE670ADFEDEF
:109360002E7A20EE270A30B5FDEEC07A87B017EED0
:10937000904A054684EAE470002303A9A0EBE47058
:1093800001930093029332F05CFB002CACBF2023CE
:109390002D2303A88DF8003035F084FA012803A9A5
:1093A00024D002282DD0032805BF30236846684604
:1093B0008DF8013037F0E4FA684635F073FA033877
:1093C000C4B222466946284637F011FB00232B55CC
:1093D000284635F067FA2E22431C2A540DEB04016F
:1093E000E81837F0EAFA284607B030BD302368465F
:1093F0008DF801308DF802308DF8033037F0C0FA67
:10940000DAE7302368468DF801308DF8023037F006
:10941000B7FAD1E76F12033A00007A442DE9F04120
:10942000064615460846B6FBF2F43CB905FB146443
:10943000124B1B5D00F8013BBDE8F081B4FBF2F775
:1094400067B90E4B05FB174705FB1464DA5D00F89E
:10945000012B1B5D00F8013BBDE8F081B7FBF2F882
:10946000B8F1000F02D04046FFF7D8FF05FB18788F
:10947000024B13F8082000F8012BE3E7B03C040886
:10948000104B2DE93048D3E9004554EA05020BD1D1
:109490000346012200201871587198719A70DA7091
:1094A00018801881BDE83088074B1A6814EB020B4E
:1094B00045F1000C5A466346FEF708FE0120BDE860
:1094C000308800BF40250020ACB40020F0B40288F2
:1094D0008578154FC37804794179A2F2B27202F00F
:1094E000030606EB4606013D05EB8605013B37F812
:1094F00015608579008940F2B557920807FB023262
:10950000931903EB430304EBC303C3EB031301EB16
:109510008303C3EB031305EB830300214FF47A723B
:10952000C2FB0301F0BC7047500A0408FAB170B4E2
:109530008E18044603E0101A14D1B14214D014F866
:10954000012BA2F14103192B11F8013BA3F14105B5
:1095500098BF2032192D03F12000ECD9D01A01D187
:10956000002BEAD170BC7047002070BC70471046D9
:10957000704700BF4FF0FF32FFF7D8BFA0F1610383
:10958000192B98BF20387047A0F14103192B98BFC1
:1095900020307047202805D0093804288CBF0020CF
:1095A0000120704701207047613819288CBF0020C6
:1095B00001207047413819288CBF002001207047D6
:1095C000303809288CBF002001207047A0F13003FB
:1095D000092B07D920F02000413819288CBF002022
:1095E000012070470120704730B402681146531CB7
:1095F000036011F8024B0160D31C5178036093782B
:10960000151D05601B0443EA0123D078234343EA78
:10961000006030BC704700BF0368591C1A460160E7
:1096200012F8021B0260587841EA0020704700BF20
:1096300003685A1C02601878704700BF38B50446AA
:109640000068154637F06FF922682A44226038BD59
:10965000036810B40A0E5C1C04601A7003680A0CDC
:109660005C1C04601A7003680A0A5C1C04601A70AF
:1096700003685A1C026019705DF8044B704700BF04
:10968000036810B40A0A5C1C04601A7003685A1C50
:10969000026019705DF8044B704700BF03685A1CE4
:1096A000026010B4197003680A0A5C1C04601A7026
:1096B00003680A0C5C1C04601A700368090E5A1CCB
:1096C000026019705DF8044B704700BF03685A1CB4
:1096D000026019700368090A5A1C02601970704709
:1096E0002DE9F047002488B080460F461E46A1466B
:1096F00005AD531C0393117839B3252933D1931C3D
:10970000CDF810900393507830284ED04FF0000AD7
:10971000A0F13003DBB2092B42D96C2819D06428A0
:1097200000F0938024D825281CD063D9582876D0FF
:1097300063281BD131784046B847039A531C0393E2
:109740001178043601340029D7D1204608B0BDE88D
:10975000F087039B5A1C03921B78642B7CD02AD879
:10976000252B54D1252140460134B847039AC0E740
:10977000732833D044D975284FD106F1040E3068D0
:109780002B4600220A217646FEF768FC049A0095D3
:10979000534639464046FEF753FD039A0444A8E772
:1097A00004AA03A932F02AF9B7E7D31C03939078EF
:1097B0004FF0010AACE7732B10D05BD9752B3AD070
:1097C000782B96D1A3F15802B2FA82F2306852098E
:1097D0002B4610210436FEF741FCD7E73368049A84
:1097E0000093394600234046FEF72AFD0436044420
:1097F000039A7EE70028B9D1204608B0BDE8F0877B
:109800006E28B3D1039A336804361C6071E72AD9F5
:10981000582BD7D0632B8DD06BE77828A6D1A0F139
:109820005802B2FA82F2306852092B461021FEF734
:1098300015FC0436AAE706F1040E30682B46002218
:109840000A217646FEF70AFCA0E7331D3068294658
:109850001E46FEF7D5FB99E7331D306829461E46A4
:10986000FEF7CEFB92E7002B7FF443AF204608B013
:10987000BDE8F0876E2BC6D03BE700BF0EB400B545
:1098800084B005AB019053F8042B0649039301A85B
:10989000FFF726FF019B00221A7004B05DF804EB6D
:1098A00003B07047358200082DE9F047484BB3F903
:1098B0000C708CB00646002F56D13D463C460A88B7
:1098C00040F2B1739A4203D98B78581E0B282FD9D6
:1098D000002301201946ADF824308DF828308DF88A
:1098E00029308DF82A30ADF82C309C469A4699469E
:1098F0001A46984686468DF826008DF827000346BE
:10990000002CACBF2B242D24049107950697CDF88D
:109910000CC0CDF808A0CDF80490CDF800E030469A
:1099200005942C49FFF7AAFF40460CB0BDE8F0872C
:1099300091F803E00EF1FF301E28C9D891F8049089
:10994000B9F1170FC4D891F805A0BAF13B0FBFD8F1
:1099500091F806C0BCF13B0FBAD80989B1F57A7FFE
:10996000B6D24FF00108CBE71B4C84FB0734E31958
:10997000FC17C4EB6314C4EB0415A7EB85052DB2EB
:10998000002D0846B8BF6D42FFF7A0FD4FF47A7274
:1099900000238046894635F02FFC3C2307FB030754
:1099A0004FF47A7200234046494635F025FC24B234
:1099B0004FF47A7192B20023C1FB072309A884EA0D
:1099C000E477FEF783FBA7EBE47709A977E700BF0D
:1099D000681E0020D83C0408898888880FB430B5F8
:1099E00083B006AB0A490B4853F8042B096800689A
:1099F0000193FFF775FE084C0546206804F0D0FA85
:109A00000028FAD0284603B0BDE8304004B07047C3
:109A1000EC600020F0600020CC1F0020DFED2B7AEE
:109A2000B4EEE70AF1EE10FA4ADDDFED296A9FEDA8
:109A3000297A01E0B0EE670AB4EEC70AF1EE10FA37
:109A400070EE667AF6DC9FED247AF4EEC77AF1EEDA
:109A500010FA38D5DFED1E6A9FED207A01E0F0EEB6
:109A6000407AF4EEC77AF1EE10FA37EEA60AF6D491
:109A7000DFED1B7AB4EEE70AF1EE10FA14DDDFED4C
:109A8000137A37EEC00A60EE006A9FED166A9FED0A
:109A9000167ADFED167AA6EE867A20EE266AE6EED4
:109AA000877AA6EE270A7047DFED117AB4EEE70A4F
:109AB000F1EE10FA44BFDFED087A37EEC00AE2E7B4
:109AC000F0EE407ABFE7B0EE670AD1E7DB0F49401E
:109AD000DB0FC940E4CB1641DB0F49C0E4CB16C114
:109AE000DB0FC93F92E741B99730083C15A82ABE61
:109AF000DB0FC9BF80EAE073A3EBE0738B4205DBA9
:109B0000002801DD401A704702D1704700207047DD
:109B10000844704709B909E0194690FBF1F301FBCD
:109B200013030846002BF7D1084670470146FBE7B0
:109B3000F0EEC07AB0EEE07AB4EEE77AF1EE10FA29
:109B4000B4BFB0EE676AB0EE476AB5EE406AF1EEB8
:109B500010FA46D0B4EEE77AF1EE10FA8CBFF0EED0
:109B6000675AF0EE475AC5EE866A9FED1F3A9FEDA1
:109B70001F6A9FED1F4A9FED1F5ADFED1F3ADFED71
:109B80001F4ADFED1F5AA6EEC36AE6EEA34AA6EE11
:109B9000864AB7EE006AA6EE845AA6EEA46AE6EEFE
:109BA000855AC5EE866AB4EEE77AF1EE10FA48BF40
:109BB000DFED147AF5EEC00A48BF77EEE66AF1EE03
:109BC00010FA48BFDFED107AB5EEC00A48BF77EE55
:109BD000E66AF1EE10FA48BFF1EE666AB0EE660A88
:109BE0007047DFED076ADEE739094E3DE3B59E3E7B
:109BF00088FA163E45FE7F3F99FB243F69A2163E38
:109C0000A7DFA834DB0FC93FDB0F4940DFED317A16
:109C100030EE277AFDEEC76A16EE903A2033402BDD
:109C200002D99FED2D0A7047B4EEE70AF1EE10FA63
:109C30004DDD9FED2A6ADFED2A6A01E0B0EE677A1A
:109C4000B4EEE67AF1EE10FA77EE467AF6DC9FEDA6
:109C5000257AF4EEC77AF1EE10FA35D5DFED1F6AFA
:109C60009FED217A01E0F0EE407AF4EEC77AF1EE52
:109C700010FA37EEA60AF6D4DFED167AB4EEE70A4C
:109C8000F1EE10FA1BDCDFED197AB4EEE70AF1EE23
:109C900010FA44BFDFED137A37EEC00A60EE006AB7
:109CA0009FED136A9FED137ADFED137AA6EE867AA5
:109CB00020EE266AE6EE877AA6EE270A7047DFEDE9
:109CC0000F7A37EEC00AE9E7B0EE670AD4E7F0EEA4
:109CD000477ABCE7DB0FC93F00000000DB0FC9403B
:109CE000E4CB1641DB0F49C0E4CB16C1DB0FC9BF83
:109CF00092E741B99730083C15A82ABEDB0F4940CE
:109D0000FDEEC07A17EE903A2033402B51D8DFEDAC
:109D10002D7AB4EEE70AF1EE10FA50DDDFED2A6A93
:109D20009FED2A7A01E0B0EE670AB4EEC70AF1EEC1
:109D300010FA70EE667AF6DC9FED257AF4EEC77ABB
:109D4000F1EE10FA38D5DFED206A9FED227A01E0BE
:109D5000F0EE407AF4EEC77AF1EE10FA37EEA60A8A
:109D6000F6D4DFED1D7AB4EEE70AF1EE10FA1BDC53
:109D7000DFED1A7AB4EEE70AF1EE10FA44BFDFED38
:109D8000147A37EEC00A60EE006A9FED156A9FED07
:109D9000157ADFED157AA6EE867A20EE266AE6EED3
:109DA000877AA6EE270A7047DFED067A37EEC00AFB
:109DB000E9E79FED0E0A7047B0EE670AD1E7F0EED3
:109DC000407AB9E7DB0F4940DB0FC940E4CB1641CD
:109DD000DB0F49C0E4CB16C1DB0FC93FDB0FC9BFA6
:109DE00092E741B99730083C15A82ABE0000000050
:109DF00007EE901AF8EE677A9FED837A27EE800AD5
:109E000020EE070AFDEEC07A17EE903A2033402B81
:109E100000F28C80DFED7D7AB4EEE70AF1EE10FA05
:109E200040F3E880B0EE407A9FED796ADFED796A21
:109E300001E0B0EE677AB4EEE67AF1EE10FA77EE72
:109E4000467AF6DC9FED747AF4EEC77AF1EE10FAFA
:109E500040F1CD809FED6E6ADFED706A01E0F0EEBB
:109E6000477AF4EEE67AF1EE10FA37EE867AF6D417
:109E7000DFED6B7AB4EEE77AF1EE10FA51DCDFED4C
:109E8000697AB4EEE77AF1EE10FA44BFDFED627A58
:109E900037EEC77A27EE076ADFED635ADFED637AA4
:109EA000DFED636A9FED635AE6EE257A67EE065AA8
:109EB000E6EE276AF7EE007AA5EEA67AF0EE675A8C
:109EC000E7EE055AE7EE457A87EEA55ADFED547ABC
:109ED00030EE277AFDEEC76A16EE903A2033402B1B
:109EE00029D99FED557AF6EE006AB7EE006AF7EED3
:109EF000004AC4EEA57A0023836143610362C36113
:109F000080ED045A67EEA66A27EE866A27EE877A06
:109F1000C0ED006AC0ED026A80ED016A80ED037A4F
:109F20007047DFED3A7A37EEC77AB3E7B7EE005AFB
:109F3000F0EE455ACAE7B4EEE70AF1EE10FA5FDD3B
:109F40009FED336ADFED336A01E0B0EE677AB4EE7D
:109F5000E67AF1EE10FA77EE467AF6DC9FED2E7A8D
:109F6000F4EEC77AF1EE10FA47D59FED296ADFEDDE
:109F70002B6A01E0F0EE477AF4EEE67AF1EE10FAA1
:109F800037EE867AF6D4DFED267AB4EEE77AF1EE94
:109F900010FA27DCDFED237AB4EEE77AF1EE10FA5F
:109FA00044BFDFED1D7A37EEC77A27EE076ADFED93
:109FB0001E4ADFED1E6ADFED1E7AE6EE246A67EECA
:109FC000064AE6EE267AB7EE006AA4EEA77AF6EE27
:109FD000006A36EE476AF8EE007A27EE277A66EED8
:109FE000266A84E7DFED097A37EEC77ADDE7B0EE5F
:109FF000677A3DE7F0EE407A24E7B0EE677AC2E791
:10A00000F0EE477AAAE700BF27D4D236DB0F4940EB
:10A01000DB0FC940E4CB1641DB0F49C0E4CB16C1CE
:10A02000DB0FC93FDB0FC9BF92E741B99730083C4E
:10A0300015A82ABEF304353F0000008070B40668FE
:10A040008E4217D90139751E002311F8014F0822DD
:10A05000634013F0800F4FEA430318BF83F0D5032A
:10A06000013ADBB2F5D18D42EFD1721C0260337040
:10A0700070BC70470023F8E710B44C09012250F877
:10A08000243001F01F0102FA01F10B4340F82430A3
:10A090005DF8044B704700BF4B0901F01F0150F8F9
:10A0A0002320012303FA01F1114214BF18460020B6
:10A0B000704700BFF0B55FEA930E33D000F1100691
:10A0C00001F1100502F11004774616ED046A55ED12
:10A0D000044A56ED026A15ED025A16ED037A55ED63
:10A0E000035A56ED017A26EE246A66EE856A04ED7F
:10A0F000046A15ED016A44ED026A27EE257A67EEDF
:10A10000867A013F04ED037A44ED017A06F11006E8
:10A1100005F1100504F11004D7D14FEA0E142044C4
:10A120002144224413F003030BD000EB8303F0EC33
:10A13000017AB1EC017A67EE877A8342E2EC017A28
:10A14000F5D1F0BD144B984224D003F580639842BA
:10A1500020D0028822F040021204120C02800288F1
:10A1600022F038031B041B0C59B141F48071002903
:10A1700091FAA1F2B2FA82F108BF4FF0FF31013932
:10A18000C9000B439BB2038003889BB243F040039A
:10A19000038070474908DCE7003800400C4B9842C8
:10A1A00013D0A3F5806398420FD003F58043984203
:10A1B0000BD003F58063984207D003F58063984283
:10A1C00003D0044B186840087047024B186870476A
:10A1D00000040140707F0020F0B5774B774A87B0CC
:10A1E0001968914200AF00F0DB800023744A3B60A5
:10A1F0007B60136843F48033136003E03B68B3F57E
:10A20000A04F09D0136803F400337B603B6801332F
:10A210003B607B68002BF1D0694B1B6813F4003363
:10A2200018BF01237B607B68012B7BD0654D644B9D
:10A23000654AEA606549586F654A0860AA605E6BC6
:10A24000644C654A654826F080065E635E6F46F0A2
:10A2500080765E67196B0C431C63596B5963996B6D
:10A260009963196C41F05B5141F47B1141F41F611A
:10A2700041F00F011964596C07F118040A4348F2C0
:10A28000FF715A6444F8101D002621460123FB7318
:10A290003E737E73BE731FF0DBFA21464FF6FF73E9
:10A2A0004F48BB601FF0D4FA4FF6FF7321464D486C
:10A2B000BB601FF0CDFA21464B481FF0C9FA21467A
:10A2C0004A481FF0C5FA214649481FF0C1FA214605
:10A2D00048481FF0BDFA214647481FF0B9FA214609
:10A2E00046481FF0B5FA20461FF070F8444B454C25
:10A2F0001B68BA6844484549A4FB03439B09A0FB7B
:10A300000202013B920CB3F1807F0A6007D2404AFF
:10A31000F0200721536085F82300966011601C37F8
:10A32000BD46F0BD264B3B4D1A6C3B4842F0805277
:10A330001A642C684268816844F440442C609C682C
:10A340009C609C6844F400449C609C6844F4A05465
:10A350009C600068120642EA801242F480024908BA
:10A3600042F00802013942EA01425A601A6842F09A
:10A3700080721A601A689201FCD52849104A40F28E
:10A3800005700860996821F003019960996841F0AF
:10A3900002019960936803F00C03082BFAD145E79A
:10A3A00000221A6062B61E4B1B6883F308881D4B9F
:10A3B0001B689847FEE700BFFCFF0120EFBEADDE43
:10A3C0000038024000ED00E00005FA05108800208A
:10A3D00000000008FF916700335F070000000240A3
:10A3E0000004024000080240000C0240001002403D
:10A3F0000014024000180240001C024000200240ED
:10A40000707F0020D34D621083DE1B43B0B4002068
:10A4100010E000E00070004000000020003C02401E
:10A420000000FF1F0400FF1F08B5054B1B6803B1A8
:10A430009847044B044A1A6072B6FEF7CFF800BF83
:10A4400020460020FCFF0120EFBEADDE08B5034B27
:10A450001B6803B1984772B6FEF7C0F8204600208B
:10A46000084B10B507281B68C8BF143818440C46A1
:10A47000007E02F0F3FE20B12146BDE8104003F05B
:10A48000E1BF10BD1861002038B50C4B07281B68D0
:10A49000CCBFA0F11404044623440546187E02F004
:10A4A000DDFE50B128220134C471827133F022F9EB
:10A4B00028460021BDE83840D2E738BD18610020A9
:10A4C000064A00235168814202F11C0204D0013384
:10A4D000102BF7D100207047D8B27047141A002013
:10A4E0002DE9F04F684C54F8204083B0002C00F068
:10A4F000C780256E002D00F0C580D5F810B0D5F8C6
:10A5000004A0C4F858A09846174604F166035F4AB1
:10A510002260636104F266224FF400730646A16074
:10A52000A261E3602361A146BBF1000F19D0584638
:10A53000FFF7C6FF564B5749C0EBC00003EB800046
:10A540000A6B03694FF00C0E1A43731C0A634376BF
:10A5500080F818E0AA68E2630AF104036365C4F8AE
:10A5600034B0E86870B3FFF7ABFF494A494BDFF8F6
:10A5700028E1196BC0EBC00002EB800002691143B7
:10A5800019630B210176711C4176196B0A43E97F2F
:10A590001A638B090022417B8DF805304461012349
:10A5A000C0F808E001A88DF804108DF806208DF899
:10A5B00007301EF0C3FEA36DA968EA68A2630433E6
:10A5C0002164236594F8650002F048FE824694F801
:10A5D000640002F043FE8346287F00284DD118F026
:10A5E000080F36D1BA070DD5BAF1000F0AD00B22E9
:10A5F000731C8AF806208AF8073050466A7F2221A9
:10A6000002F094FCFB0715D4E36B7BB9AA7F8DF8AD
:10A61000042095F820208DF8063001A89309012226
:10A620008DF805308DF807201EF088FE484603B0EF
:10A63000BDE8F08FBBF1000FE6D001360C238BF89C
:10A6400007608BF8063058466A7F222102F06EFCC4
:10A65000DAE70136F6B2BAF1000F04D00B238AF81C
:10A6600007608AF8063018F0100F504614BF022118
:10A6700012216A7F02F05AFCC6E733F01DF8AEE7FC
:10A68000A146D3E7A946D1E7F8600020EC0A040808
:10A69000141A002000380240F58B00080348D0F857
:10A6A000AC3113B100F5D27018477047141A00206E
:10A6B0000348D0F8903113B100F5C47018477047C3
:10A6C000141A00200348D0F8743113B100F5B670A5
:10A6D00018477047141A00200348D0F8583113B1B6
:10A6E00000F5A87018477047141A00200348D0F8E6
:10A6F0003C3113B100F59A7018477047141A0020C6
:10A700000348D0F8203113B100F58C70184770471A
:10A71000141A00200348D0F804310BB1FC3018475C
:10A72000704700BF141A00200348D0F8E8300BB17E
:10A73000E0301847704700BF141A00200348D0F8D3
:10A74000CC300BB1C4301847704700BF141A00203A
:10A750000348D0F8B0300BB1A8301847704700BF9D
:10A76000141A00200348D0F894300BB18C301847ED
:10A77000704700BF141A00200248836F0BB170307D
:10A7800018477047141A00200248C36D0BB15430AB
:10A7900018477047141A00200248036C0BB1383078
:10A7A00018477047141A00200248436A0BB11C3046
:10A7B00018477047141A00200248836803B11847ED
:10A7C000704700BF141A0020F8B50501684C694BAA
:10A7D000625961199A4204EB050704BF01230B7308
:10A7E0000646387A32F068FF3B7A03F01F015B09B6
:10A7F0000122032B02FA01F26DD0042B66D0022B4A
:10A800005CD063190136187902F028FDF6B20746CC
:10A8100010B11223C67183716319587902F01EFDBD
:10A8200010B11323C67183716319987902F016FD74
:10A8300010B11423C671837166190A21F279384662
:10A8400002F074FB707902F009FDF2790A2102F03E
:10A850006DFBB07902F002FDF2790A2102F066FB8D
:10A860006359454A934247D0424A934250D0434AA3
:10A87000934259D0424A934262D0424A93426BD0AB
:10A88000414A93422CD02C44227BE2B9012002227F
:10A89000198801F4415141F445710A4302431A8079
:10A8A0009A8B22F400621204120C07219A831982F7
:10A8B0001A8892B242F040021A80F8BD334B596AAE
:10A8C0000A435A629DE700200246E1E72F4B1969CF
:10A8D0000A431A6195E72D4B196A0A431A6290E7F9
:10A8E00002F564424FF40010536A43F400135362BC
:10A8F0001EF05CFD6359C6E702F584324FF48050C8
:10A90000536A43F4805353621EF050FD6359BAE713
:10A9100002F500324FF48040136A43F4804313621F
:10A920001EF04CFD6359AEE702F5FE324FF40040D5
:10A93000136A43F4004313621EF040FD6359A2E71B
:10A9400002F582324FF40050536A43F400535362CD
:10A950001EF02CFD635996E702F568424FF4801013
:10A96000536A43F4801353621EF020FD63598AE753
:10A97000ACB100200038004000300140003C0040F5
:10A9800000340140005001400054014000380240B2
:10A99000431C00F014812DE9F04F4FEAC00808EB8A
:10A9A00000039B00DFF8F4A25AF803B087B00AEB6B
:10A9B0000304BBF1000F00F0FF8014330AEB030126
:10A9C0000022DBF804704AF803204A608A60CA60FB
:10A9D0000346A56801900133D4F80C90DBB2002D3A
:10A9E00000F0EE801522EB71AA71B9F1000F00F0B2
:10A9F0000081162289F8062089F807309BF80E009E
:10AA000032F05AFEBB8823F440731B041B0CBB803E
:10AA1000284603F011FD484603F00EFD112128469B
:10AA200003F0F6FA1121484603F0F2FA08266424EE
:10AA300004E00A203CB102F0B1FF013C284603F0DB
:10AA40004DFD0028F5D0284603F0F0FC0A2002F066
:10AA5000A5FF284603F0F0FC0A2002F09FFF013E0C
:10AA6000ECD1484603F0E2FC0A2002F097FF2846AA
:10AA700003F0DCFC0A2002F091FF284603F0DCFC26
:10AA80000A2002F08BFF484603F0D6FC019B08EB3E
:10AA900003040AEB84042846637C002B0CBF1221BC
:10AAA0003221042202F042FA637C002B0CBF1221F7
:10AAB00032214846042202F039FA704B9F4200F0DE
:10AAC000B7806F4B9F4200F0BD806E4B9F4200F0FD
:10AAD000A580BB8801996C4A6C4C23F440731B041D
:10AAE0001B0CBB803B8888440AEB880A9BB243F06E
:10AAF00001039AF810103B80BD8802A8002918BFF6
:10AB000014461EF063FC049A6148B2FBF4F325F08E
:10AB10003F05A0FB02122D04900C2D0C0543BD80B7
:10AB20005C4C39884FF4967202FB00F284FB0240C1
:10AB30009BB2D217002BC2EBA01221F0010108BF7B
:10AB400001230904013243F40043090C92B2398015
:10AB50003A84BB833B889BB243F001033B803B8834
:10AB600023F4816323F002031B041B0C43F4806372
:10AB70004FF480423B803A813B8823F080031B04E2
:10AB80001B0C3B809BF810308DF80830002401230B
:10AB900002A88DF80B308DF809408DF80A401EF0A0
:10ABA000CDFB9BF80F308DF8083002A88DF80940D6
:10ABB0008DF80A401EF0E8FB07B0BDE8F08F704743
:10ABC000B9F1000F48D0162289F8073089F806201D
:10ABD0009BF80E0032F070FDBB8823F440731B0419
:10ABE0001B0C2846BB8003F027FC484603F024FCDE
:10ABF00018E79BF80E0032F05FFDBB8823F440732A
:10AC00001B041B0CBB80284603F016FC484603F0CF
:10AC100013FC1121284603F0FBF907E71E4A136ACB
:10AC200043F4000313624FF400001EF0C7FB50E72B
:10AC3000194A136A43F4001313624FF400101EF014
:10AC4000BDFB46E7144A136A43F4800313624FF4D2
:10AC500080001EF0B3FB3CE79BF80E0032F02CFDA9
:10AC6000BB8823F440731B041B0C4846BB8003F0D5
:10AC7000E3FB484603F0E0FBD8E600BF0054004089
:10AC800000580040005C0040009F2400804F1200EC
:10AC900083DE1B43D34D6210003802402861002040
:10ACA0002DE9F0410678012E82B005464CD0022EE7
:10ACB00052D1806841F0800110B1046880886083BF
:10ACC000686840F2E93402E0002C00F099800689BF
:10ACD000013C16F0020FA4B2F6D089B2818140F295
:10ACE000E93102E0002900F08B800489013914F079
:10ACF000010F89B2F6D0818981894FF0000C4FF4A1
:10AD00007A714FF6FF764FF0FF0E634502D129E0CE
:10AD1000B14225D004890139A70789B2F8D5A0F836
:10AD20000CE04FF47A7102E0B9B2B14218D0048954
:10AD3000E40701F1FF37F7D58489A4B20AB1147092
:10AD400001320CF1010CE0E790F904E0BEF1FF3FA5
:10AD500002D0BEF1030F0FDD002002B0BDE8F0818C
:10AD6000FDF7AAFFAB68002B5CD01A689B881383A1
:10AD7000012002B0BDE8F0814FEACE08DFF8ACC098
:10AD800008EB0E070CEB870778680028E5D06C7994
:10AD90003A6264000025E4B2BC75F9757D76BE7632
:10ADA0003B767E753D758388FA61990514D40388D6
:10ADB000DA050CD44FF4805401E0013C28D003881C
:10ADC0009B05FAD403889BB243F480730380838885
:10ADD0009BB243F440738380F0440CEB88024FF441
:10ADE000805401E0013C13D0537D002BFAD10CEBD1
:10ADF000880898F8144084F0010002B0BDE8F081A2
:10AE00008DE80C00FDF758FF68689DE80C0073E7BB
:10AE1000054A1388013370469BB21380FFF7B8FDD3
:10AE200020469AE7012098E7A22D00202861002003
:10AE300037B506236A4604460D460C300321FFF75A
:10AE40002FFF024690B1B4F91A106846FDF7DDFAFB
:10AE50002880B4F91E100DF10200FDF7D6FAA88083
:10AE6000B4F91C1001A8FDF7D0FA6880104603B0B1
:10AE700030BD07B5032301AA0021FFF711FF9DF89C
:10AE800005309DF804001B0243EA00439DF80600CC
:10AE9000184303B05DF804FB08B5FFF7EAFF014B68
:10AEA000586008BD681E002008B5FFF7E2FF014B9F
:10AEB000186008BD681E00202DE9F04F90F855304D
:10AEC00085B00646002B40F0AB8002AB0093514B9F
:10AED0009B7B002B00F0568170694F4B984200F02D
:10AEE000D2844E4A90420CBF30223822038823F08D
:10AEF00040031B041B0C038003889BB223F0380320
:10AF00001A43028003889BB243F040030380B36975
:10AF100096F84E1013B11A689B88538340F2E933B8
:10AF200004E0013B9BB2002B00F058850289970793
:10AF3000F7D51A23838140F2E93304E0013B9BB249
:10AF4000002B00F04B850289D507F7D5838940F2A5
:10AF5000E93304E0013B9BB2002B00F03B85028902
:10AF60009407F7D589B2818140F2E93304E0013BCF
:10AF70009BB2002B00F02E850289D207F7D583897A
:10AF8000B36913B11A689B881383012002F006FD90
:10AF90007369214A934200F0498520498B4214BFCE
:10AFA000082100211A8822F040021204120C1A8093
:10AFB0001A8892B222F03802114319801988009A37
:10AFC00089B241F04001198006F1100006234321A7
:10AFD000FFF766FE002800F083849DF80A509DF874
:10AFE0000B309DF808409DF809109DF80C009DF865
:10AFF0000D2043EA05231BB241EA042142EA002264
:10B0000073873187B2875BB2013300F03F8405B0AC
:10B01000BDE8F08F681E002000380040003C004072
:10B020001C09013C042C03F00F0300F20685B94A09
:10B0300032F8140040FA03F2D20740F1FE844FF0D8
:10B04000010808FA03F3013B184034F025F9B24B2C
:10B05000B24F1D5D054417EBC50400F0EE842022BD
:10B060000023A271E37157F83500AD4A00F13F4368
:10B0700003F57E039B0AD25C02F01F035209032AE8
:10B0800008FA03F300F02A85042A00F02185022A39
:10B0900000F01885A388029302A94FF000080091E0
:10B0A000CDF80C801EF0D4FBA2889E4BF360B2FA60
:10B0B00082F2C2F11F02531C00F0BB84D3B203F032
:10B0C000FC0E0EF1804E0EF59C3E03F00300DEF800
:10B0D000081057F83530944FDFF870C285000F2004
:10B0E000A84021EA000103F13F4306F10C0047F8B4
:10B0F000220003F57E03CEF80810C3F38720DEF8A4
:10B1000008308A498A4FA8400125184305FA02F3FE
:10B11000CEF808004B61D1F800E0D8430EEA000EEB
:10B12000C1F800E0D1F804E000EA0E0EC1F804E036
:10B13000D1F800E043EA0E0EC1F800E0D1F808E0D3
:10B1400000EA0E0EC1F808E0D1F80CE000EA0E00AB
:10B15000DFF8FCE1C86039687244194392F8C420F2
:10B1600039601CF80210F02900F39084002B3FF4A2
:10B17000AEAE6E490A6813430B606E4B9B7B002B8F
:10B180007FF4AAAE70696C4B984200F0AF846B4AB2
:10B1900090420CBF30223822038823F040031B0466
:10B1A0001B0C038003889BB223F038031A430280F0
:10B1B00003889BB243F040030380B36913B11A685C
:10B1C0009B88538340F2E93304E0013B9BB2002BA0
:10B1D00000F0378402899407F7D56B23838140F20E
:10B1E000E93304E0013B9BB2002B00F02A84028982
:10B1F000D107F7D5838940F2E93304E0013B9BB2E4
:10B20000002B00F0238402899207F7D580238381E5
:10B2100040F2E93304E0013B9BB2002B00F01684BE
:10B220000289D707F7D58389B36913B11A689B8858
:10B2300013839623424C434DDFF818A14248DFF8B0
:10B2400018C101964FF010084FF47A779946DAF852
:10B250000430C3F30803002B40F08283EFF3118323
:10B26000002B40F07D832368816800BF22689342F1
:10B27000F9D12A6807FB02FEAEEB010EBEFBF2FE1F
:10B2800007FB03EE0126DAF80430C3F30803002BB2
:10B2900040F02A83EFF31183002B40F025832368CD
:10B2A000816800BF22689342F9D1D5F800B007FB4E
:10B2B0000BF2521AB2FBFBF207FB0323A3EB0E03C4
:10B2C000B3F57A7FDFD3B9F10109C0D1019EB3692B
:10B2D00013B11A689B885383706940F2E93304E024
:10B2E000013B9BB2002B00F0CA8302899707F7D578
:10B2F0006823838140F2E93304E0013B9BB2002BD9
:10B3000000F0BD830289D107F7D5838940F2E93384
:10B3100029E000BFA43C04089C3C0408F4B10020D0
:10B32000943C0408D5850008841E0020003C0140A0
:10B33000083C0140681E002000380040003C0040EE
:10B34000ACB40020B0B4002010E000E0C41E002027
:10B35000500A040800ED00E0A8B40020013B9BB2B5
:10B36000002B00F0908302899207F7D50323838195
:10B3700040F2E93304E0013B9BB2002B00F08383F1
:10B380000289D707F7D58389B36913B11A689B88F7
:10B3900013839623DFF878A29C48DFF878C20196E1
:10B3A0004FF010084FF47A779946DAF80430C3F377
:10B3B0000803002B40F0F182EFF31183002B40F0E3
:10B3C000EC822368816800BF22689342F9D12A6821
:10B3D00007FB02FEAEEB010EBEFBF2FE07FB03EE27
:10B3E0000126DAF80430C3F30803002B40F09A82F8
:10B3F000EFF31183002B40F095822368816800BF32
:10B4000022689342F9D1D5F800B007FB0BF2521A2B
:10B41000B2FBFBF207FB0323A3EB0E03B3F57A7F2A
:10B42000DFD3B9F10109C0D1019EB36913B11A6824
:10B430009B885383706940F2E93304E0013B9BB27F
:10B44000002B00F0EC8202899107F7D56B238381F2
:10B4500040F2E93304E0013B9BB2002B00F0DF82B5
:10B460000289D207F7D5838940F2E93304E0013B32
:10B470009BB2002B00F0D78202899707F7D50323F0
:10B48000838140F2E93304E0013B9BB2002B00F0E2
:10B49000CA820289D507F7D58389B36913B11A68BF
:10B4A0009B8813830F2002F079FAB36913B11A68ED
:10B4B0009B885383706940F2E93304E0013B9BB2FF
:10B4C000002B00F0908202899407F7D56A238381CC
:10B4D00040F2E93304E0013B9BB2002B00F0838291
:10B4E0000289D107F7D5838940F2E93304E0013BB3
:10B4F0009BB2002B00F07B8202899207F7D51023C4
:10B50000838140F2E93304E0013B9BB2002B00F061
:10B510006E820289D707F7D58389B36913B11A6898
:10B520009B8813830F2002F039FAB36913B11A68AC
:10B530009B885383706940F2E93304E0013B9BB27E
:10B54000002B00F0578202899507F7D56C23838181
:10B5500040F2E93304E0013B9BB2002B00F04A8249
:10B560000289D407F7D5838940F2E93304E0013B2F
:10B570009BB2002B00F0428202899107F7D500238D
:10B58000838140F2E93304E0013B9BB2002B00F0E1
:10B5900035820289D207F7D58389B36913B11A6856
:10B5A0009B8813830F2002F0F9F9B36996F85010C5
:10B5B00013B11A689B885383706940F2E93304E041
:10B5C000013B9BB2002B00F01C8202899707F7D544
:10B5D0001923838140F2E93304E0013B9BB2002B45
:10B5E00000F00F820289D507F7D5838940F2E9334D
:10B5F00004E0013B9BB2002B00F007820289940714
:10B60000F7D589B2818140F2E9330AE010E000E029
:10B6100000ED00E0A8B40020013B9BB2002B00F03D
:10B62000F4810289D107F7D58389B36913B11A6808
:10B630009B8813830F2002F0B1F9B36913B11A6824
:10B640009B885383706940F2E93304E0013B9BB26D
:10B65000002B00F0DD8102899207F7D51B2383813F
:10B6600040F2E93304E0013B9BB2002B00F0D081B3
:10B670000289D707F7D5838940F2E93304E0013B1B
:10B680009BB2002B00F0C88102899507F7D51823DB
:10B69000838140F2E93304E0013B9BB2002B00F0D0
:10B6A000BB810289D407F7D58389B36913B11A68BE
:10B6B0009B8813830F2002F071F9B36913B11A68E4
:10B6C0009B885383706940F2E93304E0013B9BB2ED
:10B6D000002B00F0BF8102899107F7D51C238381DD
:10B6E00040F2E93304E0013B9BB2002B00F0B28151
:10B6F0000289D207F7D5838940F2E93304E0013BA0
:10B700009BB2002B00F0AA8102899707F7D510237E
:10B71000838140F2E93304E0013B9BB2002B00F04F
:10B720009D810289D507F7D58389B36913B11A685A
:10B730009B8813830F2002F031F9B36913B11A68A3
:10B740009B885383706940F2E93304E0013B9BB26C
:10B75000002B00F0868102899407F7D53723838177
:10B7600040F2E93304E0013B9BB2002B00F0798109
:10B770000289D107F7D5838940F2E93304E0013B20
:10B780009BB2002B00F0718102899207F7D510233C
:10B79000838140F2E93304E0013B9BB2002B00F0CF
:10B7A00064810289D707F7D58389B36913B11A6811
:10B7B0009B8813830F2002F0F1F8B36913B11A6864
:10B7C0009B885383706940F2E93304E0013B9BB2EC
:10B7D000002B00F04D8102899507F7D5382383812E
:10B7E00040F2E93304E0013B9BB2002B00F04081C2
:10B7F0000289D407F7D5838940F2E93304E0013B9D
:10B800009BB2002B00F0388102899107F7D5012304
:10B81000838140F2E93304E0013B9BB2002B00F04E
:10B820002B810289D207F7D58389B36913B11A68CE
:10B830009B8813830F2002F0B1F87369AD4A9342DD
:10B8400000F05281AC498B4214BF082100211A88B4
:10B8500022F040021204120C1A801A8892B222F0CE
:10B860003802114319801A8892B242F040021A80BD
:10B87000012002F093F8A14A7069012393739D4B54
:10B8800098427FF42EAB3022FFF730BB96F9383068
:10B8900001337FF4BCAB0A26322032F02DF94FF48D
:10B8A000FA7502F02FF8044602F02CF8001BB0F5F0
:10B8B0007A7FF9D3013DF4D1072031F07FFF4FF4B7
:10B8C0007A7502F01FF8044602F01CF8001BB0F570
:10B8D0007A7FF9D3013DF4D1013EDDD1FEF7A4FD1D
:10B8E000B6F93A30FFF78FBBEFF3118188F3128876
:10B8F000D0F808B00368DB0344BFCCF80060D0F890
:10B9000008B02368DCF80020C9B281F311882968E7
:10B910001A4407FB01F3A3EB0B03B3FBF1F307FBA3
:10B920000233CBE4EFF3118188F31288D0F808B02A
:10B930000368DB0344BFCCF80060D0F808B023688C
:10B94000DCF80020C9B281F3118829681A4407FB8A
:10B9500001F3A3EB0B03B3FBF1F307FB02335BE54E
:10B96000EFF3118288F3128881680368DE0303D540
:10B970000123CCF8003081682368DCF80060D2B283
:10B9800082F311882A6806EB030E07FB02F35B1AA9
:10B99000B3FBF2F307FB0E3E74E4EFF3118288F37E
:10B9A000128881680368DE0303D50123CCF80030D8
:10B9B00081682368DCF80060D2B282F311882A68BB
:10B9C00006EB030E07FB02F35B1AB3FBF2F307FB74
:10B9D0000E3E05E5FDF770F9FFF7D2BAFDF76CF9F9
:10B9E0007069FFF7B4BAFDF767F970697CE5FDF798
:10B9F00063F992E5FDF760F97069B5E5FDF75CF96B
:10BA0000CBE5FDF759F97069F0E5FDF755F90CE65E
:10BA1000FDF752F970692FE6FDF74EF945E6FDF79F
:10BA20004BF9706920E5FDF747F936E50021FFF78E
:10BA3000B9BA01239340FFF799BB314BF360FFF78D
:10BA400044BAFDF739F97069FFF7D5BBFDF734F952
:10BA5000FFF7EABBFDF730F970694DE6FDF72CF909
:10BA600063E6FDF729F9706986E6FDF725F99CE69E
:10BA7000FDF722F97069BFE6FDF71EF9D5E6FDF77F
:10BA80001BF9706942E4FDF717F97DE40EEB020340
:10BA9000F02193F8D4308DF8083000988DF80A80A2
:10BAA00003238DF809308DF80B500CF802101DF0AF
:10BAB00045FCA388B3FA83F3C3F11F0305FA03F32C
:10BAC000FFF754BB0F4A516C0B435364FFF7E2BAC4
:10BAD0000C4A116B0B431363FFF7DCBA094A116C74
:10BAE0000B431364FFF7D6BA0021B0E63022FFF70C
:10BAF00053BB00BF00380040003C0040681E0020DF
:10BB0000D585000800380240F0B5C60033189B0008
:10BB1000254DEA585468A28A83B092B20192019AE4
:10BB20002B4412F4706F1CBF01221A75019B13F491
:10BB3000E06F07460CD1A38A3E4423F4706305EB03
:10BB400086051B041B0C0022A3826A7503B0F0BD9E
:10BB5000238BA38823F480631B041B0CA380019B0D
:10BB60009B05E8D423889805E5D42388D9050ED50C
:10BB70002388DA05FCD423889BB243F40073238026
:10BB800023889B05FCD43846FEF702FFD3E72388C1
:10BB90009BB243F400732380A38823F440731B04F7
:10BBA0001B0CA380C7E700BF28610020F0B5037A13
:10BBB000012B83B0014664D0022B68D1036913B115
:10BBC0001A689B885383C86840F2E93302E0002B6F
:10BBD00000F0AA800289013B12F0020F9BB2F6D05E
:10BBE000BB23838140F2E93302E0002B00F09C800C
:10BBF0000289013B12F0010F9BB2F6D08389838941
:10BC00004FF0060E4FF47A736E464FF6FF74FF271F
:10BC100003E0013B9BB2A3423CD002899507F8D5D3
:10BC200087814FF47A7302E0ABB2A34232D002892B
:10BC3000D20703F1FF35F7D5828992B20EB1327087
:10BC40000136BEF1010EE8D10B6913B11A689B8869
:10BC500013839DF800609DF801009DF802509DF847
:10BC600003209DF804409DF8053040EA062042EA92
:10BC7000052243EA0423C88201200A834B8303B0D0
:10BC8000F0BD90F90C00451C01D0032805DD002013
:10BC900003B0F0BDFDF710F8D6E7C700294E3A18FB
:10BCA00006EB82025568002DF1D04C7B6400E4B2B3
:10BCB00094754FF0000E06244FF03B0C82F817C02D
:10BCC00082F819E093761476537582F814E0AB8805
:10BCD000C2F820D09C05C2F81CD014D42B88DA05F9
:10BCE0000CD44FF4805401E0013C21D02B889B05FB
:10BCF000FAD42B889BB243F480732B80AB889BB221
:10BD000043F44073AB80074406EB87024FF4805442
:10BD100001E0013C0CD0537D002BFAD106EB8707E4
:10BD20003B7D002B95D0B2E7FCF7C6FFC86866E7FD
:10BD3000054A138801339BB21380FEF729FE204683
:10BD4000A6E700BF28610020A22D0020F0B583B037
:10BD5000441C8DF8073001D0032802DD002003B019
:10BD6000F0BDC700244E3B1806EB83035D68002D31
:10BD7000F4D04900C9B2997501240021DA755C76C6
:10BD800099761C765C751975A9880DF107028905ED
:10BD9000DA611A6214D42B88DA050CD44FF480547B
:10BDA00001E0013C1ED02B889B05FAD42B889BB266
:10BDB00043F480732B80AB889BB243F44073AB8019
:10BDC000074406EB87024FF4805401E0013C09D0A0
:10BDD000537D002BFAD106EB87073C7D84F00100F0
:10BDE00003B0F0BD054A138801339BB21380FEF700
:10BDF000CFFD2046B3E700BF28610020A22D002020
:10BE00000378012B46D0022B42D12DE9F041836803
:10BE100001F07F0113B11C689B88638305461746B8
:10BE2000406840F2E93401E0002C39D00689013C39
:10BE300016F0020FA4B2F7D089B2818140F2E93145
:10BE400000E069B30389013913F0010F89B2F8D01A
:10BE5000838940F2E93100E031B30489013914F0FB
:10BE6000020F89B2F8D0BFB2878140F2E93300E017
:10BE7000D3B10289013B12F0010F9BB2F8D0838944
:10BE8000AB68A3B11A689B8813830120BDE8F081D9
:10BE90000020704713460A46417990F9040055E79F
:10BEA000FCF70AFF6868D4E7FCF706FFE8E7012023
:10BEB000BDE8F0812DE9F04F4FF4807385B04383E6
:10BEC0008383C38300F10C050446322001F0C0FDDA
:10BED000112200212846FFF793FF60220121284606
:10BEE000FFF78EFF642001F0B3FD02A92046002772
:10BEF000FEF79EFF0123B946B8463E460193012E48
:10BF000014BF1122122200212846FFF779FF002ECC
:10BF10000CBF4FF0010B4FF0FF3B4FF00A0A01221C
:10BF200002212846FFF76CFF142001F091FD02A9C1
:10BF30002046FEF77DFFBDF90A20BDF90C00BDF9D2
:10BF40000810234B82420BFB0299A8BF02468A428B
:10BF5000A8BF0A469A4201FB0B880BFB007733DB34
:10BF6000012002F045F8BAF1010AD8D10136022EBB
:10BF7000C5D1184B93FBF8F893FBF9F97022A3F5A0
:10BF80008423002193FBF7F7A4F81A80A4F81C90EF
:10BF9000E7832846FFF734FF202201212846FFF7D8
:10BFA0002FFF002231462846FFF72AFF642001F0C8
:10BFB0004FFD019B23B94FF480736383A383E38315
:10BFC000012005B0BDE8F08F00230193CEE700BF4C
:10BFD00001F0FFFF00D03B000122482110E70122C1
:10BFE00058210DE70220FCF7A7BB00BF02208BE51C
:10BFF0000120FCF7A1BB00BF012085E50020FCF774
:10C000009BBB00BF00207FE51549164B16480A6808
:10C0100010B48C681549B2FBF4F203FB02F3036021
:10C02000D1F88820124B134C42F47002C1F88820DA
:10C030001A68002042F001021A6098601A6822F023
:10C04000847222F480321A605C601A684FF00064D7
:10C0500022F480221A60D8608C605DF8044B70472F
:10C060000000002040420F00707F002000ED00E043
:10C070000038024010300024044B4FF4F0700A21C5
:10C08000022283E80700FFF7BFBF00BF00000020C7
:10C090000B4B002210B4027203F5C074022102E0BF
:10C0A000072A09DC9979890702D519798154013267
:10C0B0009C4203F11803F3D15DF8044B704700BFB5
:10C0C000002F040810B40D4C02232146002200E08A
:10C0D0008B7913F0010301F1180106D10132112A05
:10C0E000F6D103705DF8044B704702EB420204EB9B
:10C0F000C2025DF8044B137903707047002F0408E7
:10C10000012310B432213324312244704171C270B2
:10C1100003720370037183705DF8044B704700BFB6
:10C12000436A8269D154436A0169826B01338B424D
:10C1300028BF00234362002A2FD0EFF3118250233F
:10C1400083F31288836B1968C9072CD470B45E68B6
:10C150006EB9456A816A8D4217D084690C44DC60EF
:10C160000ED9691A59608562002180F85C1019683F
:10C1700041F00101D2B2196082F3118870BC70479E
:10C180000469611A59608662EEE7012380F85C3029
:10C19000D2B282F3118870BC7047826DD36843F0CD
:10C1A0008003D3607047D2B282F31188704700BF1A
:10C1B000426B10B462B1C36CC2684469D11A013BCE
:10C1C000615C5DF8044B08BF1346C364C8B2704796
:10C1D000016A4369C4685B5C0131A14228BF114612
:10C1E00001625DF8044BD8B2704700BF836B13B196
:10C1F00090F85C007047836A406A181AB0FA80F0C1
:10C2000040097047416A836A99420AD3CB1A816B0D
:10C21000026961B14968501E0B4483420AD2C01AB8
:10C22000704702691144CB1A816B0029F2D1501E6C
:10C23000C01A704700207047436B43B1C26C5B6803
:10C2400093422FBF981AC0689B1AC0187047C269E2
:10C25000036A9A422FBFD01AC0688018C01A70476C
:10C260000A4B30B503F11C0493F900205D78072ACE
:10C27000C8BF143A811804330D7313F8025C855457
:10C2800013F8012C0A76A342EED130BD2C0B040822
:10C2900003682DE9F041DF691FB13B46BDE8F0417D
:10C2A0001847002A164611DD04460D460E4400E0EC
:10C2B00023689B68204698470028F9D0236815F822
:10C2C000011B1B6820469847AE42F1D1BDE8F081C2
:10C2D00010B4522153245122002304704170827003
:10C2E000C3705DF8044B704710B5084B03F10C01A7
:10C2F00093F900205C78845402449C78D470DC78F4
:10C30000947104338B42F3D110BD00BF480B040875
:10C31000038A2DE9F0478589ADB21D4029D00F462B
:10C3200006464FF000484FF00009B5FA85F328FAA9
:10C3300003F2D24391B21B3B15403182042B16D835
:10C34000DFE803F03129211903007B6A002B32D08A
:10C3500003F1FF3A1FFA8AFAC7F824903C6A34B115
:10C3600023682046514698476468002CF8D1002D78
:10C37000DBD1BDE8F0873868716B036889B29847F4
:10C38000002DD2D1F5E77868B16B036889B2984780
:10C39000002DCAD1EDE7B868F16B036889B2984700
:10C3A000002DC2D1E5E7F868316C036889B298477F
:10C3B000002DBAD1DDE7F36A1FFA83FACEE700BF9A
:10C3C00030B50446806D61718389A26823F40053FF
:10C3D0001B041B0C838185B0A379009213F0040227
:10C3E00030D04FF4805213F00203ADF8042063D133
:10C3F000ADF806304FF480630022ADF8083011F03C
:10C400000103ADF80C2028D1ADF80A3008238D07C0
:10C41000694648BFADF80A301DF020F8A279A36D37
:10C42000D10724D412F0080F9A8A1BD122F00802F7
:10C430001204120C9A829A8992B242F400529A81A2
:10C4400005B030BD13F00203ADF8042031D04FF435
:10C4500000551346ADF80650CEE70423ADF80A3078
:10C460000C23D4E792B242F008029A82E3E714491F
:10C470008B421CD0A1F54C418B4216D001F5806156
:10C480008B4210D001F580618B420AD001F5484102
:10C490008B42C7D105200121FDF7E2FFA279A36DF0
:10C4A000C0E70320F7E70220F5E70120F3E70020CB
:10C4B000F1E7ADF806309FE74FF4005398E700BF6F
:10C4C0000010014010B50446806DA160838923F4FB
:10C4D00000531B041B0C8381A37984B013F0040266
:10C4E000009135D04FF4805213F00203ADF80420D0
:10C4F00063D1ADF806304FF480636279ADF808304F
:10C50000D1074FF00003ADF80A30ADF80C3045BF4D
:10C510000423ADF80A3008230C236946920748BF6C
:10C52000ADF80A301CF09AFFA279A36DD1071FD491
:10C5300012F0080F9A8A16D122F008021204120C87
:10C540009A829A8992B242F400529A8104B010BD44
:10C5500013F00203ADF804202CD04FF40051134621
:10C56000ADF80610C9E792B242F008029A82E8E7F5
:10C5700013498B421CD0A1F54C418B4216D001F5DA
:10C5800080618B4210D001F580618B420AD001F5A9
:10C5900048418B42CCD105200121FDF761FFA279F2
:10C5A000A36DC5E70320F7E70220F5E70120F3E7D5
:10C5B0000020F1E7ADF806309FE74FF4005398E70D
:10C5C000001001402DE98048013085B0C3B20393CB
:10C5D0008B4D8C4F8C4C8D4E0A2302933220DFF80A
:10C5E000309231F089FA4FF4FA7A4FF0100C4FF490
:10C5F0007A70D9F80430C3F30803002B40F0C180EF
:10C60000EFF31183002B40F0BC802968A26800BFC3
:10C610002B689942F9D1D7F800E000FB0EF39B1A82
:10C62000B3FBFEF300FB01314FF0010E0191D9F88D
:10C630000430C3F30803002B40F08780EFF311832D
:10C64000002B40F082802B68A16800BF2A689342CB
:10C65000F9D1D7F800B000FB0BF2521AB2FBFBF293
:10C6600000FB0323019A9B1AB3F57A7FDFD3BAF15B
:10C67000010ABED1039B002B40F0BD804FF47A7AB3
:10C68000DFF88C9150464FF0100CD9F80430C3F30A
:10C690000803002B40F09280EFF31183002B40F051
:10C6A0008D802968A26800BF2B689942F9D1D7F81C
:10C6B00000E000FB0EF39B1AB3FBFEF300FB01311D
:10C6C0004FF0010E0191D9F80430C3F3080303BB06
:10C6D000EFF31183EBB92B68A16800BF2A6893427E
:10C6E000F9D1D7F800B000FB0BF2521AB2FBFBF203
:10C6F00000FB0323019A9B1AB3F57A7FE3D3BAF1C7
:10C70000010AC2D1029B013B02937FF467AFFDF7A0
:10C710008BFEEFF311888CF31288A1682368DB038A
:10C7200044BFC6F800E0A1682B6832685FFA88F859
:10C7300088F31188D7F800801A4400FB08F35B1ACD
:10C74000B3FBF8F300FB0233D4E7EFF311888CF36B
:10C750001288A1682368DB0344BFC6F800E0A16823
:10C760002B6832685FFA88F888F31188D7F8008060
:10C770001A4400FB08F35B1AB3FBF8F300FB023327
:10C7800070E7EFF311828CF31288D4F808E0236885
:10C79000D90303D501233360D4F808E02B6831684E
:10C7A000D2B282F311883A68194400FB02F3A3EB7A
:10C7B0000E03B3FBF2F300FB013135E7EFF3118217
:10C7C0008CF31288D4F808E02368D90303D5012339
:10C7D0003360D4F808E02B683168D2B282F3118854
:10C7E0003A68194400FB02F3A3EB0E03B3FBF2F328
:10C7F00000FB013164E7184630F0E0FF3EE700BF80
:10C80000ACB40020B0B4002010E000E0A8B40020D8
:10C8100000ED00E038B5484B5A899989914224BF10
:10C8200000225A81198ADA89914224BF0022DA81D2
:10C83000DA78CAB1072A41496AD091F85300404DCD
:10C84000012400210A282C709C70D9715DD00C281D
:10C8500007D0002A6CD0DFED3B7A072A0ED00A28D9
:10C8600062D0DFED397A09E0344A92F853000A28A1
:10C8700056D00C285BD1D979DFED347A344C9FED5A
:10C88000350AA278002918BFF0EE407A062A04D8AB
:10C89000314901EB820191ED0A0A217979B1013A1E
:10C8A000032A0BD8F7EE007A87EE800A33F09AF865
:10C8B0002388984228BF1846208038BD38BD9B7811
:10C8C0001F4A07EE103A1178B8EEC77A67EE277A5A
:10C8D00007EE101AB8EEC77A27EE277AB4EEC70A29
:10C8E000F1EE10FAEADD80EE277AFDEEC77A17EE58
:10C8F000903A102BA8BF1023012BB8BF0123DBB245
:10C900008B4238BF0B46137038BDDFED147AA4E7B5
:10C9100091F853000A2803D00C28ACD0D9799AE7B3
:10C92000D979DFED0E7AA9E7DFED0D7AA6E7D9799F
:10C93000DFED047AA2E700BF2472002038720020E5
:10C940007C8700206F1203396F12833A0AD7A3390C
:10C95000247C00206F1203382C0B04085304E938A0
:10C960000F506E3A2DE9F047AE4FAF4E12F02CFF4C
:10C97000BE421ED2DFF83483DFF834934446258864
:10C9800062197DB14A450DD2052D0BD933886188D6
:10C99000C3F30B03994200F0E8801446258862191E
:10C9A000002DEFD1716830461436FCF7F3FABE4221
:10C9B000E4D39E4A1378A3F1170102290FD99C49A9
:10C9C00011F83300002840F0FF80D8000144497876
:10C9D00029B1984911F833300BB918231370964BCD
:10C9E0005A78022A00F2E1809449954802EB42020B
:10C9F00001EB82011A780160022A00F2DF8002EB6B
:10CA00008201904BC2EBC10203EB4203998C5A8C1A
:10CA10008D4C9142236001D300225A848B4B9A782B
:10CA2000042A00F0F28032B91A88B2F5F07F84BF90
:10CA30004FF4F0721A80864DFFF7ECFE2B68854AA2
:10CA40001A40002A00F0EA80D80700F1D980590482
:10CA500000F1D1801A0700F1C0809B0400F1C4806E
:10CA600028F056FB10B97C482CF0ACFC4FF4007059
:10CA7000FCF7D6FA4FF48030FCF7D2FA4FF480205E
:10CA8000FCF7CEFA4FF40010FCF7CAFA4FF0007032
:10CA9000FCF7C6FA4FF08060FCF7C2FA2CF09CFA63
:10CAA000002130226D4833F063FF20682BF006FA36
:10CAB0006B4B256803F1500103E00433994200F009
:10CAC00081801A78002AF8D19C78D8788442F4D2F0
:10CAD0006449654B0A7028461D6017F073FE634A6F
:10CAE00063491079634A644B1160C822642111FBC9
:10CAF0000021002259609A60DA601A615A619A61D5
:10CB0000DA6183F8202083F8212024F087F95B4B39
:10CB10009FED5B5A1B885B4A9FED5B6A55795B4CC6
:10CB20005B495C48086006EE903AF8EEE66A1388C6
:10CB3000C5EE265A07EE103A53881279C4ED005A12
:10CB400007EE903AB8EEC77A534BF8EEE77A1D72CB
:10CB50005A7227EE067A67EE867ABDE8F04783EDD3
:10CB6000017AC3ED007A12F017BE63799B077FF458
:10CB700014AF716894F804A03046FCF70BFA3388C0
:10CB8000BAEB133F04D01436BE42FFF4F7AE10E701
:10CB900073887068AA1FC3F30B039A4204F106015D
:10CBA000A8BF1A4633F0BFFEEDE700225A701A788C
:10CBB000234822490160022A7FF621AF00221A7021
:10CBC000204B23E7012283E7D8000C186468002C6F
:10CBD0007FF4FCAE17241470F8E63048FCF720FA16
:10CBE0002B689B047FF53CAF2D48FCF719FA4020D9
:10CBF000FCF716FA34E72B48FCF712FA2B6829E702
:10CC00002948FCF70DFA2B6821E79A8AB2F57A7F5A
:10CC1000BFF411AF4FF47A729A820CE743F0080325
:10CC20002B6011E7180600089001000888B1002069
:10CC30008C360408F4270408A92F0020B62F002002
:10CC4000503A00203E4100204C3A0020247C002035
:10CC5000AC8700200960000280700020681F00205F
:10CC60002C290020901C00209C1F0020E081002027
:10CC70008E870020A41F00204C320020B824002002
:10CC8000C0C9FB483425002017B7D138BC24002088
:10CC9000A88000203661023D8480002001600002EF
:10CCA000094000020920000208600002024000085A
:10CCB000008000082DE9F84F4FF48C7200218B485A
:10CCC0008B4C8C4D8C4E8D4FDFF84C82DFF84C92A4
:10CCD00033F04EFE8A488B49DFF844E2DFF844C265
:10CCE000002213588B4200F0C280B3F1804F00F055
:10CCF000D180AB4200F0D580B34200F0D580BB427A
:10CD000000F0D580734500F0D580634500F0D580F4
:10CD1000434500F0D5804B4500F0D580DFF808A2F0
:10CD2000534500F0D3800AF5806A534500F0D18066
:10CD3000AAF5983A534500F0CF800AF5806A53452A
:10CD400000F0CD800AF5806A534500F0CB801832A0
:10CD5000B2F5CC7FC5D16A4E6B4F06F5CC784FF05B
:10CD6000030A4FF0020902E0183646457DD0B37938
:10CD7000002BF9D033791C09013C042C03F00F037C
:10CD8000F2D8624A32F8140040FA03F2D207EBD527
:10CD9000012505FA03F3013B184032F07DFA5C4BA4
:10CDA0001B5D184417EBC002DED057F83030594CE9
:10CDB000317A03F13F4000F57E00800A205C00F0EC
:10CDC0001F044009032805FA04F55DD0042855D056
:10CDD000022804D14648406C054345484564B2F8F2
:10CDE00004E0BEFA8EF2C2F11F0292B2D00803EB49
:10CDF000800002F00702046A92000F25954024EAA1
:10CE000005040462046A01FA02F222430025026268
:10CE10004FF0010C2A4603E0102A05F10205A3D0C9
:10CE20000CFA02F030EA0E0102F10102F4D11C68A2
:10CE30000AFA05F1C9430C401C60D3F800B009FAA6
:10CE400005F444EA0B041C609C680C409C609C68E0
:10CE50009C605C6824EA0000586058685860D86894
:10CE60000140D960D968D960D6E7BDE8F88F4FF0A6
:10CE7000010A636C43EA0A03636468E71C48006BB9
:10CE800005431B480563AAE71948006C0543184889
:10CE90000564A4E74FF0010A236C43EA0A03236404
:10CEA00055E74FF0020AF7E74FF0040AF4E74FF0B6
:10CEB000080AF1E74FF0100AEEE74FF0200AEBE71F
:10CEC0004FF0020AD5E74FF4803AD2E74FF4003A28
:10CED000CFE74FF4802ACCE74FF0400ADCE74FF071
:10CEE000800AD9E74FF4807AD6E700BF6425002096
:10CEF000003802400004004000080040000C0040E0
:10CF0000002F040800000140F4B10020A43C0408F4
:10CF10009C3C0408943C040800040140004001408B
:10CF200000100040001400400044014000286AD076
:10CF300003682DE9F04F03F13F4404F57E045F4E92
:10CF4000A40A0125345D04F01F066409032C05FAC8
:10CF500006F559D0042C00F0AC80022C59D08588FD
:10CF6000B5FA85F0C0F11F0080B2C40803EB840459
:10CF700000F00700266A80000F27874026EA070690
:10CF80002662276A01F003068240701E3A43012898
:10CF9000C1F3810CC1F300182262C1F341113DD9E4
:10CFA0000024224601274FF0030E03E0102A04F16B
:10CFB000020426D007FA02F0A84302F10102F5D1DB
:10CFC000D3F800C00EFA04F0C04300EA0C0CC3F81A
:10CFD00000C0D3F8008006FA04FC4CEA080CC3F841
:10CFE00000C0D3F80CC000EA0C00D860D3F80CC025
:10CFF00001FA04F040EA0C00102AD86004F102049F
:10D00000D8D1BDE8F08F70472D4C266C3543256490
:10D01000A5E72B4C666C35436564A0E7002002460B
:10D020004FF0010E4FF0030904E00132102A00F125
:10D0300002003CD00EFA02F737EA0504F5D1D3F826
:10D0400000A009FA00F4E4430AEA040AC3F800A0C5
:10D05000D3F800B006FA00FA4AEA0B0AC3F800A0B7
:10D06000D3F808A004EA0A0AC3F808A0D3F808B065
:10D070000CFA00FA4AEA0B0AC3F808A0D3F804A095
:10D080002AEA07075F60D3F804A008FA02F747EA24
:10D090000A075F60DF683C40DC60DF6801FA00F48B
:10D0A00001323C43102ADC6000F10200C2D1BDE82D
:10D0B000F08F034C266B3543256350E7943C0408FE
:10D0C0000038024003682DE9F04F03F13F4404F5B6
:10D0D0007E04604EA40A0125345D04F01F06640935
:10D0E000032C05FA06F500F0AF80042C00F0A780B1
:10D0F000022C54D08588B5FA85F0C0F11F0080B2AB
:10D10000C40803EB840400F00700266A80000F27A0
:10D11000874026EA07062662276A01F0030602FA1C
:10D1200000F0721E3843012AC1F3810CC1F30018CC
:10D130002062C1F3411137D90024224601274FF064
:10D14000030E03E0102A04F1020426D007FA02F0CD
:10D15000A84302F10102F5D1D3F800C00EFA04F0A1
:10D16000C04300EA0C0CC3F800C0D3F8008006FAF4
:10D1700004FC4CEA080CC3F800C0D3F80CC000EA69
:10D180000C00D860D3F80CC001FA04F040EA0C009F
:10D19000102AD86004F10204D8D1BDE8F08F2E4CDB
:10D1A000666C35436564A5E7002002464FF0010E2A
:10D1B0004FF0030904E00132102A00F102003CD0D4
:10D1C0000EFA02F737EA0504F5D1D3F800A009FA00
:10D1D00000F4E4430AEA040AC3F800A0D3F800B05C
:10D1E00006FA00FA4AEA0B0AC3F800A0D3F808A02E
:10D1F00004EA0A0AC3F808A0D3F808B00CFA00FA47
:10D200004AEA0B0AC3F808A0D3F804A02AEA0707E1
:10D210005F60D3F804A008FA02F747EA0A075F60E4
:10D22000DF683C40DC60DF6801FA00F401323C4317
:10D23000102ADC6000F10200C2D1BDE8F08F064C7C
:10D24000266B3543256355E7034C266C354325642F
:10D2500050E700BF943C04080038024010B50409B0
:10D26000013C042C17D80D4B33F8142000F00F00AC
:10D2700042FA00F313F001030DD0012303FA00F08A
:10D280000138104032F008F8054A064B125D104490
:10D2900003EBC00010BD002010BD00BFA43C04087B
:10D2A0009C3C0408F4B1002001490248FFF730B863
:10D2B000542600200040014001490248FFF728B8E9
:10D2C0002C2600200004014001490248FFF720B845
:10D2D0002C2600200004014001490248FFF718B83D
:10D2E00004260020000C004001490248FFF710B856
:10D2F000DC2500200008004001490248FFF708B87B
:10D30000B42500200004004002494FF08040FEF7A1
:10D31000FFBF00BF8C25002001490248FEF7F8BF7F
:10D32000642500200000014001490248FEF7F0BFDB
:10D330006425002000000140F0B504684D4DA30AAB
:10D34000AB427AD009D94C4DAB426ED00F35AB42CF
:10D350005AD0103DAB4274D0F0BD023DAB4268D014
:10D3600056D8B3F5801F70D14FF0480E012647798B
:10D37000B0004FEA970C002968D063460227A589C0
:10D380009F4083190CEB43032F4303F1040C3B4DE7
:10D39000BFB245F8231045F82C20A781EFF3118187
:10D3A000502282F31288821905EBC2021369002B06
:10D3B00032D013620433821905EBC202576917B1E8
:10D3C0001F6053690433821905EBC202976917B1D4
:10D3D0001F6093690433821905EBC202D76917B144
:10D3E0001F60D36904330027CAB21F6082F311881B
:10D3F000304405EBC000036A8BB9A38923F0010315
:10D400001B041B0CA381F0BD4FF4887E0626AEE7FB
:10D410004FF0980E0326AAE705EB0E03CBE7A3898E
:10D420009BB243F00103A381F0BD4FF0E80E052647
:10D430009DE74FF0700E022699E74FF0C00E0426CC
:10D4400095E74FF0200E002691E7F0BD0223BF08BC
:10D4500003FA07F7A389094D9BB223EA070387194B
:10D460000CEB470CA3810CF1040345F82C1045F894
:10D47000232093E7030010004100100064250020E2
:10D4800010B5036882480139834282B089B200F046
:10D49000CA80A0F58060834200F0C58000F580401E
:10D4A000834200F0B78000F58060834200F0B280D4
:10D4B00000F58060834200F0AD80764C18882468C7
:10D4C0006408B4FBF2F4013CA4B282B2B3F1804F21
:10D4D0000AD07148834207D000F58060834203D0B0
:10D4E00000F58060834202D122F0700292B26B4854
:10D4F000834200F0A18000F58060834200F0A680A6
:10D5000022F4407200F56C4092B283421A80D962D4
:10D510001C854FD05E4A93424CD001229A821A88D1
:10D5200092B242F001021A80B3F1804F00F098806D
:10D53000594A934200F0968002F58062934200F0CF
:10D54000938002F58062934200F0908002F5806241
:10D55000934200F08D8002F58062934200F08A8051
:10D5600002F57042934200F0878002F570529342B8
:10D5700000F0848002F58062934200F0818002F521
:10D58000806293427ED0A2F5983293427CD002F51D
:10D59000806293427AD002F58062934208BF0D22E6
:10D5A00015D002A84FF0012340F8043D1BF0C6FE41
:10D5B00002B010BD0122002119869A821A883848CB
:10D5C00092B242F0010283421A80ADD10A46354B35
:10D5D00003EBC20301A85C798DF80440012300220B
:10D5E0008DF805308DF807308DF806201BF0A6FE6B
:10D5F0001B2C08D02E2CDBD12B4B019301A81BF048
:10D600009DFE02B010BD294B019301A81BF096FEB0
:10D6100002B010BD1F4C18882468B4FBF2F4013C22
:10D62000A4B282B252E71B4C18882468B4FBF2F40F
:10D63000013CA4B282B257E701201A80D9621C854E
:10D6400098821A8892B202431A8071E701201A80E8
:10D65000D9621C8598821A8892B202431A8063E7C5
:10D660000122B4E70222B2E70322B0E70422AEE7C8
:10D670000522ACE70622AAE70722A8E70822A6E7C8
:10D680000922A4E70A22A2E70B22A0E70C229EE7C8
:10D6900000040140707F00200004004000100040A2
:10D6A00000000140C43004082C01000119010001F0
:10D6B0002DE9F04F013085B0C3B203930B460291C0
:10D6C0008B4C8C4E002B00F09A8032208A4D8B4F71
:10D6D000DFF82C9230F010FA4FF4FA7A4FF0100C79
:10D6E0004FF47A70D9F80430C3F30803002B40F0EC
:10D6F000DE80EFF31183002B40F0D9802968A26807
:10D7000000BF2B689942F9D1D7F800E000FB0EF377
:10D710009B1AB3FBFEF300FB01314FF0010E0191A8
:10D72000D9F80430C3F30803002B40F08780EFF3EF
:10D730001183002B40F082802B68A16800BF2A680B
:10D740009342F9D1D7F800B000FB0BF2521AB2FBAA
:10D75000FBF200FB0323019A9B1AB3F57A7FDFD318
:10D76000BAF1010ABED1039B002B40F0BD804FF4FB
:10D770007A7ADFF88C9150464FF0100CD9F80430CB
:10D78000C3F30803002B75D1EFF31183002B71D184
:10D790002968A26800BF2B689942F9D1D7F800E048
:10D7A00000FB0EF39B1AB3FBFEF300FB01314FF0BD
:10D7B000010E0191D9F80430C3F3080313BBEFF352
:10D7C0001183FBB92B68A16800BF2A689342F9D185
:10D7D000D7F800B000FB0BF2521AB2FBFBF200FBD1
:10D7E0000323019A9B1AB3F57A7FE3D3BAF1010AB6
:10D7F000C4D1029B013B0293002B7FF466AF05B0BE
:10D80000BDE8F08FEFF311888CF31288A1682368CC
:10D81000DB0344BFC6F800E0A1682B6832685FFAFA
:10D8200088F888F31188D7F800801A4400FB08F3C1
:10D830005B1AB3FBF8F300FB0233D2E7EFF3118876
:10D840008CF31288A1682368DB0344BFC6F800E0AC
:10D85000A1682B6832685FFA88F888F31188D7F8D6
:10D8600000801A4400FB08F35B1AB3FBF8F300FBDB
:10D87000023370E7EFF311828CF31288D4F808E0DA
:10D880002368D90303D501233360D4F808E02B685B
:10D890003168D2B282F311883A68194400FB02F36E
:10D8A000A3EB0E03B3FBF2F300FB01317FE7EFF3D1
:10D8B00011828CF31288D4F808E02368D90303D5C9
:10D8C00001233360D4F808E02B683168D2B282F3C8
:10D8D00011883A68194400FB02F3A3EB0E03B3FB73
:10D8E000F2F300FB013118E718462FF067FF3EE71F
:10D8F00010E000E0A8B40020ACB40020B0B40020D8
:10D9000000ED00E0204B5B68C3F3080330B4BBB903
:10D91000EFF31183A3B91D4B1D4C1868A16800BF1C
:10D920001A689042F9D11B4B1C684FF47A7202FBC3
:10D9300004F3591AB1FBF4F130BC02FB001070473C
:10D94000EFF31182102383F3128811498C680B685E
:10D9500013F4803F104B02D0012018608C680B49F3
:10D96000D2B20D68186882F311880A4B19684FF417
:10D970007A72284402FB01F31B1B30BCB3FBF1F3AA
:10D9800002FB0030704700BF00ED00E0ACB40020A7
:10D9900010E000E0B0B40020A8B400202DE9F84F5A
:10D9A0008046FFF7AFFF254E2549DFF8A0E0254A66
:10D9B000254D844610274FF47A740120DEF8043098
:10D9C000C3F30803D3B9EFF31183BBB90B68D2F8E3
:10D9D00008A000BFD1F800904B45F7D1D6F800B0B1
:10D9E00004FB0BF9A9EB0A09B9FBFBF904FB039350
:10D9F000A3EB0C034345E1D3BDE8F88FEFF3118AA5
:10DA000087F31288D2F808B01368DB0344BF28609C
:10DA1000D2F808B00B68D5F800905FFA8AFA8AF35A
:10DA20001188D6F800A0994404FB0AF3A3EB0B037A
:10DA3000B3FBFAF304FB0933DAE700BFB0B400200C
:10DA4000ACB4002010E000E0A8B4002000ED00E03D
:10DA50002DE9F04FDFF830C1474A4849484E494D5B
:10DA60008046102718F1FF38C0F08480DCF80430BD
:10DA7000C3F30803002B5CD1EFF31183002B58D1C3
:10DA80000B68946800BF08688342F9D1D6F800900B
:10DA90004FF47A7000FB09FEAEEB040EBEFBF9FEFC
:10DAA00000FB03EEDCF80430C3F308034FF47A7490
:10DAB0000120FBB9EFF31183E3B90B68D2F808A09A
:10DAC00000BFD1F800904B45F7D1D6F800B004FB69
:10DAD0000BF9A9EB0A09B9FBFBF904FB0393A3EBD0
:10DAE0000E03B3F57A7FBDD2DCF80430C3F308032C
:10DAF000002BDFD0EFF3118A87F31288D2F808B039
:10DB00001368DB0344BF2860D2F808B00B68D5F86F
:10DB100000905FFA8AFA8AF31188D6F800A0994437
:10DB200004FB0AF3A3EB0B03B3FBFAF304FB093387
:10DB3000D5E7EFF3118487F31288D2F808901368C1
:10DB4000D80303D501232B60D2F808900B6828680E
:10DB5000E4B284F31188D6F800A04FF47A7400EB95
:10DB6000030E04FB0AF3A3EB0903B3FBFAF304FB74
:10DB70000E3E97E7BDE8F08F10E000E0ACB4002067
:10DB8000B0B40020A8B4002000ED00E030B4EFF302
:10DB90001183102282F312880649074C0A6807484D
:10DBA000013200250A602560DBB2026883F3118828
:10DBB00030BC7047ACB40020A8B4002010E000E0F6
:10DBC00038B5264B5C69636B73B1A36DA26BD2B1A0
:10DBD000998A1A88C90592B201D5D20700D438BDF6
:10DBE0004FF6F7721A8038BDA36D99891A88890695
:10DBF00092B2EBD59206E9D5E26AD2B19888216B50
:10DC000080B29047E1E799891A880D0692B2DFD574
:10DC10001006DDD5A26A616A8A4219D0A169256918
:10DC2000885C98800132B2FBF5F105FB1122A262FB
:10DC3000CEE79B88E2696169DBB28B54E269E068F8
:10DC4000A36D0132B2FBF0F100FB1122E261BDE7EE
:10DC5000DA6822F08002DA60BAE700BFF8600020DC
:10DC600038B5264BDC68636B73B1A36DA26BD2B180
:10DC7000998A1A88C90592B201D5D20700D438BD55
:10DC80004FF6F7721A8038BDA36D99891A888906F4
:10DC900092B2EBD59206E9D5E26AD2B19888216BAF
:10DCA00080B29047E1E799891A880D0692B2DFD5D4
:10DCB0001006DDD5A26A616A8A4219D0A169256978
:10DCC000885C98800132B2FBF5F105FB1122A2625B
:10DCD000CEE79B88E2696169DBB28B54E269E06858
:10DCE000A36D0132B2FBF0F100FB1122E261BDE74E
:10DCF000DA6822F08002DA60BAE700BFF86000203C
:10DD000038B5264B9C68636B73B1A36DA26BD2B11F
:10DD1000998A1A88C90592B201D5D20700D438BDB4
:10DD20004FF6F7721A8038BDA36D99891A88890653
:10DD300092B2EBD59206E9D5E26AD2B19888216B0E
:10DD400080B29047E1E799891A880D0692B2DFD533
:10DD50001006DDD5A26A616A8A4219D0A1692569D7
:10DD6000885C98800132B2FBF5F105FB1122A262BA
:10DD7000CEE79B88E2696169DBB28B54E269E068B7
:10DD8000A36D0132B2FBF0F100FB1122E261BDE7AD
:10DD9000DA6822F08002DA60BAE700BFF86000209B
:10DDA00038B5264B5C68636B73B1A36DA26BD2B1BF
:10DDB000998A1A88C90592B201D5D20700D438BD14
:10DDC0004FF6F7721A8038BDA36D99891A888906B3
:10DDD00092B2EBD59206E9D5E26AD2B19888216B6E
:10DDE00080B29047E1E799891A880D0692B2DFD593
:10DDF0001006DDD5A26A616A8A4219D0A169256937
:10DE0000885C98800132B2FBF5F105FB1122A26219
:10DE1000CEE79B88E2696169DBB28B54E269E06816
:10DE2000A36D0132B2FBF0F100FB1122E261BDE70C
:10DE3000DA6822F08002DA60BAE700BFF8600020FA
:10DE400038B5264B1C68636B73B1A36DA26BD2B15E
:10DE5000998A1A88C90592B201D5D20700D438BD73
:10DE60004FF6F7721A8038BDA36D99891A88890612
:10DE700092B2EBD59206E9D5E26AD2B19888216BCD
:10DE800080B29047E1E799891A880D0692B2DFD5F2
:10DE90001006DDD5A26A616A8A4219D0A169256996
:10DEA000885C98800132B2FBF5F105FB1122A26279
:10DEB000CEE79B88E2696169DBB28B54E269E06876
:10DEC000A36D0132B2FBF0F100FB1122E261BDE76C
:10DED000DA6822F08002DA60BAE700BFF86000205A
:10DEE00070B4EFF31186502383F31288836B1A68A2
:10DEF000D20720D45D686DB9446A826A944217D013
:10DF000081691144D9600ED9A21A5A608462002234
:10DF100080F85C201A6842F00102F1B21A6081F3C5
:10DF2000118870BC704701698A1A5A608562EEE7F1
:10DF3000012380F85C30F3B283F3118870BC704722
:10DF400003685B6A03B11847704700BF03681B6A28
:10DF500003B11847704700BF03682DE9F041DF693E
:10DF60001FB13B46BDE8F0411847002A164611DDB7
:10DF700004460D460E4400E023689B6820469847FF
:10DF80000028F9D0236815F8011B1B682046984724
:10DF9000AE42F1D1BDE8F08103689B69184700BF2C
:10DFA00003685B69184700BF03681B69184700BF17
:10DFB0000368DB68184700BF03689B68184700BF09
:10DFC00003685B68184700BF03681B68184700BFF9
:10DFD00038B50C46097849B1054601342B68284606
:10DFE0001B68984714F8011B0029F7D138BD00BF02
:10DFF000064B53F820302BB11A689B8851690B42AD
:10E0000001D1138370475383704700BF78B4002059
:10E01000026802F13F4303F57E032DE9F04F9B0AAE
:10E02000544DEB5C03F01F055B090124032B04FA3C
:10E0300005F400F09980042B00F09180022B3ED073
:10E0400001F00306731E012BC1F3810CC1F300180C
:10E050008588C1F3411137D90024234601274FF0A9
:10E06000030E03E0102B04F1020426D007FA03F09C
:10E07000A84303F10103F5D1D2F800C00EFA04F071
:10E08000C04300EA0C0CC2F800C0D2F8008006FAC7
:10E0900004FC4CEA080CC2F800C0D2F80CC000EA3C
:10E0A0000C00D060D2F80CC001FA04F040EA0C0079
:10E0B000102BD06004F10204D8D1BDE8F08F2E4BB4
:10E0C0005D6C2C435C64BBE7002003464FF0010EFF
:10E0D0004FF0030904E00133102B00F102003CD0A3
:10E0E0000EFA03F737EA0504F5D1D2F800A009FAD1
:10E0F00000F4E4430AEA040AC2F800A0D2F800B02F
:10E1000006FA00FA4AEA0B0AC2F800A0D2F808A000
:10E1100004EA0A0AC2F808A0D2F808B00CFA00FA19
:10E120004AEA0B0AC2F808A0D2F804A02AEA0707B4
:10E130005760D2F804A008FA03F747EA0A075760C5
:10E14000D7683C40D460D76801FA00F401333C43FF
:10E15000102BD46000F10200C2D1BDE8F08F064B55
:10E160001D6B2C431C636BE7034B1D6C2C431C6421
:10E1700066E700BF943C0408003802402DE9F04FE8
:10E180004A484B494B4B4C4C4FF0010A4FF00209A7
:10E190004FF004084FF0080C4FF0100E20274026D7
:10E1A000802530F8022B12F0010F03D01960A3F87C
:10E1B00004A0083312F0020F03D01960A3F80490F2
:10E1C000083312F0040F03D01960A3F80480083359
:10E1D00012F0080F03D01960A3F804C0083312F03E
:10E1E000100F03D01960A3F804E0083312F0200FD9
:10E1F00002D019609F80083312F0400F02D01960DE
:10E200009E80083312F0800F02D019609D80083381
:10E2100012F4807F05D04FF4807B1960A3F804B01E
:10E22000083312F4007F05D04FF4007B1960A3F887
:10E2300004B0083312F4806F05D04FF4806B19607E
:10E24000A3F804B0083312F4006F05D04FF4006B4C
:10E250001960A3F804B0083312F4805F05D04FF4BE
:10E26000805B1960A3F804B0083312F4005F05D096
:10E270004FF4005B1960A3F804B0083312F4804F28
:10E2800005D04FF4804B1960A3F804B00833D20BCB
:10E2900004D04FF4004219609A80083301F5806180
:10E2A000A1427FF47EAFBDE8F08F00BFA43C04081C
:10E2B00000000240F4B1002000140240002855D0B4
:10E2C000026802F13F4303F57E032DE9F04F9B0AFC
:10E2D000544DEB5C03F01F055B090124032B04FA8A
:10E2E00005F444D0042B00F09780022B44D001F0B9
:10E2F0000306731E012BC1F3810CC1F3001885883E
:10E30000C1F341113DD90024234601274FF0030EEC
:10E3100003E0102B04F1020426D007FA03F0A8430F
:10E3200003F10103F5D1D2F800C00EFA04F0C043A6
:10E3300000EA0C0CC2F800C0D2F8008006FA04FC17
:10E340004CEA080CC2F800C0D2F80CC000EA0C007D
:10E35000D060D2F80CC001FA04F040EA0C00102B97
:10E36000D06004F10204D8D1BDE8F08F70472E4B85
:10E370001D6C2C431C64BAE72B4B5D6C2C435C6416
:10E38000B5E7002003464FF0010E4FF0030904E00B
:10E390000133102B00F102003CD00EFA03F737EAEC
:10E3A0000504F5D1D2F800A009FA00F4E4430AEA22
:10E3B000040AC2F800A0D2F800B006FA00FA4AEA4D
:10E3C0000B0AC2F800A0D2F808A004EA0A0AC2F8B0
:10E3D00008A0D2F808B00CFA00FA4AEA0B0AC2F810
:10E3E00008A0D2F804A02AEA07075760D2F804A0D0
:10E3F00008FA03F747EA0A075760D7683C40D46039
:10E40000D76801FA00F401333C43102BD46000F1CB
:10E410000200C2D1BDE8F08F034B1D6B2C431C637F
:10E4200065E700BF943C04080038024010B103685F
:10E4300082885A83704700BF10B1036882881A83AC
:10E44000704700BF18B10368828809B95A837047C2
:10E450001A8370470E4B1B8801463BB90D4B0E4A81
:10E460001B7810680BB981F00101EBE70B4B5A697F
:10E470001AB118B91A68106058747047084A1868B9
:10E480001188084A92FBF1F2012102605974704729
:10E4900084B4002086B4002088B400208CB400200E
:10E4A000A4B4002020A1070010B40A4B0A4A1C782B
:10E4B00001238340234052F8200029B9B3FA83F1A5
:10E4C00049095DF8044BBDE7191C18BF01215DF82F
:10E4D000044BB7E774B4002078B4002030B103686F
:10E4E00082881B691A4214BF01200020704700BFB8
:10E4F0002DE9F0410B4E346873691C400FD0DFF8F2
:10E5000028800127B4FA84F3C3F11F0307FA03F547
:10E5100058F8230003689847AC437561F2D1BDE811
:10E52000F08100BF003C0140841E00202DE9F04135
:10E530000B4E346873691C400FD0DFF82880012728
:10E54000B4FA84F3C3F11F0307FA03F558F8230064
:10E5500003689847AC437561F2D1BDE8F08100BF14
:10E56000003C0140841E00202DE9F0410B4E346830
:10E5700073691C400FD0DFF828800127B4FA84F3B8
:10E58000C3F11F0307FA03F558F8230003689847FF
:10E59000AC437561F2D1BDE8F08100BF003C0140A1
:10E5A000841E00202DE9F0410B4E346873691C4035
:10E5B0000FD0DFF828800127B4FA84F3C3F11F03DA
:10E5C00007FA03F558F8230003689847AC437561D0
:10E5D000F2D1BDE8F08100BF003C0140841E002064
:10E5E0002DE9F0410B4E346873691C400FD0DFF801
:10E5F00028800127B4FA84F3C3F11F0307FA03F557
:10E6000058F8230003689847AC437561F2D1BDE820
:10E61000F08100BF003C0140841E00202DE9F04144
:10E620000B4E346873691C400FD0DFF82880012737
:10E63000B4FA84F3C3F11F0307FA03F558F8230073
:10E6400003689847AC437561F2D1BDE8F08100BF23
:10E65000003C0140841E00202DE9F0410B4E34683F
:10E6600073691C400FD0DFF828800127B4FA84F3C7
:10E67000C3F11F0307FA03F558F82300036898470E
:10E68000AC437561F2D1BDE8F08100BF003C0140B0
:10E69000841E0020084A536C10B5084C43F4804394
:10E6A000536420464022002132F062F94FF0FF33DC
:10E6B0002364C4F8433010BD00380240841E00209B
:10E6C0002DE9F041044618460D461646984630F0AE
:10E6D000E9F82768E6722844A07229467D69434616
:10E6E00032462046AC46BDE8F0416047036810B5AD
:10E6F00004461B689847236820469B689847A37B7D
:10E700000133A37310BD00BF38B50B4C23688BB128
:10E710005A68821A002A054604DA0CE05A68AA1AD6
:10E72000002A07DB9A68226018461A689047236817
:10E73000002BF3D138BD38BDC82800202DE9F04F9B
:10E740009F4BA04A1C7897B000F59C412031814630
:10E750000B911160002C00F018859B4A12689042C2
:10E7600040F28380994A089216689949994A07911C
:10E77000013C1C70984B059206F480560A93002EBB
:10E7800040F08180954B1B78022B00F06687042BAC
:10E7900000F05687012B00F00A87914B99450A9BA0
:10E7A0009B7800F2C183002B40F0C2838D4B09930C
:10E7B000089B1E6816F4805740F0B584DFF8549229
:10E7C000059BB3F90610079B5C8BA142B4BF0024E4
:10E7D0000124854B1B6813F080535ED0099A127890
:10E7E00012F001025FD00798408C884241F3CA8042
:10E7F000002C5ED17D4D95F88C10002959D17C48B4
:10E800007C49006890F82D0000250D604D608D60FA
:10E81000794900284ED10870002A4FD0F1064DD515
:10E82000764A1278D20649D4002F47D1002B45D121
:10E83000750243D4724B1B78002B02F09A80714B07
:10E840009B78002C42F028813BB16F4A6F4B1268D5
:10E850001B689B1A002BC2F22B811020634D2BF0FA
:10E8600023FB012385F88D3028E0584B08931E6860
:10E87000584B574A059306F48056574B07920A9314
:10E88000002E3FF47FAF00215748FBF705FC00281E
:10E890007FF478AF0EF040FC74E770029ED4099AC2
:10E8A000127802F00102514D002185F88C10002CE5
:10E8B000A5D0514901200870002AAFD1544B1A78D5
:10E8C000002A40F0C3800799059D488BB5F9007078
:10E8D000898BB5F90250B842B4BF8026002646F0B5
:10E8E0004003B942D8BF33469B0843F08006A84294
:10E8F000B8BF3346059F43F04006A942C8BF334620
:10E900009B08B7F90450B7F9066043F080078542C9
:10E91000C8BF3B4643F040078D42B8BF3B469B080B
:10E9200043F08007314D8642C8BF3B4643F0400765
:10E9300095F88EE08E42B8BF3B469E4501F08A8234
:10E94000A5F8902085F892202D4985F88E300E7814
:10E95000002E01F076815F2B01F000826F2B01F019
:10E960003E82099B1B78DB0770D495F89210002932
:10E970006CD1B5F99030322B68DD95F88E200120EE
:10E98000572A85F8920001F0B485089B1B685C0744
:10E9900041F1C4805A2A41F0C18095F89430002B8F
:10E9A00041F0F78795F8963083F0010385F89630AB
:10E9B000002B42F062800C202BF076FA01F0E1B9D6
:10E9C000C42800206C270020C0280020247A0020C2
:10E9D0005470002048A600204C320020DC45002066
:10E9E000404B4C00143900208CAF0020CC1E00207E
:10E9F0004C3A0020A0AF0020542400204A3A0020C6
:10EA0000901C0020A8870020ACB40020882600209D
:10EA1000BF3200207C290020B5490F68440037B17F
:10EA2000261803EB86067F787678BE4208D2044427
:10EA3000B04EB14803EB840300240B6034800460C3
:10EA4000FA3A0023A5F8902085F89230089BAB4A4B
:10EA50001B680692AA4C5F0700F17E840DF1500AF4
:10EA6000DFF8C4820B940022CAF8042045461492B1
:10EA700040F6330B192740F28336059C02E004353B
:10EA8000A94520D0A978EB78994217FB0160F6D20E
:10EA90006978043117FB036334F911105945A8BF95
:10EAA0005946B1F5617FB8BF4FF461718142E6DD2F
:10EAB0009942E4DC29782729E1D850460435FBF750
:10EAC000DBFAA945DED18F4A0B9C13788E4A9AE86F
:10EAD000030082E80300002B40F03A818B4B1F7843
:10EAE000002F00F0C38301218748FBF7D5FA0028E7
:10EAF00040F04F810A9BDB78002B40F04A8123884D
:10EB00001DB225F00105AEB2B342268000F0CA85E1
:10EB10007F4D02270E204FF014094FF0FF082F7091
:10EB200085F8019085F802802BF0BEF939467648C9
:10EB30002688FBF7B1FA002841F0E18026F00203B5
:10EB40009BB2B34223800AD0714B1421FF220225CD
:10EB50000E201D7059709A702BF0A6F92688DFF8E8
:10EB6000CCA1DFF8CCB19AF80010DBF80400B507AF
:10EB700008BF81F00201C1F34001FFF763FC2421CB
:10EB80006148FBF789FA30B9099A1378590744BFED
:10EB900023F004031370069B1B6813F00A0F1DD0AB
:10EBA00005215948FBF778FA002800F0C28625882D
:10EBB0006F0741F15B8054480621FBF76DFA00288E
:10EBC00000F0A4866E0641F1498007214E48FBF70C
:10EBD00063FA002840F0C085069B1B689D0600F183
:10EBE0001683268848480C21FBF756FA002800F0C7
:10EBF000EB8046F48073B342238009D0444B022556
:10EC00001421FF220E201D7059709A702BF04CF9C0
:10EC1000404B1B78082B00F0E3800E2B00F0E080C7
:10EC2000089B1B685D0548D53B4B1B79002B00F00A
:10EC3000948014213448FBF72FFA002840F092808A
:10EC40001BF09EFC01202BF02BF8002835D0DFF8BC
:10EC5000E48000254FF0CC0902E0DDB2022D2CD873
:10EC600009FB05F76B1C58F80760002EF5D103224D
:10EC700090F9023002960192C278284951F8222078
:10EC8000009218463246334601212AF0E5FB03463E
:10EC900005EB450000EB0010079353B1314608EB3C
:10ECA0008000CC2231F064FE079B48F80730013524
:10ECB000EDB226F0B1FA0028D0D1099B1B78D80715
:10ECC00040F1A1809AF80010154A164DDBF80000BB
:10ECD000012301F0010113702B70FFF7B3FB069BBA
:10ECE0001B685A0700F1038117B0BDE8F08F00BF21
:10ECF0007C2600208026002084260020EC3900207D
:10ED0000483A0020487C00208CAF002024320020AC
:10ED1000B02D002088B10020403F0020042A0408C4
:10ED2000C0240020153900202C29002074B40020B4
:10ED300078B40020F0A2002098F8022098F8033060
:10ED40009A42C0F0988608F10408A8453FF4C6AE80
:10ED500098F800102329F6D1EEE7099B1B78D90714
:10ED60007FF56EAF4FF40F702DF014F80028A4D08B
:10ED700023F042F84FF40F702CF09AFF00289CD03B
:10ED800023F03AF84FF40F702CF092FF0028EFD1E7
:10ED900093E7069B1B689A077FF5B1AE2688F307B9
:10EDA0003FF5CCAE46F001039E4223803FF4C6AE51
:10EDB000B64B1421FF2202250E201D7059709A7047
:10EDC0002BF072F82688B9E626F480739BB2B34222
:10EDD00023807FF413AFAE4B1B78082B7FF41DAF5D
:10EDE000228822F040039BB29A4223803FF418AF5E
:10EDF000A64B02251421FF220E201D7059709A7017
:10EE00002BF052F80CE7A34B1E78002E65D1A24BD5
:10EE10001B68002B61D0DFF8CC82DFF8CC9218F8A9
:10EE2000030C99F800704146A8F103052AF046F852
:10EE3000002800F0BF85002F40F0108605F1080182
:10EE400068792AF03BF8002841F05C859349A87A5C
:10EE50002AF034F8002800F0C085022F41F05E85CA
:10EE60008F49E87B2AF02AF8002841F053858D4924
:10EE7000287D2AF023F8002800F0C085042F41F0F7
:10EE80005D858949687E2AF019F8002841F052858D
:10EE90008649A87F2AF012F8002800F0C085062FC6
:10EEA00041F04485824995F823002AF007F80028AC
:10EEB00041F038857F4995F8280029F0FFFF0028A8
:10EEC00000F0C085082F41F021857B4995F82D0081
:10EED00029F0F4FF002840F0C085784B01221A7019
:10EEE0002FF010FB069B1B685A077FF5FDAE032031
:10EEF0002AF00EF8002800F0C587238813F00804D4
:10EF00007FF4F2AE08200DF0BFFA059E6C486D4DFF
:10EF10006D496E4A6E4BF68800682E80086014605A
:10EF20001C6017B0BDE8F08F13B90A9A01239370E3
:10EF3000684B0A9A1D7892F8214009931B2029F00A
:10EF4000E7FF012C05F00108814600F0218705F05C
:10EF500002050A9A604E92F82030DFF890A15F4FC8
:10EF600006959346052B00F29287DFE813F0C10067
:10EF700084000600FF000101F400012C04BF0523FA
:10EF80008BF82030B8F1000F12D0079B3088B3F90E
:10EF900018100022134661F30F0260F31F4261F361
:10EFA0000F03059861F31F43036003234260069338
:10EFB0004B4DDBF814102A68914280F0328647F2FC
:10EFC00030510322CBF81C108BF8202002200DF0CA
:10EFD00073FA0EF0A1F82968DBF81C200A4404211A
:10EFE000CBF818208BF82010012C40F095872A6868
:10EFF000DBF81810914280F04A879AF8000020B997
:10F0000029F086FF002840F042873A6822F0020289
:10F010003A602A687388642101FB03234FF48060FF
:10F020000022CBF810308BF820208BF803200DF055
:10F0300013FA9BF8203095E729F070FF012807D1DB
:10F04000274D72882B68642101FB0233CBF8103006
:10F05000B9F1000F02D0B379002B7ED1012C00F062
:10F0600016871F4DDBF810102A689142C0F06187A7
:10F0700001238BF82030012C6DD0F379012B79D04E
:10F0800029F0DAFE9BF820306CE700BFB02D00209D
:10F0900088B1002015390020183900206C2D00207F
:10F0A000712D0020762D00207B2D0020802D00204A
:10F0B000852D00208A2D00208F2D0020C0240020C7
:10F0C000F0390020A0240020AC240020A42400203B
:10F0D0009C24002014390020E0810020443A0020C4
:10F0E000ACB40020622D00201C000020901C0020E9
:10F0F000B8F1000FA0D1069D4FF48060B9F1000F68
:10F1000000F0EE820DF0C0F90A9A00231361002D81
:10F110003FF44EAB28462AF0C7FE089B1E6816F443
:10F1200080573FF44BAB1D219E48FAF7B5FF0028EE
:10F130007FF444AB9C4B03F1500903E00433994541
:10F1400000F0AB861A78262AF8D19978DA789142BD
:10F15000F4D2FFF735BB954D5BE729F06DFE032236
:10F160004FF47A738BF82020CBF81C308F4D2DE7AD
:10F170008E4D39E729F060FE032240F6B8338BF854
:10F180002020CBF81C30894D20E7894F3B78002B9D
:10F1900001F09082874BDFF85082DFF850B2DFF841
:10F1A00050A2079345465E46059099460EE019F831
:10F1B00004109847032C28DC88B93B782AF8020F02
:10F1C00001349C4205F1040580F21881072CE1B25C
:10F1D0003046DBF80430EADD984700B2EDE738F856
:10F1E00024206B88801A4FF47A719B1A01FB00F07F
:10F1F00040F6CA0290FBF3F00844904240F2EE233E
:10F20000A8BF10469842B8BF184600B2D5E76A4B6F
:10F210001B78980704D5694D2B7D042B00F294864A
:10F22000268816F0300F3FF4DDAC10200DF014F9F5
:10F2300020200DF011F9624B268800221A70614AD5
:10F240006148624F624D00211160624A39600023BB
:10F25000296041608161036083604361C361136021
:10F260005160936053619161D361BBE4DFF884A185
:10F27000DFF88481584D0AF15A064FF001095146D2
:10F280001AF8010C29F01AFEF8B19AF804009AF85D
:10F2900002309AF803E000EB400105EB8101013BED
:10F2A000D1F8A02003EB4303434493420DD095F8DB
:10F2B000CC2081F89CE009FA00F022EA0000C1F8B5
:10F2C000A030C1F8A47085F8CC000AF1060A5645B2
:10F2D000D5D14249354A424B424D09681B78D2F894
:10F2E00000B00C910B93A5F19C0A00266B6863B3E8
:10F2F0001F7857B3AA68ABEB0202002A0ADB9AF820
:10F30000CC200121B14022EA01020BF5FA718AF802
:10F31000CC20A9600B9AC2B12A7859780432D2B2B3
:10F32000002940F0358307990598098B30F91220A0
:10F3300001F1C800824240F3C2859AF8CC109A7855
:10F3400041FA06F3D80740F167860136042E05F12D
:10F350000C05CBD1FFF7C7BB1F4D95F896305BB1BD
:10F36000099B1B78DE0707D5059BB3F90620079B91
:10F370005B8B9A4200F3428611210A48FAF78CFE11
:10F38000002800F0EE8295F89A302BB995F8943069
:10F3900013B93223A5F89830012385F89A30FFF786
:10F3A0005DBB00BF8CAF00202C290020ACB4002036
:10F3B000F0290020547000204A3A002028880020BC
:10F3C0002A3C0020143D0020C43C002028240020BA
:10F3D0001C250020EC3C0020CC1E0020503A0020D0
:10F3E00070320020681F0020042A0020DC2F00203B
:10F3F000CA1E0020792C0020700B0408DDF8149040
:10F40000B94A0892B949126842F2010AA1FB091BE4
:10F4100012EA0A0A4FEA9B1B00F0A082B44DB548DD
:10F42000B54CB6492E780078267008701EB1B349E5
:10F430000E7886F00106B24D0F2185F82410002BBE
:10F4400000F03184079CAF4BB4F826C0B4F824E038
:10F45000079C10931846248B0078AB4B129495F8B8
:10F4600025400994A94C0F9005940446A3FB000382
:10F470005B0803EB4303E31ADBB2CDF834C002F4BC
:10F4800080520C9397F80080DFF8C4C29F4C0E9115
:10F490000BF5967305F12800CDF844901392DDF832
:10F4A00024900A930995002106967546069B002B29
:10F4B00000F05A83099B33F911201FFA82FEAE45F2
:10F4C0004FEA410303D30D9EB64540F29A835CF8A0
:10F4D0002120934580F05183E25EBAF1000F40F0A5
:10F4E0006F8301314145E25200F10600DEDB0E9AE6
:10F4F000099D874B85F824200F2A49460CBF01221D
:10F500000022DDF8449085F825101A7000F0D283AF
:10F51000804B7849794ADFF83CB20A931C460420B4
:10F5200001230B7013700CF0C7FFDBF80030A168EB
:10F530006268E3605B1A934284BF002384F8213041
:10F54000089B3C781E68002C01F0CB80079A724D16
:10F55000B2F824E0178B6D4916F48056284640F027
:10F56000DF8332460EE0437803EB830303EB830330
:10F5700003F2EE239BB20132944221F8023B00F1E8
:10F5800002000ED015F81230002B00F03E83022B43
:10F59000E9D001320B8821F8023B944200F10200CD
:10F5A000F0D1109A137801331370FFF7E8B8544D77
:10F5B000D5F88830A9EB0303002BFFF6EEA8574AD5
:10F5C000574B527C079933F812308A7DDFED556A2C
:10F5D0009FED556AC97D9BB207EE102A07EE903A5F
:10F5E000B8EEC77AF8EEE77A27EE267A67EE867AE3
:10F5F0000B9AC5F88820C7EE876A40F2FF32FCEE0E
:10F60000E67ACDED067ABDF81830934228BF13464E
:10F6100009B1D31A9BB24548454D0178454C35F8A0
:10F620001160226825F81130921B13440131424DBC
:10F63000236001F00F021B0902702B80FFF7ADB8A9
:10F64000FEF760F93D4B3E4A1B68C31A9342C2BFA6
:10F65000394B00221A80FFF7A0B8079A0599537D0D
:10F66000D27D013B31F913301AB1C3F53B63083346
:10F670001BB2A3F57A7307EE903A9FED327A2E4AC9
:10F68000F8EEE77A40F2FF3167EE877AFCEEE77A30
:10F69000CDED067ABDF818308B4228BF0B4613809B
:10F6A000FFF77BB802212848FAF7F6FC00283FF460
:10F6B00045AA2580B7073FF552AA46F00203B34298
:10F6C00023803FF44CAA214B02201421FF22187002
:10F6D0000E2059709A702AF0E7FB2688FFF73FBA90
:10F6E0000CF0BAFE10E500BF247A0020D34D621062
:10F6F00048270020B000002070320020B100002018
:10F70000CC1E0020E1280020ABAAAAAA48A600200F
:10F71000713200204C320020382A0020386A002044
:10F72000586A00200000C84200008044DD450020E7
:10F73000E4450020E0450020E4AF002048250020FB
:10F7400060E316006F12833F8CAF0020B02D0020C5
:10F75000E4280020ACB40020D44AB2F90030002BD9
:10F76000B8BF5B42B3F5E17FBFF636AAB2F902300B
:10F77000002BB8BF5B42B3F5E17FBFF62DAACC4B9F
:10F7800093ED096AD3ED076A93ED057AD3ED037A19
:10F7900076EE866A77EE877A76EEA66AB7EE007A1C
:10F7A00037EE666A77EEA77AB0EEC66AF0EEE75AF1
:10F7B000B4EEE56AF1EE10FAB4BFB0EE655AB0EE01
:10F7C000465AB5EE405AF1EE10FA40F0E7839FED4D
:10F7D000B97AB4EEE56AF1EE10FA44BF9FEDB66A6D
:10F7E00036EE477AB7EE006AF4EEC66AF1EE10FA2A
:10F7F000C8BFDFEDB26AF5EEC07AC8BF36EEC77A91
:10F80000F1EE10FA48BFB1EE477AF6EE007A27EE35
:10F81000677ADFEDA97A77EE276ABDEEE66A16EE23
:10F82000103A2033402B40F2C486DFEDA56AA54A8A
:10F83000DFEDA37AC2ED006AFDEEC76AC2ED017A80
:10F8400016EE903A2033402BC2ED027A49D8DFED14
:10F850009B7AB4EEE77AF1EE10FA41F3A7809FEDC0
:10F860009A6ADFED9A6A01E0B0EE677AB4EEE67A62
:10F87000F1EE10FA77EE467AF6DC9FED957AF4EE2B
:10F88000C77AF1EE10FA41F18D809FED8F6ADFEDBE
:10F89000916A01E0F0EE477AF4EEE67AF1EE10FAC2
:10F8A00037EE867AF6D4DFED847AB4EEE77AF1EEBD
:10F8B00010FA40F3CE86DFED817A37EEC77A27EE75
:10F8C000076ADFED855ADFED856ADFED857AE6EEC2
:10F8D000256A67EE065AE6EE267AA5EEA77AF0EEDE
:10F8E000477A804BC2ED037A1A6812F4003240F076
:10F8F000A8867D4B1046995C0A2902F10C0200F0A3
:10F900009F8501301828F6D1FFF766B925F040032E
:10F910009BB2AB4223803FF458A9744B02251421BB
:10F92000FF220E201D7059709A702AF0BDFAFFF761
:10F930004CB9238823F00405ADB2AB4225803FF4D7
:10F940003AA96A4B02251421FF220E201D7059701E
:10F950009A702AF0A9FA2588FFF72DB964490E7824
:10F9600064E595F89430002B3FF478A8099B1B7848
:10F9700013F0010302BF012285F8943085F8952029
:10F98000FFF76CB85B4D012185F88C10FEF791BF35
:10F99000012900F06F859AF8CC200123B34001368D
:10F9A0001343042E8AF8CC3005F10C057FF49EAC8D
:10F9B000FFF799B808F10501687929F07FFA002866
:10F9C0003FF444AA012F40F09D8705F10D01A87A6C
:10F9D00029F074FA002840F0A1874749E87B29F014
:10F9E0006DFA00283FF443AA032F40F09387434960
:10F9F000287D29F063FA002840F0A0874049687EFE
:10FA000029F05CFA00283FF443AA052F40F09287C2
:10FA10003C49A87F29F052FA002840F087873A49EC
:10FA200095F8230029F04AFA00283FF443AA072F4B
:10FA300040F07887354995F8280029F03FFA0028EA
:10FA400040F06487324995F82D0029F037FA0028F4
:10FA50003FF443AA092F3FF440AA0926334603EB9B
:10FA600083031D442B4B6978AA7889F800601970CC
:10FA70005A70FFF732BA2848FAF70EFB00283FF415
:10FA80002DA8184B1B6813F4003340F0CA860022DF
:10FA9000154B1046995C142902F10C0200F0728596
:10FAA00001301828F6D1FFF719B800BFF839002047
:10FAB0004C1C0020A7DFA834DB0FC93FDB0F4940F7
:10FAC000000000009C000020DB0FC940E4CB164181
:10FAD000DB0F49C0E4CB16C192E741B99730083C2F
:10FAE00015A82ABE6C2C002060110408B02D00203F
:10FAF00070320020CC1E0020712D0020762D0020B9
:10FB00007B2D0020802D0020852D00208A2D0020B7
:10FB10008F2D00201C3900208CAF00205D2A00F0C2
:10FB200081825B2A00F0CA855E2A00F07086562A20
:10FB300000F0BE86972A00F00587A72A00F04C86C1
:10FB4000B14C23889B0740F0D085A2F1B703072B67
:10FB500000F29282DFE813F08A0290029002900293
:10FB60008402900276027602002D48D05CF82120B3
:10FB700093454FEA4103FFF4AFACA44AA34ED25CD5
:10FB800006EB030E002A00F0AE80022A47D19EF851
:10FB9000012002EB820202EB820202F2EE2292B21A
:10FBA0000329DFBF012606FA01FE0E9E26EA0E0695
:10FBB000CEBF12B212B20E96BAF1000F3FF491AC62
:10FBC0000C9E20F81620B9F1000F03D10F9E022ED3
:10FBD0007FF687ACB0F800904288B0F804E04A4461
:10FBE00096448B4A0FFA8EFE82FB0E62894EA2EB80
:10FBF000EE7226F803E012B24FF0010971E42A46D2
:10FC00004B000A9E4CF8216067E4D3B2022B04D962
:10FC1000032B7FF4BEAC7346ADE43B46ABE4E25A43
:10FC2000BEE77D4A1278002A7FF4C9A9B8F1000F17
:10FC30003FF4C5A9012C40F02A819BF82030FFF742
:10FC400091B931467548FAF727FA002800F0A380E9
:10FC500085F893600DF094FEFEF783BE45F04003F7
:10FC6000AB4223807FF459AEFEF7AFBF45F00403EB
:10FC70009D4223800AD06A4B02251421FF220E20C8
:10FC80001D7059709A702AF00FF92588654B664AE5
:10FC9000B3F90430654982FB0302DB17C3EBA2030F
:10FCA0000B80FEF788BF624B624A109201221A70E5
:10FCB000614B05931B215948FAF7EEF900287FF4B0
:10FCC00027AC5E4BDFF888B10A931946DBF80030A9
:10FCD000CA688B609B1AC82B00F2F484089B1E68CC
:10FCE00006F480565DE4CAB2022A40F2C083032AB9
:10FCF00095D1129A139E002E08BF2A4650E726F08F
:10FD000001039BB2B34223803FF4D4AC0E202F708A
:10FD100085F8019085F802802AF0C6F82688C9E4A3
:10FD200000220FE0437803EB830303EB830303F22A
:10FD3000EE239BB20132944221F8023B00F1020013
:10FD40003FF42FAC15F812301BB1022BEAD00B8810
:10FD5000F0E7D3B2032BFAD83B46EBE7B2F5FA7FD4
:10FD6000FEF674AE95F89230002B7EF46FAE099BD0
:10FD70001B7801210B4085F8921000F0D9830DF01B
:10FD8000CBF92F4B0693089B1F4C1B68FEF763BEF5
:10FD90000025FFF7DEB8099B2A4A1B781060D807B8
:10FDA0007EF5E3AD284B1B78002B3EF44FAE0A9B4B
:10FDB000DB78002B7EF44AAE95F893300133DBB24A
:10FDC000032B85F893307EF641AE204B5B7813B958
:10FDD000002C7EF43BAE0DF09FF9FEF7C2BDB2F5EC
:10FDE000FA7FFEF633AE95F89220002A7EF42EAE0E
:10FDF000099B1B78012185F89210D90700F15184E5
:10FE00000DF0BEFDBDE700BF483A0020382A0020B3
:10FE1000565555553C1F0020442400208CAF00202F
:10FE2000B02D0020F839002067666666343D00205A
:10FE300071320020E128002048A600204C3200202A
:10FE4000EC3900208C26002070320020A88700208A
:10FE5000ACB40020BF4AC0491068B5F99020C6690B
:10FE600081FB06018911F617701A00F5FF407F30FB
:10FE700082423EF769AD891B0A4412B2A5F8902070
:10FE8000FEF762BD08200CF0E7FAFEF72DBF069DD5
:10FE9000002D3EF48DACFFF73DB9B04A079BD488E6
:10FEA000059A1B8BB2F906101A1B914240F3A380EE
:10FEB00023449942B4BF00240124FEF78ABCC83908
:10FEC0008A425EDA9AF8CC109A7841FA06F3D9079A
:10FED0003FF53BAAC2F1000801202AF00DF97B1E74
:10FEE000162B00F23381DFE813F0430259022A0295
:10FEF00082026F02960215020002E901D201BB01E3
:10FF000031018202A5019602150200028E017701DD
:10FF100061011F010701F100AB460A99DBF80020DF
:10FF2000CB69069D13448B61002D3EF441ACFFF775
:10FF3000F1B828F081FF032140F6B8328BF8201089
:10FF4000CBF81C20FFF742B80A2028F0E1FF2688F2
:10FF50000746002800F0FF82F10640F1BE84804D84
:10FF600095F8D470002F7EF43DAE0D2029F09CFF53
:10FF7000012385F8D4302688002F7FF460A9FEF78E
:10FF800031BE9AF8CC300122B24023EA02030BF5CD
:10FF9000FA728AF8CC30AA60FFF7D7B9B4EEE56AF6
:10FFA000F1EE10FA8CBFB0EE654AB0EE464AC4EEF0
:10FFB000054A9FED6C2A9FED6C5ADFED6C1ADFED60
:10FFC0006C2A9FED6C3ADFED6C3A9FED6C4AA4EE23
:10FFD000825AE4EEE12AA4EE857AA4EEA23AB0EECB
:10FFE000475AB0EE637AA4EE837AA4EE874A84EE91
:10FFF000057AFFF7EEBB0124FEF7EBBB002160485A
:020000040801F1
:10000000FAF74AF800287FF4B7A9322385F896005A
:10001000A5F89830FFF7B0B99046002A0CBF012030
:1000200002205AE7574B002201205749574C0B60DA
:10003000574B227006932AF05FF8089B554C1B68BB
:10004000FEF709BD544A5549504B116002225A70BF
:100050004F4B069328F0C0FF089B1B68FEF7FBBCC4
:100060004D4A4F491160494B0022F0E74A4A4D4939
:100070001160464B0122EAE7792A00F0D7847A2AF8
:1000800000F0CD849E2A00F0C2849D2A00F0B7843F
:10009000AE2A00F0AC84AD2A00F0A184EF2A00F073
:1000A0009B84FD2A00F08684FB2A00F0EF84FE2A60
:1000B00000F0E984F72A00F0E3847B2A00F0C3848F
:1000C000089B334A1B680692FEF7C5BCDAF8D000DD
:1000D000DFF8D49090F8361099F802304144642942
:1000E000A8BF642121EAE17180F83610002B40F0AE
:1000F000E78428F045F84EE4DAF8D000DFF8A8905D
:1001000090F8371099F802304144FE29A8BFFE212B
:1001100021EAE17180F83710002BEAD0162028F090
:1001200041FFDAF8D000E4E70C9ADFF87C905178D0
:100130004144B1F5967FA8BF4FF4967121EAE17171
:10014000517099F80230002B40F0BF84DAF8D000EB
:10015000CFE700BF743D0020D34D6210C481002062
:10016000CC1E002099FB243F69A2163E39094E3D62
:10017000E3B59E3E88FA163E45FE7F3FA7DFA834D2
:100180008CAF00203E4100204C3A0020A92F0020D7
:10019000EC390020483A0020503A0020CE2F0020B1
:1001A000B62F0020C22F00205E420020DAF8D000D7
:1001B000DFF8009681784144C829A8BFC82121EA08
:1001C000E171817099F80230002B92D0142028F050
:1001D000E9FEDAF8D0008CE7DAF8D000DFF8D49541
:1001E00041784144C829A8BFC82121EAE171417082
:1001F00099F80230002B3FF47CAF132028F0D2FE98
:10020000DAF8D00075E7DAF8D000DFF8A8950178C1
:100210004144C829A8BFC82121EAE171017099F8B9
:100220000230002B3FF465AF122028F0BBFEDAF855
:10023000D0005EE7DFF87C950C9A99F8023051798E
:1002400041446429A8BF642121EAE1715171002B66
:100250003FF47CAF0E2028F0A5FEDAF8D00048E786
:10026000DAF8D000DFF84C95017A99F80230414471
:10027000C829A8BFC82121EAE1710172002B3FF40F
:1002800038AF0B2028F08EFEDAF8D00031E7DAF82C
:10029000D000DFF82095C17999F802304144C8298F
:1002A000A8BFC82121EAE171C171002B3FF421AF41
:1002B0000A2028F077FEDAF8D0001AE7DAF8D00042
:1002C000DFF8F094817999F802304144C829A8BF39
:1002D000C82121EAE1718171002B3FF40AAF0920A6
:1002E00028F060FEDAF8D00003E7DAF8D000DFF893
:1002F000C494417999F802304144C829A8BFC82163
:1003000021EAE1714171002B40F0EC83112F7FF461
:1003100051AFEEE6DAF8D000DFF89894017999F859
:1003200002304144C829A8BFC82121EAE171017106
:10033000002B40F0D183102F7FF452AFD9E60C9AF6
:10034000DFF8709417794744642FA8BF642727EA21
:10035000E777177128F040FE99F80230002B3FF440
:10036000F5AE0320394628F01DFEDAF8D000C0E6CD
:100370000C9ADFF8409411784144FA29A8BFFA2179
:1003800021EAE171117099F80230002B3FF4DEAEE2
:10039000012028F007FEDAF8D000AAE60C9ADFF870
:1003A0001494917841446429A8BF642121EAE17141
:1003B000917099F80230002B3FF4C8AE022028F06B
:1003C000F1FDDAF8D00094E60C9ADFF8E893D179E1
:1003D00099F80230414481F30801D171002B3FF4B8
:1003E000B5AE052028F0DEFDDAF8D00081E60C9AE3
:1003F000DFF8C093917999F8020041446429A8BFBD
:10040000642121EAE1719171002840F071830D2F80
:100410007FF412AF9AE6DAF8D000DFF89893C1784B
:1004200099F802304144C829A8BFC82121EAE171E6
:10043000C170002B40F01B830F2F7FF4E8AE58E60D
:10044000C2490D6846003DB1321803EB82026D7857
:100450005278AA42BEF4C0AB3044BD4DBD4E00221E
:1004600003EB80030B6032802A60FEF7B5BB129A63
:10047000FFF796BB059931F912209978B2F5617FA3
:100480004FF4966393FBF1F3C0F2F08040F6330132
:100490009142A8BF11460C2FA1F5617191FBF3F1B8
:1004A00000F05B82182F7FF476AAC9B2C8290B46E8
:1004B000A8BFC823DAF8D000C27DDFB297423FF46C
:1004C0006AAA9A1ADFF8EC92C77548BF0732D710AC
:1004D00099F802300137FFB23BB9002F3FF45BAA15
:1004E000384629F009FEFFF756BA182028F05AFDC1
:1004F000F3E7994B99491A684FF47A73B3FBF2F317
:10050000C3EB431203EB8202089B1B68D2001F0659
:10051000A1F8A82000F16C81914A06921268550753
:100520007EF598AA8F4A904C0A211180FEF793BA63
:100530008E49096811F4003140F0C9818C4B08469E
:100540005C5C0F2C01F10C013EF466AA0130182806
:10055000F6D1FEF775BAF20600F1A2810B2028F061
:10056000D7FC002840F06681B30600F1C481814DBC
:1005700095F8D430002B3FF4F8AC002F7EF45FAE3A
:10058000FEF730BB71490E6842003EB1151803EB0F
:10059000850576786D78B542BEF4A0AA02446D4D0B
:1005A0006B4803EB820300220B602A800260FEF797
:1005B00095BAB4EEE77AF1EE10FA40F34182DFED3E
:1005C0006E5A9FED6E6A01E0F0EE676AF4EEC66A5D
:1005D000F1EE10FA76EEE57AF6DCDFED786AF4EE0D
:1005E000E67AF1EE10FA40F12882DFED635A9FEDD2
:1005F000646A01E0F0EE667AF4EEC67AF1EE10FA83
:1006000077EEA56AF6D4DFED5F7AF4EEE76AF1EEF5
:1006100010FA40F3D580DFED5C7A77EEE66A66EE9D
:10062000A65A9FED5A5A9FED5A6ADFED5A7AA5EE07
:10063000856A26EEA55AE5EE867AE5EE276AFFF78B
:10064000F6B8554B1B78032B00F089810022FFF789
:1006500050B9DFED597AB4EEE77AF1EE10FA44BF03
:10066000DFED567A37EEC77AFFF729B90C2F40F045
:10067000D28000273946494B0D915B78BB423FF44D
:100680008AA9DFF83091384620F0CAFF99F8023085
:100690000D991BB1C9B20C2028F084FC0137FFB2C0
:1006A0001BE73F49089B0A602D4A1B6806922E4CA7
:1006B000FEF7D1B93B4A0792FEF7A2BE3A4B0122A0
:1006C0000220B2E4394A089B1E68136823F0040331
:1006D00013600A9A012306F4805682F82130FEF74F
:1006E00060BF06F48056FEF75CBF0023BB2A14935C
:1006F00000F0BA81B72A00F0B381BE2A00F0AE81C3
:10070000BD2A7FF4B9AC4FF6FE71294A1448D68948
:1007100006909089334401449181D3810FF054F8BD
:10072000F8F7BCFC0FF038F8FCF71CF9012029F0B1
:10073000E3FCB5F89020089BFA3A00211B68A5F865
:10074000902085F89210FEF786B900BF7C26002025
:100750008426002080260020147A00203872002091
:10076000EC390020CEB50020483A00206C2C002047
:1007700060110408CC1E0020DB0FC940E4CB1641F9
:10078000E4CB16C1DB0FC93FDB0F494092E741B90B
:100790009730083C15A82ABEA02D0020A92F0020C4
:1007A0008C260020547000208C410020443A002008
:1007B000888700205E420020DB0FC9BFDB0F49C0E5
:1007C0005FED037AF4EEE76AF1EE10FA44BF5FEDF5
:1007D000057A77EEE66A22E7C749089B0A78C74898
:1007E0001B68069042F004020A70C54CFEF733B94C
:1007F000C14A127896077FF58FAEC24A127D042A4D
:100800007FF68AAE1AF060F9089B1B6884E6BE4B3F
:100810000222032009E4182F7FF4BDA800210B4613
:1008200048E6BA4B1B78032B7FF431A929F01EFB55
:10083000FEF754B9B64AB74B528993ED007A07EEEA
:10084000902AF8EEE77AB0EEC77AB4EEE77AF1EEE6
:1008500010FA7FF589AE93ED017AB0EEC77AF4EE27
:10086000C77AF1EE10FA7FF77FAEB3063FF57FAEA1
:1008700020200BF009FE95E80C00A7490A60084605
:1008800041F8043F13F049FFA44B01221A70A44D14
:1008900095F8D430002B00F0FC802688FEF7CFBC02
:1008A00010200BF0D9FD9D4B26881F70012755E6BF
:1008B0000EF08AFFF8F7F2FB0EF06EFFFCF752F82D
:1008C000012029F019FC95F88E20FFF733B98F49E4
:1008D0000978032947D0194630E610200BF0D4FDE3
:1008E00020200BF0B9FD8F49081F13F016FF8B4B2A
:1008F00002221A70CBE720200BF0AEFD874B0022BE
:100900001A70C4E701263346FFF7A9B80826334614
:10091000FFF7A5B803263346FFF7A1B802263346F2
:10092000FFF79DB807263346FFF799B806263346EA
:10093000FFF795B805263346FFF791B804263346EE
:10094000FFF78DB86D49784A089B06914FF4C8713E
:100950001B6811806A4CFEF77EB8CFB28BE629F097
:1009600085FAFEF739B929F081FAB5F99020FEF73A
:1009700067B8002C3DF471AF694D95F88D30002BB0
:100980003DF49CAF29F072FA002385F88D30FDF715
:1009900095BF5A4B85F8941085F895000693584CEE
:1009A000FEF7DBBCB0EE677AFEF77DBFF0EE477A6C
:1009B000FEF763BF002101200DF012FEB5F8902074
:1009C000089B4E491B680691963AA5F89020002294
:1009D00085F89220FEF73FB800210846ECE7FF219A
:1009E000002018F080FF95F88E20FFF757BB0121FB
:1009F000002018F078FF95F88E20FFF74CBB0021FF
:100A0000FF2018F070FF95F88E20FFF741BB002102
:100A1000012018F068FF95F88E20FFF736BB434A97
:100A2000137A43F001031372FFF74ABB3F4A137A6C
:100A300023F001031372FFF743BBF0EE676AE2E5B0
:100A4000F0EE667AC9E54FF4FA6102200DF0C8FDB8
:100A50002A4B0693089B1B68FDF7FDBF022154E655
:100A600019464FF6FE7350E6194602234DE60F2055
:100A700028F098FADAF8D000DEE40B20FDF79CBFEE
:100A80000021042098E70021032095E7002102209F
:100A900092E70127FFF769BA002B3FF46DAF2449B5
:100AA000244A09684FF47A7000FB0313136063E76C
:100AB0001B4D0CF031FB002385F88D30FDF7FEBE99
:100AC000172028F06FFAFFF741BB152028F06AFACB
:100AD000DAF8D000FFF70DBB102028F063FADAF83F
:100AE000D00028E4112028F05DFADAF8D0000DE4F7
:100AF0000D2028F057FA8AE44A3A0020EC39002009
:100B0000483A002028880020DA410020A02D00204B
:100B1000B83C0020503F00202C2500202A3C00201B
:100B2000CC1E0020043C0020D0B500203432002030
:100B3000ACB40020882600202DE9F047C74C63683C
:100B400020469847002800F0C380C54B1B7801223F
:100B5000042B84F83C2000F0BD80B4F91610B4F9E1
:100B60001820B4F91A3021636263A363BD4B1B885C
:100B7000002B69D0BC4DD4ED0C7AD5ED004A95ED33
:100B8000050A95ED015A95ED067AD5ED035A95EDD6
:100B9000026AF8EEE76AD5ED047AA4EEA60AA5EE9D
:100BA000267A67EEC07AA5EEC07AE6EE267A85ED63
:100BB000057AC5ED067A2EF015FFD4ED0D6AD5ED58
:100BC000094A95ED0E0A95ED0A5A95ED0F7AD5ED85
:100BD0000D7AD5ED0C5A95ED0B6A2063F8EEE66AB6
:100BE000A4EEA60AA5EE267A67EEC07AA5EEC07A34
:100BF000E6EE267A85ED0E7AC5ED0F7A2EF0F2FE3E
:100C0000D4ED0E6AD5ED124A95ED170A95ED135AFB
:100C100095ED187AD5ED167AD5ED155A95ED146A3D
:100C20006063F8EEE66AA6EEA40AA6EE857A67EEA1
:100C3000C07AA0EE657AE6EE867A85ED177AC5ED84
:100C4000187A2EF0CFFEA063884FA17F884820F04D
:100C500067F83B88002B40F08480864ED6F8D85049
:100C6000854B1B685B0743D4B5F90070216B636B40
:100C7000A06B824A824E92ED026AD2ED006AD2EDFA
:100C8000015AC91B2163B5F90270DB1B6363B5F917
:100C900004703568C01B07EE900AB8EEE75A07EEFD
:100CA000901AB8EEE77A07EE903AF8EEE77A36EE69
:100CB000056A36EE877A77EEA57A0135A06382ED74
:100CC000026A82ED007AC2ED017A3560BDE8F087F4
:100CD000BDE8F0876B4BB4F91600B4F91810B4F9FD
:100CE0001A2018802063598061639A80A2633DE7CF
:100CF000B6F89820322A00F08880002A66D196F84B
:100D00009530002BB0D06048D6F8F4205F4980FBC6
:100D10000273D217C2EB23122A80D6F8F82080FB88
:100D20000273D217C2EB23126A80D6F8FC30A78A6E
:100D300080FB0302DB17C3EB2213DB1BAB8000231A
:100D4000CB6086F895300EF03FFDF8F7A7F90EF06E
:100D500023FDFBF707FE012029F0CEF9D6F8D85085
:100D600082E7444E226BD6F8D850B3F5C87F4FF0D7
:100D7000000323632B80398818BFD6F8DC00B7F84E
:100D8000008008BF0020B1F5C87F18BFD6F8E0305A
:100D9000616B02440B440020B8F5C87F6063C6F85D
:100DA000DC20C6F8E030688052D0D4F838E0D6F8BD
:100DB000E410A0637144B8F1010FA880C6F8E410F4
:100DC00068D008F1FF38A7F8008049E7D6F8F400AA
:100DD000236B00210344C6F8F43021632980D6F840
:100DE000F800636B61630344C6F8F8306980A36B55
:100DF000D6F8FC00A1630344012AC6F8FC30A980A0
:100E000075D0013AA6F8982079E72B8820491F4829
:100E1000276BA6F8E8300023B5F802E0B5F804C067
:100E2000C0684B608B602363C6F8F4702B80616BE5
:100E3000C6F8F81063636B80A16BC6F8FC10A3635F
:100E4000A6F8EAE0A6F8ECC0C6F8F000AB80D8E758
:100E5000A36BC6F8E430A063A880B2E7003A002094
:100E60002C3E00205C49002060490020D0B50020C5
:100E7000303A0020CC1E0020247A00207880002008
:100E800074800020303E00201F85EB5188870020B1
:100E9000C01F0020DFF804C1DFF8F0E0C8328CFB8F
:100EA00002A9C833D217C2EBE9128CFB03A9DB17E6
:100EB000C3EBE913C8316B802A808CFB013CA28A0A
:100EC000CB17C3EBEC139B1AAB80CEF80C000EF0E3
:100ED0007BFCF8F7E3F80EF05FFCFBF743FD4046C0
:100EE00029F00AF9B7F80080D6F8D85069E7254B01
:100EF00086F89A101B6886F8942013F4003334D1D6
:100F000019462148475C0B2F01F10C0110D0013329
:100F1000182BF7D1B6F8E8101C4B2980B6F8EA7008
:100F2000B6F8EC00D6F8F0106F80A880D96068E7BA
:100F3000174FD7F800C05900BCF1000F09D001EBE2
:100F4000030E00EB8E0E9CF801C09EF801E0E64512
:100F5000E0D20B44DFF848E00E4900EB83000023A9
:100F60003860AEF800300B60D4E70B4B1B78032BD6
:100F700001D00B46C5E728F079FFD6F8D850B6F86F
:100F80009820C7E76C2C0020601104088887002097
:100F90007C26002084260020A02D00201F85EB51F8
:100FA000802600202DE9F0478C4B1B78DB07074695
:100FB00044D58B4B8B4D1C788B4E012C59D01CD3B8
:100FC000022C07D189498A4A09881288914201D99D
:100FD00001241C70EB7AE3B12B89D3B1854B1B78CC
:100FE000BBB120F03FFB002800F09B802B7B8342AD
:100FF0002CBF0121002131700CE07C497E4A098818
:1010000010886A7B801A8842E2DAEB7A0024002B8F
:10101000E2D131782A79632A06D8022C774E00F083
:10102000BA803378002B5DD1754AAB7A8C4238BFD9
:101030000C461470002B4CD1BDE8F0876B4B694D0A
:1010400019885B88E878CB1A83EAE3728142A2EBC5
:10105000E3721DD32B788B421AD3614B1C78E01EB0
:10106000012861D96749097802294FD0012C5E4EC9
:10107000A5D15F4A5D491288687B0988121A91429E
:1010800039DD5D4A12888A42A4D200241C70A1E78F
:10109000B1EB400FE1DC524B1C78E11E012940F21C
:1010A0009480022ADEDC57494F4E0878DFF84481ED
:1010B000DFF844C1DFF838E100210324022834704E
:1010C0001C7088F80010ACF80010AEF8001081D148
:1010D0001FE0012C71D0022C0BD10720BDE8F04796
:1010E00028F0E2BE7068381A474B984258DD72709B
:1010F0009AE7BDE8F08702241C706BE7022AD2DD74
:101100004049097802294FF0040464D13949364E28
:1011100009783E48022ACCBF00220122C280818089
:101120004BE70221317075E7022A9BDC95F800C07D
:1011300091FBFCFC0CF1010CBCF1080FDFF8B4A032
:10114000304EA87895F801E096F800802A4CDFF838
:10115000A090254EA8BF4FF0080C8AF800C01FFAD7
:101160008CFA10FB0AF01EFB0AFE80B2DFF88CA09E
:101170002080A9F800E000244FF0640EB8F1020FBF
:1011800034701C70CAF804408AF801E07FF439AF6B
:101190000FFA8CF1BDE73078A0B901237760337086
:1011A000C2F164021A4B00FB02F083FB0023C0175C
:1011B000A0EBA3506430707036E70820BDE8F0471C
:1011C00028F072BE7368F81A8EE7032C96D10D4989
:1011D000097802299AD0044EFCE600BF1439002099
:1011E000744A0020DC3900207A4A0020383F002071
:1011F000784A00204E3F0020764A002084240020B8
:10120000A02D00202C3E00207F969800303E00202C
:101210006BCA5F6B022828BF022010B4084C094B30
:10122000207000EB8002C0EBC20207495DF8044B5E
:10123000013003EB4203C0B20B6028F05DBF00BF7A
:10124000A92F00203E4100204C3A002008B50EF0A6
:10125000BBFAF7F723FF0EF09FFAFBF783FB0120A1
:10126000BDE8084028F048BF08B501210220FDF77D
:101270001BF9094B1B7803F00503052B08D000214F
:101280000120FDF711F900210846FDF70DF9FEE7F1
:1012900027F0BEF9F3E700BFF460002010B5F7F7C0
:1012A0009DFE094A094B0A490A4C0B48146000226A
:1012B0001A705A7008600EF087FAF7F7EFFEBDE873
:1012C00010400EF069BA00BF4C3A0020A92F002050
:1012D000503A00203E410020B62F002008B50EF005
:1012E00073FAF7F7DBFEBDE808400EF055BA00BF11
:1012F0002DE9F04FBB4B1E788BB0002E40F0818063
:10130000B94BBA4C1D78BA4FDFF808B305F00105A8
:10131000A4F10A0954F80A0CB8B14FF0CC0808FB44
:101320000698FCF74DFE80B154F80A0CFCF740FE1D
:1013300014F8023C024683B924283BD075B354F814
:101340000A0CFCF73DFE0028EED10136032E04F115
:10135000CC04DFD10BB0BDE8F08F012B2ED0022BD7
:1013600033D0032B40D0042B00F06781052B00F015
:101370005581062BE3D114F801ECBEF1000F00F00B
:10138000DB81BEF1010F00F01E8201360023032E27
:1013900004F8023C04F1CC04BCD1DBE7232A54F866
:1013A0000A0C00F08081934B93F842309342B8D1FD
:1013B000F9F73AF8012304F8023CC0E74D2800F0A1
:1013C0006581002304F8023CB9E700233C2804F8B7
:1013D000023C00F055813E28B1D10122032304F8DC
:1013E000012C04F8023CAAE7C028EAD80021042313
:1013F00004F8050C04F8040C04F8061C04F8023C7C
:101400009DE77D4B18680028A4D0F7F723FDDFF88F
:1014100008A27A4DDFF8F491DAF80000FCF7D0FD6D
:10142000002897D0DAF80000FCF7C2FD09281BD08D
:101430003F2819D02B68002B66D1042800F0BD810D
:101440000C2800F0C8807F28E6D0A0F12002D2B29C
:101450005E2AE1D80BB92028DED05A1C09F8030017
:101460002A6015F0D3FCD7E72C68002C59D1644BC7
:10147000264603F5107B002E08BF1E4610335B4541
:10148000F9D1002E00F05281A3F110083068D8F88D
:101490000020075D135D9F42204402EB040140F0F1
:1014A0004381671E4F4422460BB9FD2A5BD907F8DA
:1014B000013F01322A6010F8013F11F801EF9E450B
:1014C000F2D00AB1B04512D04E4815F0A7FCB04595
:1014D00008D356F8100B15F0A1FC092015F096FC66
:1014E0004645F6D9484815F099FC2A6800249442EC
:1014F00092D2661E4E4416F8010F15F087FC2B6839
:1015000001349C42F7D387E70C2864D00A2833D0F3
:101510000D2831D07F2800F0BD80FF2B3FF67CAF37
:1015200093E7374F4FF0000807F5107B464602E07F
:1015300010375F450DD0224639684846F7F7F6FF69
:101540000028F5D1B846002EF2D13E4610375F454F
:10155000F1D1002E9AD1B8F1000F3FF45DAF2948C8
:1015600015F05CFCB5E7511C202009F80200296049
:1015700009F801300A46A5E715F0D1FC23212348DC
:101580002FF00DFA002800F01681A0EB090028606A
:1015900090B1431E19F80310202940F0318109EB66
:1015A000030243B112F8011D202903F1FF304FD18E
:1015B0000346002BF6D12B604FF480720021484681
:1015C0002FF0D6F9074B1B78002B3FF4C3AE0E4823
:1015D00015F024FC20E70E4815F020FC0A4815F011
:1015E0001DFC19E72432002014390020FAA2002043
:1015F000CC1E002080700020AC2D0020182F002071
:10160000380E0408083D0408103D0408182E002078
:10161000183D0408B80B0408142E002014F8063CEA
:1016200014F8051C994273D814F8043C83427FF4E3
:10163000C8AE062304F8023C9DE614F8043C04F806
:10164000030C5A40052304F8042C04F8023C76E607
:101650002B606C4C002204F5107B09F8032002E09B
:1016600010345C4550D02168484612F0F7FB002842
:10167000F6D05C4548D2E368984700232B609BE78F
:10168000032204F8013C04F8022C58E6022304F873
:10169000023C54E6013B00225B482B6009F8032022
:1016A00015F0BCFBB8E6594B5949DB78594ADFF8CD
:1016B00090E11060003318BF01230B70564B574A5E
:1016C000CEF80030564BC7F804214FF0400E0121F0
:1016D00087F80CE1C7F80001C7F8080187F80D5139
:1016E0005048197015F0A6FE4F4815F097FB4FF4BF
:1016F00000600AF0E1FE4D4B93F84230232B3FF49B
:1017000057AE14F8023C34E6494815F087FBB4E7BD
:1017100014F8041C08EB03005140013304F8041CC6
:1017200004F8063C82720AE62246CAE64148A3F162
:10173000100815F073FBCCE69BE80F000DF1280CA8
:101740000DF1080888E80F004CF824ED14F8053C6A
:1017500014F803AC0694624623444FF0010C414652
:1017600006A8ADF822E00793ADF820A08DF824C0BC
:1017700007F0ECFF40B1029A2F4B03924146A4F1CF
:101780000A00029320F07CF9DDF80480002304F8BD
:10179000023CB8F1000F3FF4D8AD54F80A0C20F029
:1017A0002FFA013654F80A0CC047032E04F1CC047A
:1017B0007FF4B0ADCEE52868EAE6204811F014FACF
:1017C0000BB0BDE8F08F14F8053C14F8032C069418
:1017D000234407936E2A4FF0000308930993ADF852
:1017E00020207FF4D2AD06A8F7F722FF06A8F7F76E
:1017F00013FF06A8F7F710FF06A8F7F70DFFC4E5DB
:10180000034626E7380E0408403D0408A92F0020AF
:10181000DC4A0020142E0020D01F002091C20008B6
:1018200024320020443D0408103D0408807000204C
:10183000243D0408083D0408D8B50020182E0020D7
:10184000AC2D00202DE9F04F2DED028B95B0064612
:1018500018F096FE9D4B1D7825B115B0BDEC028B9E
:10186000BDE8F08F9A4B1B685805F6D5994F3A683A
:10187000002A00F02781984CD4F8283103F5F4337E
:1018800048339E42C0F01E81DFF8948294F82C11F8
:10189000D8F80030C4F82861013184F82C11990778
:1018A00001F15C8713F0140F41F0FF8613F0080F6D
:1018B00094F82C3140F0BE8113F0070901F0B08597
:1018C000282B864B029302F098805E209047844B31
:1018D0001B78002B6BD0804C824AD4F83431F31A39
:1018E000934201F23784DFF83CA29AF80080B8F105
:1018F000000F33D1DFF8FC91D9F80000FCF760FB52
:10190000C0B201280ED90228774F42F057813B78A8
:10191000002B42F01082D4F83C31F31AB3F57A6F01
:1019200082F0B78271480268002A40D09AF80030ED
:10193000BBB96F4BD9F800001B689B781E3B012B8D
:101940004FF0020142F24D82043018F0D1FC012226
:1019500000238AF8002084F8483126E063480268B2
:101960002AB3D4F8443140F6B731F31A8B421ED96A
:1019700094F84031002B02F0F380013BDBB284F895
:101980004031002B01F07B8712F8011B94F848715D
:10199000026094F849315748CA190133006884F845
:1019A000482184F84931FCF70FFBC4F84461524ADE
:1019B000029B12781B68012A03F101030C9301F0CA
:1019C000F2824E4B1B786BB14D4F3B6853B1424C8A
:1019D000029BD4F85C21D3F800B0ABEB0202632A7F
:1019E00001F20C82DFF8408198F80090B9F1020F03
:1019F00001F01E873C4F97F87430032B01F0D4841C
:101A0000404B1B7873B1404D2B685BB1324CFBF7F8
:101A100079FFD4F86831039044F61F62C31A9342E9
:101A200000F25C81394B1B78002B7FD1384B1B783F
:101A300043B1294CD4F8B83203F50043E8339E4251
:101A400081F02783334B1B78002B3FF406AF224EE7
:101A5000314C324D06F2C1272068FCF7B1FA00285C
:101A60003FF4FBAE2068FCF7A3FA2B7880465A1EA1
:101A700033B120682A70FCF7A3FA0028F2D1ECE613
:101A800003223946781E2EF059FF96F8C03296F898
:101A9000C12286F8C38283F47F4383F0FF039B1A3D
:101AA0001FFA88F89BB2B8EB132FD5D196F8C22253
:101AB000DBB29A42D0D1781E1BF040FF2B7818443D
:101AC0002870C9E7054B029301E700BF24320020CC
:101AD000247A00206C3A00201C200020ACB40020A6
:101AE000FE3A00203F0D030020000020643A002051
:101AF000603A00205C3A0020FF3A00200C3B0020B6
:101B00000C410020143B0020183B0020843B0020A7
:101B1000953B00201E3B0020243B0020283B00205A
:101B2000EC390020683A00207E2800205E4C2278A4
:101B3000002A41F02F825D4F3C78002C40F0A780B6
:101B40005B4D2878002842F076805A4C5A4DD4F8E4
:101B5000B0122A78594B93FBF2F30B449E42FFF4E8
:101B600065AF574A94F8B432C4F8B062D75CFA074C
:101B700002F15382BB0702F1CF81780702F1108294
:101B80003A074CD54F4BDFF850910D930DF1500BA8
:101B9000A3F13D024BF8202D0021A3F1400203F8F0
:101BA000401C02231121517093705846D9F800103F
:101BB000F7F74EFD5846D9F80410F7F749FDB9F884
:101BC0000E30414903EBC3039B00053381FB032126
:101BD000DB17C3EBA10189B25846F7F751FDB9F8FD
:101BE000103003EB8303590089B25846F7F748FDDC
:101BF000364B1B789B0743BFB9F8081001F57A7183
:101C000089B24FF47A715846F7F73AFD0C9B99F870
:101C10001420591C0C9158461A7018F057FC94F86F
:101C2000B4322978013393FBF1F201FB123384F8CB
:101C3000B432FBE613F0030A7FF43EAE5E20904719
:101C40003B6814209847224B1F4AB3F9043082FBAB
:101C500003124FEAE379C9EBA2090FFA89F95FFA97
:101C600089F018F099FBC9F3072018F095FB3B6841
:101C70005E2098473B681C209847504618F08CFB24
:101C8000504618F089FB94F82C313A6814E6114D4F
:101C9000286E002841F08C868146064B87F800901C
:101CA000C3F8B062C2E600BFF03A00208D3B0020CE
:101CB0008C3B00201C200020943B0020A0860100CB
:101CC000903B0020B03A0020676666664A3A0020E2
:101CD000F83900209C3B00202888002094F86E31C1
:101CE000002B41F0D485DB4B1A6802F00803002B6F
:101CF00048F603414AF60B404BF60F4349F60747B7
:101D000004BF03460F4612F0040F4FF0190118BF2D
:101D10001F46930684F86E1103D547F4804747F0B9
:101D200020071FF091FCC7F30909002842F0B28296
:101D3000C94B9B79002B42F08282984664204FF079
:101D4000FF3A4FF0000C0C970D97ADF83CC0CDF862
:101D500042C0CDF846C0CDF84AC0CDF83890ADF8B5
:101D60003E80ADF840A08DF84E000CAF0FCFDFF8ED
:101D700000E384F805C0AEE80F0097E80F00AEE876
:101D800007002EF8023B71464FF0010C1B0CFE279A
:101D90001F20C82201F81E39A770A27184F807C05D
:101DA000E07094F87E01207180F0F10383EA031360
:101DB000DAB2130983F0E70343EA022383EAC2039A
:101DC0001BB283EA0312D2B2C3F3072383EA1213CE
:101DD00043EA022383EAC2031BB283F0C80282EA09
:101DE0000212D2B2C3F3072383EA121343EA022397
:101DF00083EAC2031BB283EA0C0787EA0717FFB224
:101E0000C3F3072282EA171242EA072200EB0C030F
:101E100082EAC7070EEB0C0084F87E31278011F8A8
:101E2000013B7B4083EA0313DBB21A0982EA1722E3
:101E300042EA032282EAC3031BB29FB28142278097
:101E4000EDD183F07C0383EA0313DBB24FEA131E68
:101E50008EEA172E8EEA032E8EEAC30E0FFA8EFE3E
:101E60001FFA8EF9DFF80CC2A4F800905FFA8EFE1C
:101E70004FEA192984F8289084F827E00CF5D378E4
:101E800004F1220ADCF80000DCF80410DCF8082079
:101E9000DCF80C3047460FC70CF1100CD445B8469F
:101EA000F0D1DCF8000038606C4F9CF8043088F802
:101EB000043007F1270884F8CDE184F8CE9117F8B3
:101EC000011F2868FCF780F8B845F8D194F86F3105
:101ED000002B41F04A856249029A097812680A206B
:101EE00084F86F01002901F084865E4F012938884B
:101EF000069042F2E2820229B7F802E002F0E281A3
:101F0000B8880590032902F0D2820429B7F806B0F8
:101F100002F0C88238890490052902F0BC820629A3
:101F2000B7F80A9002F0B4820729B7F80C8000D005
:101F3000FB8994F87E110C92084680F0300282EA08
:101F40000212D2B217094849079087F07A0747EA88
:101F500002270988207187EAC202444FC1EB0121A0
:101F600087FB010A06984FF0000C60F30F0C0598F0
:101F70006EF31F4C4FF0000E60F30F0E0498CDF877
:101F800034C012B28A440027C917C1EB6A2A60F331
:101F90000F0782EA02110020C9B268F30F00C2F3F2
:101FA000072269F31F4782EA11126BF31F4E63F396
:101FB0001F404FF00009CDF838E00F978DF845A08D
:101FC00010908DF8449042EA01220DF1300C82EA23
:101FD000C107BCE80F003FB287F0C80888EA0818BC
:101FE000DFF88CE084F805905FFA88F8C7F30727DC
:101FF000AEE80F0087EA181747EA08239CE80300B9
:1020000083EAC8031BB283F023024EF8040B82EA72
:102010000212D2B2C3F30723079F83EA121370465A
:1020200043EA022383EAC20207F1010C20F81419E3
:102030004FF023081621FE27C82384F87EC1228092
:1020400084F80780A7700EF1020EE170A3711146AB
:1020500012E000BFEC390020DC390020C321002051
:10206000DC2F002048A60020E4AF002003082080D9
:10207000242000201E20002010F8013B4B4083EA62
:102080000313DBB21A0982EA112242EA032282EA2E
:10209000C3031BB299B270452180EDD183F0F403E4
:1020A00083EA0313DBB24FEA131E8EEA112E8EEA87
:1020B000032E8EEAC30E0FFA8EFE1FFA8EF8D14F52
:1020C000A4F800804FEA182C5FFA8EFE84F81EE018
:1020D00084F81FC07968BA683868FB6807F5D37858
:1020E000A8E80F0038697969BA6904F2A717A8E867
:1020F000070004F2C51884F8C5C184F8C4E117F8D4
:10210000011F2868FBF760FFB845F8D194F87231D9
:10211000002B41F03B84DFF80083D8F8003019220F
:10212000980684F8722140F10683B74BDFF8EC92F1
:102130001B78990741F16E8799F81430042B8CBFF6
:1021400003270227FBF7DEFBB9F81030B9F80820A7
:102150000C9003EB83035B00ADF84A304FF47A70C8
:10216000D9F800300E93B9F80E1099F814E0D9F8A8
:1021700004308DF84C7000FB02F24FF0000C4FF071
:10218000FF300DF1300B8DF84DE0CDF834C01092DA
:102190000F93ADF848101190DE46BEE80F009B4F3C
:1021A0000FC79EE80F0007C73A46182122F81C39CE
:1021B000E17194F87E1184F805C081F0780383EA18
:1021C0000313D8B2030983F0F60343EA002383EA3A
:1021D000C0031BB283EA0310C0B2C3F3072383EA30
:1021E000101343EA002383EAC0031BB283F0C80044
:1021F00080EA001E5FFA8EFEC3F3072080EA1E10FD
:1022000040EA0E2080EACE0000B280F0180383EA94
:102210000313DBB2C0F3072080EA131040EA032067
:1022200080EAC30301F1010EFE204FF01E0C4FF0B7
:10223000C80AA0700237217184F87EE1238084F8F7
:1022400003C084F806A0184612F8011B414081EA39
:102250000111C9B20B0983EA102343EA012383EA7F
:10226000C10109B288B2BA422080EDD181F01801D3
:1022700081EA0111C9B20A0982EA102383EA012323
:1022800083EAC1031BB29AB25E492280DBB2120A12
:1022900004910692059384F8272084F826300F468F
:1022A00001F5D37C04F1220A38687968BA68FB68C2
:1022B000E646AEE80F0010375745F446F4D13868CB
:1022C000CEF800009DF81430DFF854A184F8CC312A
:1022D0009DF8183084F8CD31574617F8011F28684B
:1022E000FBF772FE4A4BBB42F7D1FBF70BFBD8F86A
:1022F0000030D9F80410B9F80820059113F0140F34
:102300004FF47A71D9F800C001FB02F141F07185F8
:102310000F4694F87E910C9089F06A003D4BDFF8EF
:1023200004E1B3F90420CDF834C080EA0010C0B253
:10233000030983F0D50343EA002383EAC0031BB2F9
:1023400083EA0310C0B2C3F3072383EA101343EAFE
:10235000002383EAC0031BB28EFB020ED2174FF09C
:102360000008C2EBAE020598109783F0C80E0E90DD
:102370000F91ADF84A20ADF84480ADF84680ADF835
:1023800048808EEA0E1EDC465FFA8EFEC3F30727F6
:10239000BCE80F0087EA1E1747EA0E2787EACE0E31
:1023A0001A4F84F804900FFA8EFE0FC78EF02103A7
:1023B0009CE8070083EA0313DBB2CEF3072E8EEA14
:1023C000131E09F1010C4EEA032E87E807008EEA7E
:1023D000C30384F87EC14FF021094FF0FE0C4FF08B
:1023E0001C0EC8220C3784F8058084F8079084F806
:1023F00002C084F803E0A7F11C01A27118462380F3
:1024000012E000BF1E2000204A3A002024200020B5
:10241000E9210020F8390020EC390020288800202C
:10242000C32100206766666611F8012B424082EAEC
:102430000212D2B2130983EA102343EA022383EA89
:10244000C20212B290B2B9422080EDD182F068028D
:1024500082EA0212D2B24FEA121989EA102383EA01
:10246000022989EAC2090FFA89F91FFA89F3DD4FB7
:1024700023805FFA89F91B0A059384F8253084F8D4
:10248000249007F5D37C04F1220838687968BA688B
:10249000FB68E646AEE80F0010374745F446F4D136
:1024A0003B88AEF800309DF81430CF4F84F8CA91C5
:1024B000D04684F8CB3118F8011F2868FBF784FD5B
:1024C0004745F8D194F87EC1C84AC94F84F804C082
:1024D0008CF0EB0383EA0313D9B20B0983F0C50335
:1024E00043EA012383EAC1031BB283EA0310C0B2AB
:1024F000C3F3072181EA101141EA002181EAC001FA
:1025000009B20CCA81F0C80E8EEA0E1E5FFA8EFE6A
:102510004FF00008C1F307210D93CDF8388081EA10
:102520001E130C929BE8070043EA0E2383EACE03B6
:102530001BB283F0310E87E807008EEA0E1E5FFAA9
:102540008EFEC3F3072383EA1E1343EA0E2383EAB6
:10255000CE0394F808E0607AA17AE27A277B84F8C7
:1025600005801BB28EEA030E8EEA0E1E5FFA8EFE07
:10257000C3F3072383EA1E1343EA0E2383EACE0341
:102580001BB2584080EA0010C0B2C3F3072383EAAD
:10259000101343EA002383EAC0031BB2594081EAC7
:1025A0000110C0B2C3F3072181EA101141EA0021F2
:1025B00081EAC00109B24A4082EA0212D2B2C1F3F2
:1025C000072383EA121343EA022383EAC2031BB2FE
:1025D0005F4087EA0717FFB2C3F3072383EA1713A5
:1025E00043EA0723607BA17BE27B94F810E094F838
:1025F000118083EAC7031BB2584080EA0010C0B2C2
:10260000C3F3072383EA101343EA002383EAC003DA
:102610001BB2594081EA0111C9B2C3F3072383EA0F
:10262000111343EA012383EAC1031BB25A4082EA31
:102630000212D2B2C3F3072383EA121343EA02233E
:1026400083EAC2031BB28EEA030E8EEA0E1E5FFA05
:102650008EFEC3F3072383EA1E1343EA0E2383EAA5
:10266000CE031BB288EA030888EA08185FFA88F8E4
:10267000C3F3072383EA181343EA082383EAC80352
:10268000A17CE27CDFF874811BB2594081EA011120
:10269000C9B2C3F3072383EA111343EA012383EA90
:1026A000C1031BB25A4082EA0212D2B2C3F307231B
:1026B00083EA121343EA022383EAC2031BB283F0C4
:1026C000270787EA0712D2B2C3F3072787EA121750
:1026D00047EA022787EAC2073FB20CF10103BAB208
:1026E0005FFA87F931204FF0FE0C0C2184F87E311F
:1026F000C8234FEA122E2280E07184F802C0E170F4
:10270000A37184F81490049F84F815E07968BA687E
:10271000FB683868B7F810C0A8E80F0028F803CBAA
:1027200084F8BBE184F8BA911AF8011F2868FBF716
:102730004BFCD045F8D194F876E1BEF1000F41F0A2
:102740001F812C4B94F87EC1B3F90010B3F902201D
:10275000B3F904309FED286A84F805E007EE103ADB
:10276000029B1B680C938CF06A0383EA031306EE4A
:10277000901AD9B20B0983F0D50343EA012383EA07
:10278000C1031BB283EA03115242C9B207EE902A79
:10279000C3F3072383EA111343EA0123F8EEE77A30
:1027A000F8EEE66AB8EEC77A83EAC1031BB267EEB9
:1027B000867A66EE866A27EE067A002083F0C808DD
:1027C000CDED0E7ACDED0D6A8DED0F7A1090119052
:1027D000129088EA08170DF13009FFB2C3F30728F9
:1027E0000EE000BF1E200020E7210020003C00205A
:1027F00024200020F839002088C3E43AC4210020B6
:10280000B9E80F0088EA171848EA072888EAC708D5
:10281000DA4F0FFA88F80FC788F01E0E99E8070004
:102820008EEA0E1E5FFA8EFEC8F3072383EA1E139C
:1028300043EA0E2387E8070083EACE0EC8214FF053
:1028400005094FF01E08FE231C200CF1010284F83C
:10285000769184F80780A370E070A171A7F1100150
:1028600084F804C00C37A4F800E084F87E2111F845
:10287000013B83EA0E0383EA0313DBB21A0982EAFF
:102880001E2242EA032282EAC3031BB21FFA83FE1E
:10289000B942A4F800E0EAD183F0270383EA0313E6
:1028A000DBB21A0982EA1E2E8EEA032E8EEAC30ECE
:1028B0000FFA8EFE1FFA8EF9DFF8E8C2A4F8009036
:1028C0005FFA8EFE4FEA192984F8259084F824E0F7
:1028D0000CF5D37804F1220ADCF80000DCF80410CF
:1028E000DCF80820DCF80C3047460FC70CF1100C60
:1028F000D445B846F0D1A24FBCF80030A8F800305B
:1029000007F1240884F8CAE184F8CB9117F8011F75
:102910002868FBF759FBB845F8D194F87791B9F1DD
:10292000000F41F02780974B1B68052284F8772120
:102930009A0641F16881944ADFED947AD18907EED5
:10294000101AB8EEC77A13F0140F27EE277A01F0A9
:10295000EF848F4BDFED8D6AD3ED007AF8EEE77AE6
:1029600067EEA67A94F87E818A4B8B4AB3F90410FD
:10297000B2F90620894F8A488DED0D7A88F022033E
:1029800083EA03135FFA83FE4FEA1E1383F05903B1
:1029900043EA0E2383EACE03B2F5FA6F1BB2A8BF57
:1029A0004FF4FA6283EA031E5FFA8EFEB2F57A7F75
:1029B000C3F3072383EA1E13B8BF4FF47A724FF0B4
:1029C000640C43EA0E23A2F57A720CFB02F283EA4E
:1029D000CE0E87FB02C780FB01C00FFA8EFEC9171F
:1029E000D217C2EBA7124FF0000AC1EBA0038EF082
:1029F000C8070DF1300BCDED0E7AADF84220ADF8E1
:102A00004030CDF830A0CDF83CA0DC4687EA07176F
:102A1000BCE80F00FFB2CEF3072E8EEA171E4EEA77
:102A2000072E8EEAC707DFF854E1DCF800C084F80F
:102A30000480AEE80F003FB287F04A0383EA031335
:102A4000DBB2C7F3072181EA1311724641EA032181
:102A500008F1010881EAC303142042F810C9FE27D7
:102A60004FF04A0C002184F87E814FF0C808E070D6
:102A700023800EF1040E84F807C0A770617184F8FA
:102A80000680184612F8011B414081EA0111C9B2C3
:102A90000B0983EA102343EA012383EAC10109B247
:102AA00088B272452080EDD181F0140181EA0111D4
:102AB000C9B24FEA111E8EEA102E8EEA012E8EEA5E
:102AC000C10E384B0FFA8EFE1FFA8EFC1F464FEADE
:102AD0001C2A5FFA8EFE84F81DA084F81CE0596859
:102AE00038689A68DB68A4F800C007F5D37CACE8C6
:102AF0000F0038697969B7F818800497ACE80300CB
:102B000004F2A717ACF8008084F8C3A1B84684F893
:102B1000C2E104F2C31A18F8011F2868FBF754FA3F
:102B2000C245F8D1204B214A1B781278013B12F0A4
:102B30000100DBB214BFC0214021172B03D81C4A6F
:102B4000134493F814901B4B1A8893071ABF002361
:102B500041F01001012312F4027F18BF022312F08A
:102B6000100F18BF062312F0200F18BF10230028E3
:102B700041F085814FF003081EE000BF24200020B3
:102B8000C3210020EC390020288800200AD7233CEC
:102B9000F0390020F839002048A60020D34D6210FB
:102BA000676666661E20002088B100201439002068
:102BB000C80B0408483A002094F87EE10C938EF08C
:102BC000460383EA0313DAB2130983F0920343EA5C
:102BD000022383EAC2031BB283EA0310C0B2C3F329
:102BE000072282EA101242EA002282EAC00212B2EE
:102BF00082F0C80C8CEA0C1C00235FFA8CFC0320CA
:102C0000C2F307228DF834908DF8378082EA1C12C7
:102C10008DF835308DF836108DF8380042EA0C28E2
:102C20009BE8070088EACC0C0FFA8CFCDFF80485DF
:102C3000E3718CEA0C19A8E803005FFA89F9CCF378
:102C4000072C8CEA191C4CEA092181EAC90994F87D
:102C500008C088F800200FFA89F98CEA090C8CEA80
:102C60000C1C5FFA8CFCC9F3072282EA1C1242EAB0
:102C70000C22607AA17A94F80B90637182EACC0CF2
:102C80000FFA8CFC80EA0C0080EA0012D2B2CCF37E
:102C9000072080EA121040EA022080EAC20000B257
:102CA000414081EA0111C9B2C0F3072282EA111240
:102CB00042EA012282EAC10212B289EA020989EAE1
:102CC00009195FFA89F9C2F3072282EA191242EA66
:102CD000092294F80CC0607BA17B84F804E082EAAE
:102CE000C90212B28CEA020C8CEA0C1C5FFA8CFC52
:102CF000C2F3072282EA1C1242EA0C2282EACC02C8
:102D000012B2504080EA0010C0B2C2F3072282EA39
:102D1000101242EA002282EAC00212B2514081EA55
:102D20000111C9B2C2F3072282EA111242EA01225A
:102D300082EAC102E17B94F8109013B281EA0302A7
:102D400082EA0212D2B2C3F3072383EA121343EAE0
:102D5000022383EAC2031BB289EA030282EA021257
:102D6000D2B2C3F3072383EA121343EA022383EAAE
:102D7000C2031BB283F0320282EA0212D2B2C3F360
:102D8000072383EA121343EA022383EAC2031BB236
:102D90009AB24FF0FE0C5FFA83FB0920C8210EF1B6
:102DA000010E84F802C04FEA122CE070A17184F881
:102DB0007EE1228084F812C084F811B0049B186868
:102DC00059689A68B3F80CA008F5CC7EAEE8070005
:102DD00008F5D4788EF80290AEF800A084F8B8C157
:102DE00084F8B7B117F8011F2868FBF7EDF8B8456C
:102DF000F8D1039BC4F86831FEF714BEDFF83893AE
:102E0000DFF83883DFF838A341201BF017F8B9F951
:102E1000022088FB0230D217C2EBA00080B21AF069
:102E2000F1FFB9F9002088FB0230D217C2EBA000F5
:102E300080B21AF0E7FFB9F9042088FB0230D217FC
:102E4000C2EBA00080B21AF0DDFF9AF800103868DB
:102E5000FBF7BAF894F8609119F0010800F01C85AE
:102E6000DFF8E082D8F80020910640F18280A54A80
:102E7000DFF8D4921278920740F1B78799F81420BE
:102E8000042A8CBF03230223039347201AF0D6FFA2
:102E9000D9F800001AF082FFD9F804001AF07EFF7A
:102EA000B9F80E2098493868A1FB0232C2F34712E4
:102EB00011460492FBF788F89AF80000D8F8001041
:102EC000049A11F0140F82EA00028AF8002040F000
:102ED000AE86B9F80820642000FB02F01AF05EFF0D
:102EE00099F81480039B386843EA88085FFA88F8E9
:102EF0004146FBF769F89AF80020386888EA02082A
:102F000041468AF80080FBF75FF894F86091B9F1C8
:102F1000000F2ED1DFF834824F201AF08FFFD8F83F
:102F200000001AF03BFFD8F804001AF037FF4846BB
:102F30001AF034FF01213868FBF746F871499AF816
:102F4000002091F80080386808F0010882F0010242
:102F500041468AF80020FBF737F89AF800203868D5
:102F600088EA020211468AF80020FBF72DF894F84F
:102F70006091664AC4F85CB109F10103DBB2A2FBBF
:102F80000312D20802EB8202A3EB420384F8603101
:102F9000FEF728BD5E4B5F491868FAF7DDFF002396
:102FA0002370FEF7C8BD5C4F386800283EF409ADB9
:102FB0004FF0000ADFF89881584CAB465546FAF7B7
:102FC000FFFFF8B1F5B94FF00109AA463868FAF7E2
:102FD000EFFF83B27E2B00F0428498F80120002A94
:102FE00049D194F84C11B1B11B2B84F84C2100F05D
:102FF0000D840D2B45D0386888F80190FAF7E0FF72
:103000000028E3D1AA4650460CAA45495D4616F071
:1030100017FEFEF7D6BC7D2B00F0E18594F8502119
:1030200022B180F02003DBB284F8501194F84B21D8
:10303000062A10D8B4F84E1138681944A4F84E1175
:10304000A118013281F8543184F84B21FAF7B8FF06
:103050000028BBD1D6E7B4F84E2188F8019013447C
:103060009BB21A0A52FA83F3FF2BA4F84E31386848
:1030700002D12C4DA3E73868FAF7A2FF0028A5D1AA
:10308000C0E73868A4F84E21FAF79AFF00289DD1CE
:10309000B8E794F8BC32C4F8B862012B40F26485FA
:1030A00094F8BD222049981801EB8001013202F00A
:1030B0000102CF6A84F8BD22BFB11C4D0D950DF100
:1030C000500B123DA5234BF8205D802284F810316F
:1030D00015233146584684F8112184F81231B84737
:1030E000002840F0C28494F8BC32114A013382FBBC
:1030F0000312A2EBE37202EB42029B1A84F8BC3289
:10310000FEF7A0BC4A3A00201F85EB51CDCCCCCCB9
:10311000883B0020B03A0020583A00201C200020B4
:103120006621002070210020C80B040841210020E6
:103130005655555524200020F839002067666666EC
:1031400010410020EC39002028880020003C00209D
:10315000200000209F4AA04B92F80BC0029A1B88C7
:103160001168D4F838019D4A5FFA83FE1F0A4FF4B4
:103170007A73091A03FB0CF30020994282F81EE0CF
:10318000D77782F814E057759070107180F0D8846A
:10319000934B94481B68DFF868E2934FDEF800C059
:1031A0003968DFF86082BF68DFF85C9280FB030E4D
:1031B000DB17C3EB6E1303F5FA739BB293761B0A0E
:1031C000D37688FB0103C917C1EBA30188FB07086D
:1031D0001177FF170912C7EBA807DFF830E2517724
:1031E0000CF5EA437F4982F8207030333F121B12FE
:1031F00081FB0C019EF800E082F821704FEAEC7729
:10320000C7EB611782F82330784B99F814B083F834
:103210001AB078370CF130011EF0020F82F82470DA
:1032200082F8221000F08984D9F800C0704AD9F8D9
:1032300004E0704FDFF8D88182FB0C1A4FEAEC7182
:1032400082FB0E02C1EBAA514FEAEE7ACAEBA25200
:1032500007FB01CA07FB02E70AEB4A0A07EB47072D
:103260004FEA4A0A7F000392384688FB0A27BF14B8
:1032700088FB0028039A0597B9F80E70079001EBB8
:10328000810102EB820207EBC70701EB810102EB30
:103290008202069109920599BA0004924FEAA84861
:1032A0004FEAEA72CDF820808F1AB9F808800699A3
:1032B000DFF860913A467FB209FB12A207EB810A60
:1032C0000899BBF1050F4FEAE07BA1EB0B073946EC
:1032D00009FB17070998DFF8409149B201EB80011B
:1032E00008F5FA783F48B9F800B01FFA88F8CDF829
:1032F0000C8080FB02084FEAE2720592394A4FEADD
:10330000DE7E4FEADC7C83F80EE083F809C082FBA6
:1033100007E0DFF808C1049A4FEAE777C7EB6010CF
:10332000039F8CFB02EC4FEAE27E9DF80C205A755D
:103330004FEA1727059A03971FFA8AF989B22E4F89
:1033400083F80A90C2EB6812CEEBAC1C4FEA192846
:103350004FEA112E83F810E03F8883F80B804FEA84
:10336000222AD9734FEA20291A73CCF307284FEA8F
:103370001B2134BF4FF0320E4FF0330E9DF80C205E
:1033800083F80DA0587483F812909A7583F807C0DB
:1033900083F8088083F813B0197583F81BE01F7752
:1033A000C4F83461FEF79FBA144B03931868FAF718
:1033B000F7FD00283EF424AB039B01211868FAF7BF
:1033C000EBFD0222002387F8742088F80030FEF716
:1033D00017BB00BF403F0020383F00202C3B00209F
:1033E000F03900201F85EB51C4390020583B0020E4
:1033F0006BCA5F6B806967FF6C3C0020C8290020A6
:10340000F439002067666666288800204A3A002062
:1034100083DE1B4340420F00543A0020D34D62101C
:103420005E2090473B6802209847FF201AF00CFA74
:103430000378FF2B00F08A8490F901304FEAE3799A
:103440005FFA89F9D8B216F0A7FF484616F0A4FF34
:103450003B685E2098473B6803209847FF201AF09E
:10346000F3F90378FF2B00F06C84B0F90830D8B280
:10347000C3F3072916F090FF484616F08DFFD24B94
:103480001B78042B75D0DFF86CB3B4F82E319BF8A1
:103490000010DFF864A393FBF1F201FB123292B249
:1034A000BAF80030A4F82E211201642092B200FB79
:1034B00003134900B3FBF1F342EA03295E203A68A3
:1034C000C3F303231FFA89F949EA030990473B68CC
:1034D000062098475FFA89F016F05EFF4FEA192040
:1034E00016F05AFFB949B4F82E214B7ABAF8009079
:1034F0000132012BA4F82E2100F0F8864A7B09EB5B
:1035000089031FFA83F9002A40F0B3843B685E20E8
:1035100098473B683A209847AD4BA3FB09234FEAF5
:10352000531A1FFA8AFB5FFA8BF016F035FF4FEA49
:103530001B2016F031FF3B685E2098473B683B201C
:103540009847642303FB1A939BB2A248053380FB80
:103550000320DB17C3EBA000C0B216F01DFF002054
:1035600016F01AFFDFF8949299F80630002B40F01D
:103570004B84D8F800309A0640F10D82DFF8808243
:1035800098F800309B0700F1E483DFF878924FF061
:10359000000BDA463B685E2098473B68012098475D
:1035A000504616F0F9FE584616F0F6FE3B685E20CF
:1035B00098473B6809209847002016F0EDFE002050
:1035C00016F0EAFEB9F8123099F814B0B3F5967F08
:1035D0000AD994F82C2102F00F02072A04D842F2EB
:1035E0000F7B9B4528BF9B463B68DFF8E0A15E2030
:1035F00098473B68052098479AF80830002B00F060
:103600005885ABF1200307EE903A9FED737AF8EE00
:10361000E77AF6EE006A67EE877ABEEE007AF5EE9C
:10362000C07AF1EE10FA58BFB0EE667A77EE877A7C
:10363000FDEEE77ACDED027ABDF908B05FFA8BF0C6
:1036400016F0AAFECBF3072016F0A6FE98F800208D
:10365000002391070A930B9300F1628394F83031B1
:10366000012B00F05D83BAF90030DFED5C6A07EEF4
:10367000103ABAF9023007EE903AB8EEC77AF8EE8F
:10368000E77A27EE267A67EEA67ABDEEC77AFDEED8
:10369000E77A0CA88DED0C7ACDED0D7A16F09EFE32
:1036A00094F82C313A68FEF70BB95E2090473B68DE
:1036B000302098474A4BD3F800905FFA89F016F013
:1036C0006BFEC9F3072016F067FE94F82C3113F057
:1036D00003097EF4DAAA434AD4F82811424B9142F6
:1036E000186840F28D8380EAE073A3EBE073384AF8
:1036F0001BB282FB03124FEAE37ACAEB621A4FF065
:10370000640909FB1A390FFA89F90FFA8AFA5FFA84
:1037100089FB5FFA8AF2C9F30729CAF3072A3B68D3
:1037200002925E2098473B6810209847029A104604
:1037300016F032FE504616F02FFE3B685E2098478A
:103740003B6821209847584616F026FE484616F05A
:1037500023FED8F800303A68FEF7A8B8DFF8A89042
:103760009FED228A4FF0240B5E20904758463B681D
:1037700098471F4BF9EC016A9B8A07EE103AF8EE66
:10378000E66AB8EEC77A0BF1010BC6EE877A5FFAEC
:103790008BFB67EE887AFDEEE77ACDED027ABDF914
:1037A00008A05FFA8AF016F0F7FDCAF3072016F0BA
:1037B000F3FDBBF1270F01D03A68D5E7D8F8003008
:1037C0003A68FEF76FB800BFA02D0020403F0020F0
:1037D0001F85EB5167666666E4380E3F0050C347AD
:1037E000F43900203F4B4C00F039002000007A44AF
:1037F000003A00204E3F0020383F0020DC390020F6
:103800004A3A002028880020303A00203868FAF729
:10381000D7FB00287FF4EFAB386884F84A9188F82A
:103820000190FAF7CDFB00287FF4D0ABFFF7EABB9D
:10383000FAF768F8CF4B1B68A0EB030A40F6B833E1
:103840009A4500F2C181DFF868B39BF804303A2B47
:1038500000F03984002388F80030FEF7D1B83868CA
:1038600084F84AA184F84BA184F84C9188F801A00F
:10387000FAF7A6FB00287FF4A9ABFFF7C3BB94F8C7
:10388000481194F84931BC484A1CFEF786B8013B00
:1038900084F86E31FEF71ABBB84A1288D30515D4E6
:1038A000D00600F1E382910600F11385530600F182
:1038B0004685100700F15885D10700F15D8512F0AB
:1038C000020F0CBF4FF004084FF00C08AC49AD4A92
:1038D0000B78D27803F001030AB143F002035320BE
:1038E00003931AF0ABFAA84A128802EB820202EBA9
:1038F0008202900080B21AF085FA00201AF082FA53
:10390000A249A34AB1F800903868C9EBC9194FEA37
:10391000490982FB09324A444FEAE979C9EB622935
:103920005FFA89F94946FAF74FFB9AF80020039BA2
:10393000386848EA030889EA020900218AF80090F9
:10394000FAF742FB41463868FAF73EFB9AF8002046
:10395000386888EA0202D2B211468AF80020FAF7E3
:1039600033FB94F86091FFF7D2BA013B84F86F31D2
:10397000FEF7CCBB09F1FF3984F87791FFF739BA2C
:103980000EF1FF3E84F876E1FEF7C7BF013B84F8F5
:103990007231FEF7D0BE1A077FF582AE7D4B93E8F9
:1039A00003000CAB83E80300184616F017FD77E61A
:1039B0000024DFF80082A1464FF0500A02E0DBB29B
:1039C00083F3118815F804B0601C594628441AF096
:1039D000E3F8002840F022810BF101031C44EFF3CF
:1039E00011838AF312882A6E9442E8DB0022DBB24C
:1039F0002A6683F31188FEF750B94FF0000A5E2063
:103A0000D3F8008084F82CA190473B68DFF8A89198
:103A100017209847504616F0BFFC5F4BA3FB0823C6
:103A20009B0BA9FB03125209C2EB0212A3EB820308
:103A3000D8B216F0B1FC3B685E2098473B6818206E
:103A40009847564BA3FB08239B09A9FB0312520975
:103A5000C2EB0212A3EB8203D8B216F09DFC5046D3
:103A600016F09AFC3A68FDF730BF0C9EAE424FF05C
:103A700000014FD941F2210015F8013B81EA0323EF
:103A80005A0013F4004F80EA020192B289B208BFD3
:103A900011464A0080EA020311F4004F99B293B232
:103AA00018BF0B46590013F4004F80EA010289B297
:103AB00092B208BF0A46530012F4004F80EA030195
:103AC0009BB289B208BF19464A0080EA020311F48A
:103AD000004F99B293B218BF0B465A0013F4004F2F
:103AE00080EA020192B289B208BF11464B0011F47C
:103AF000004F80EA03029BB292B208BF1A465300FD
:103B000080EA030112F4004F9BB289B208BF194644
:103B1000B542B1D15846F5F7D9FD21490C9D214850
:103B20006D1A152DA8BF15252A462CF0FCFE1E4A3D
:103B300094F8BC321570FFF7D8BA2D22DA762FE44C
:103B40001A4B02991B780968C4F83811013B012B04
:103B50003FF61EAB1021022391701371FFF718BBC3
:103B600016F0FCFBFDF721BF0A4A02EB8302D76A7D
:103B7000FFF7A2BA842800205C3A0020483A0020CF
:103B8000143900204C320020383F0020E4AF0020E0
:103B900003082080C80B040873B2E745D34D6210B8
:103BA0002C21002090450020A5450020A02D0020BC
:103BB0006C28002001A502088988888816F0BEFBC1
:103BC00001233B70FDF7AEBEC34AB2F8623100215B
:103BD0000133A2F8623188F80010FDF711BF386890
:103BE00084F85091FAF7ECF900287FF4EFA9FFF779
:103BF00009BA8846894604918B4605918E460691FE
:103C00000B46FEF796B99FEDB57A13F0140F08BF77
:103C1000F0EE477A7EF49DAEFEF7A4BE41463A2010
:103C200019F016FF40EA09095FFA89F9D4E6AC4AAF
:103C30001068FFF753B9AB49AB4B0093A1F13F07B5
:103C4000AA4BAB4A0B9101F8404C0CA8A9490A9722
:103C5000F5F714FE0A9F7B1C0A933C700A9B2922ED
:103C6000591C0A911A700A9BEA22591C0A911A706F
:103C70000A9BC822591C0A910CA81A702AF012FE3D
:103C800000F101080CA942460A982CF04CFE0A9A51
:103C900002EB080301330A9302F808400A9B5A1CFE
:103CA0000A921C700A9B5A1C0A921C700A9B5A1C8E
:103CB0000A921C700A9B5A1C0A921C700A9B5A1C7E
:103CC0000A921C700A9B5A1C0A921C700A9B5A1C6E
:103CD0000A921C700A9B5A1C0A921C700A9B5A1C5E
:103CE0000A921C700A9B5A1C0A921C700A9B5A1C4E
:103CF0000A921C700A9B5A1C0A921C700A9B012291
:103D0000991814A80A911A7050F8283DDB1B3B70D3
:103D100016F0DCFB704B2C70C3F8B062FDF786BE6A
:103D200099E80C0001210AA884F830110A920B933B
:103D300016F054FBB4E4C4F83C6187F80080FDF74A
:103D4000F1BD4FF000094846FFF794BB4846FFF726
:103D50007ABBDFF8B4913B68DFF8B0B15E209847DA
:103D60003B6811209847B9F80E304FF4F36A0AFB0C
:103D700003F38BFB032BDB17C3EB6B3B5FFA8BF07F
:103D800016F00AFBCBF3072016F006FB3B685E201B
:103D9000984719203B689847B9F80E30564A0AFBF5
:103DA00003F382FB0301DB17C3EB611382FB0321E7
:103DB000DA17C2EB6112642101FB1233D8B216F09C
:103DC000EBFA002016F0E8FA98F80030B9F808B0DD
:103DD00098077FF5DCAB5FFA8BFA4FEA1B2BFFF7F6
:103DE000D9BBFAF7D9F8FDF7B2BD01230393FFF76A
:103DF0004CB83B4B1F6807EB87077F00FEF789BA7B
:103E0000CB46CA464A468AE43B68DFF804B1DFF88D
:103E100004A15E2098473B6828209847DBF80030D3
:103E20008AFB032ADB17C3EBAA0A5FFA8AF016F0B3
:103E3000B3FACAF3072016F0AFFA3B685E20984742
:103E40003B6804209847B9F80830002B40F04582C1
:103E5000DBF8083083F310095FFA89F016F09CFA5A
:103E6000C9F3072016F098FAFFF783BB4FF0340828
:103E70002CE59BF8003099FBF3F9FFF747BB1F4A8D
:103E8000D278002A0CBF4FF004084FF00508FEF767
:103E900093BE0123D9F800003B70FAF789F8074672
:103EA000D9F80000FAF784F87B067DF43BAD8A2848
:103EB00000F049828E287DF435AD9AF80030002B51
:103EC0007DF44CAD0E480F4B03602D2384F8403138
:103ED0000268FDF72BBD00BF1C2000200000000081
:103EE000F0390020B03A0020AF2F0020983D0408A0
:103EF000A03D0408AC3D04081F85EB514C32002066
:103F0000643A00202C3B00202888002089B5F81452
:103F1000C439002067666666CC4ACD4B0D920DF120
:103F20005008A2F13D0048F8200D1988DFF84093B1
:103F3000A2F1400300204FF00A0E02F8400C0822C4
:103F400083F801E040469A70F5F79AFBD9F8003003
:103F5000C049DA1781FB0313C2EBA30399B24046B1
:103F6000F5F78EFB1DF07EFBD9F808900C9B4FEA0D
:103F70001942591C0C911A700C9B4FEA1922591CBA
:103F80000C911A700C9B5A1C0C9283F800900C9B9D
:103F90005A1C0C921870404616F098FAFDF7EDBDC9
:103FA000AD4AAA4B12680D930021A3F1400903F812
:103FB000401C2123D10089F8023040F1AB81A74990
:103FC0004FF00308A64B1B885A0500F19F81D807C4
:103FD00000F1CE8103F00203A24A002B1CBF4FF078
:103FE00003081146DFF89CA2424650462CF09BFC89
:103FF00008EB0A0314A80133AAF1020140F8203D9E
:1040000000225B1A08F80A2089F8013016F05EFADF
:10401000FDF7B6BD0127FEF795B8DFF86C929FED6E
:10402000928AB9F90230894A0D9207EE903AF8EE79
:10403000E77A0DF1500867EE887AA2F14003FDEEB1
:10404000E77AA2F13D0148F8201D02F8400C082251
:10405000CDED027A5A701E229A70BDF808104046C3
:10406000F5F70EFBB9F9003007EE903AF8EEE77A73
:10407000404667EE887AFDEEE77ACDED027ABDF82C
:104080000810F5F7FDFAB9F9043007EE903AF8EEAA
:10409000E77A404667EE887AFDEEE77ACDED027A60
:1040A000BDF80810F5F7ECFA404616F00FFAFDF7E8
:1040B00061BD5FFA8BF016F06FF94FEA1B2016F026
:1040C0006BF9FFF7C3BA9BF8021058460CF086FB59
:1040D00000287FF4BFAB5E4A644F654B1288654988
:1040E000654C6648FA611A6809689B68FA62B4F818
:1040F00062210390C7F86CA0FB640068F963FA655D
:10410000F8F79AF8824600287DF475AC039B49467F
:104110001868F9F741FF94F864319BF80320049282
:10412000642B4FF0040287F8742040F0298194F842
:104130006531DFF858B1072B08BF84F865A194F802
:104140006531079307EB0319D9F804100691084667
:104150002AF0A8FBD9F8083005935FFA80F91846D1
:104160002AF0A0FB5FFA80FA079B069909EB0A0286
:1041700008320AEBC9008BF8072023F00F0203F086
:104180000F038BF80A208BF80D304A468BF80E008F
:104190000BF10F002CF0C7FB0BF1060309F109002E
:1041A0001844524605992CF0BEFB9BF8073003F1EA
:1041B0000109D3B1013B5FFA83FC0CF1080CDFF875
:1041C000D0E0DC440BF10700002310F8012B5A402B
:1041D0009300D10883EA420301F0180153404EFADC
:1041E00001F253408445DBB2EFD1254A049809F827
:1041F00002302BF09FFA94F865310022013384F8E5
:10420000653184F864219BF802305BB1039B1BF895
:1042100005101868F9F7D8FE01359BF80230EDB2A9
:10422000AB42F3D894F864310322013384F864314B
:1042300087F8742088F80020039BFFF7B7B80C4B71
:104240008046B3F900A06420FDF77BBDB03A0020A2
:10425000383F0020676666668CAF0020843D040806
:10426000483A0020943D040858A08B4120000020CB
:10427000C4390020F03900201C200020C82900206B
:104280006A9A0020733A0020F8390020649A0020CE
:104290000007090E8E4B8F4A1B88927903EB83032C
:1042A00003EB83034FEA83081FFA88F8002A40F0E3
:1042B0000C814FF0FF330FFA83FA1DF0D3F940B2AF
:1042C000FDF73FBD9846994604939B460593FDF73D
:1042D00030BE4FF02408FFF7F9BA1DF0C3F916F00D
:1042E0005BF8002016F058F8FFF743B93B685E20F2
:1042F00098473B68392098475FFA89F016F04CF8E8
:104300004FEA192016F048F8FFF72CB94FF00308D0
:10431000714967E6714B724A1B68724903F4800366
:10432000002B16BF11464FF004084FF0030849E672
:10433000138907EE903AF8EE677AFEF713BB4FF059
:104340001008FFF7C3BA684B1B6898067DF5EAAA08
:104350009AF80030002B7DF401AB6448644B036095
:104360002D2384F84031B3E54FF02008FFF7AEBAB3
:1043700060494FF0040835E64FF00808FFF7A6BA89
:1043800097F87590DFF880B119F00F0F04BF09F1AD
:1043900001095FFA89F9B9F1070F28BF4FF0010948
:1043A0004FEA091A07EB0A035FFA8AFC187C524BA2
:1043B0001A180023117A8BF80A300BF10D0307EB62
:1043C0000A024CEA000001291870D26803F1010EBC
:1043D0000CD90239C9B2881C1844734603F8012B62
:1043E00083424FEA1222F9D101318E44BA4422F0BD
:1043F000600309F101099AF811205FFA89F9134362
:10440000B9F1080F8EF800300EF1010347D04FEAE2
:10441000091A07EB0A01394A087C374901449A1AFC
:10442000097A02EB010E0CF1100CBEF1130F5FFACA
:104430008CFCC4DDD2B2931DDBB243F040018BF89B
:10444000071003F1010CDFF8C4E0CBB105325FFACD
:1044500082FA0AF1080ADA440EF10100002310F88A
:10446000011B59408B0083EA4103CA084B40244991
:1044700002F0180241FA02F253408245DBB2EED15B
:1044800004980CF80E3087F875902BF053F9BAE6C3
:104490009846FDF74EBD98469946FDF74ABD174A26
:1044A0009A1AC7E7984699460493FDF742BD984685
:1044B000994604939B46FDF73CBD98469946049364
:1044C0009B4605939E46FDF734BD0E4B1B68F2E6F6
:1044D000383F0020DC390020883D0408247A002081
:1044E000843D04087C3D0408EC390020643A002037
:1044F000583B00208C3D0408C80B0408719A00202A
:104500000007090EC4390020649A00206A9A00202E
:104510002DE9F04F2DED0C8B364C95B0636804906F
:1045200020469847002800F07D82B4F8A870002249
:1045300084F85120002F67D1B4F93860206A656A89
:10454000A16AB4F93A20B4F93C30DFF8B4A0301ACB
:104550005B1A521BE06294F85210636304F12C0062
:1045600022631CF0DDFBDAF800309D0042F1E781A8
:10457000D4ED0C5ADFF88CB0D4ED0B7A1E4A9BEDCB
:10458000406ADBED416A9BED427ADBF80C31126840
:10459000B8EEE58AD4ED0D5AF8EEE77AF8EEE58A42
:1045A000013377EE867A38EE268A78EE878A934250
:1045B000CBED407A8BED418ACBED428ACBF80C31C2
:1045C00001F014850D4B029393F800E0BEF1140F37
:1045D00003F00086DBF814210025062A01F2648628
:1045E000DFE812F055194219E417D818E30D6E18D8
:1045F000461800BF38720020244600202C3E0020C0
:10460000247A0020E0220020D44BD549059391F86C
:1046100001901B68D348DFF8A08302904FF47A71B1
:10462000B1FBF3F3C3EB431603EB8603DE00B6B234
:10463000B7420578B8F9060003F00E83D4F87CE0A1
:10464000B4F93820236E0EF1010107EE902A1344CD
:104650000129E1672366F8EEE77A03F00783D4EDDA
:104660001B5AD4ED1D6A07EE101A37EEE56AB8EE54
:10467000C75A012F86EE057A37EE257A77EEC77A8C
:1046800084ED1C7AE7EE866A84ED1B7AF0EE667A9A
:10469000C4ED1E6AC4ED1D6A03F02987D4F890E0CA
:1046A000B4F93A20636E0EF1010107EE902A13442B
:1046B0000129C4F890106366F8EEE77A03F0EE8201
:1046C000D4ED205AD4ED226A07EE101A37EEE56ACF
:1046D000B8EEC75A012F86EE057A37EE257A77EEC7
:1046E000C77A84ED217AE7EE866A84ED207AF0EECF
:1046F000667AC4ED236AC4ED226A03F0D086D4F84A
:10470000A4E0B4F93C20A36E0EF1010107EE902A5B
:1047100013440129C4F8A410A366F8EEE77A03F065
:10472000D682D4ED255AD4ED276A07EE101A37EE5B
:10473000E56AB8EEC75A012F86EE057A37EE257A7C
:1047400077EEC77A84ED267AE6EE276A84ED257A3D
:10475000F0EE667AC4ED286AC4ED276A03F093860A
:10476000DFF858B2A8F80600B4F8A830029A013B66
:104770001578A4F8A83005990023072D4B608B60AD
:10478000CB6040F05781F9F7BDF8029BDFF8288233
:104790001D78049BC01A9BF82131A8F800000693ED
:1047A000002B40F04D816E4B5B79002B01F01383A1
:1047B0006D4B1B78013BDBB2072D8BF8213102F0EA
:1047C000A98400230893694ADBF82C31D2ED006AF2
:1047D000674A9FED686AD2F800A0604A0592049A81
:1047E000DBED4AAADFF8D8819BED499A9FED62AADA
:1047F000DFED62BA9FED62CA9FED62BADFF8C49145
:10480000614FCBF82C21D31A07EE903AF8EE677A75
:10481000B7EE007AC6EE279A08F11C03002507932D
:104820005A4B03932E4677EE6A8A68EEA68AF4EE18
:10483000C78AF1EE10FA88BFF0EE478A544B98ED24
:10484000008A2B44D3ED007AF5EE407AF1EE10FAAF
:1048500017D0504B2B4493ED007A78EE476AB0EEB8
:10486000E66AF4EEC67AF1EE10FA08D5F5EEC06A03
:10487000F1EE10FACCBF37EE878A37EE678A83ED08
:10488000008A454B1A8891073FD0022E3DD0434BFA
:104890009AF82E1033F9163007EE103A079B07EE00
:1048A000901A2B44F8EEE76AB8EEC77AD3ED007A97
:1048B0004B42A6EEA77A700007EE903AF8EEE77A40
:1048C000B4EEE77AF1EE10FA0AD407EE901AF8EE99
:1048D000677AF4EEC77AF1EE10FA88BFF0EE477A05
:1048E0002F4B30490344085EB3F90C30C01A07EE71
:1048F000100AB8EEC77AD207E7EE4A7A41F1018290
:10490000294B93ED008A27EE888A059B9BF864214A
:104910002B4493ED01DA78EE4DCA002A00F0E780CF
:10492000224BDBF8682104991B688A1A9A4240F3EB
:10493000DE809AF84830022B02F05684022E04F0F2
:1049400095861B4B1B689B0700F19280194B87EDE6
:1049500000CA1B689342C0F2C48035E0147A00207C
:10496000247200202C3E00207C8700201081002033
:104970004C3A002000247449CDCCCC3DAE47813F59
:10498000000000000000C842A0AF002094AF00204B
:10499000048100201C240020483A00202824002004
:1049A00088870020F8390020EC8000201881002042
:1049B000EC39002014810020303E0020E02200204D
:1049C00010240020ACAF0020F7EE007AF4EEE7AA46
:1049D000F1EE10FA40F18B8005991F4BD1ED017A71
:1049E00093ED007AF0EEE77AF4EEC77AF1EE10FA82
:1049F0007DD5D1ED027AF0EEE77AB4EEE77AF1EE0A
:104A000010FA74DDD1ED037AF0EEE77AB4EEE77ACE
:104A1000F1EE10FA6BDD114B1B68980761D5104958
:104A2000104B45E0104BDFF844B01D780293072D82
:104A30003FF4A9AE9BF821310693002B3FF4B3AEAF
:104A4000013B8BF82131012D01F0808415B0BDECC4
:104A50000C8BBDE8F08F00BF20810020EC390020D6
:104A6000F8390020888700202C3E0020E02200201A
:104A7000D74BD849DFF8CCE331F916C09EED008A58
:104A8000DFF8C4E387ED00CA03EB460028EE0A8A8C
:104A9000B0F90C00A0EB0C0007EE900AF8EEE77AF4
:104AA000DEF8000027EE888A904278EE4DCA8BDA55
:104AB000B3F90C20B1F900E0C748AEEB020E006874
:104AC0008EEAEE72A2EBEE72824210DAB3F90E3089
:104AD000B1F90220D21A82EAE273A3EBE2739842A0
:104AE00005DD002318468BF86431F9F7B3FCBB4BA6
:104AF0002B4493ED000A039B29EE000A022E20EEC0
:104B00002C0AA3EC010A039304F06585B44BD7ED9E
:104B1000006A93ED007AB34BD3ED007AB24B93ED7C
:104B2000006AB24B67EE277A2B4427EEA87AD3EDC2
:104B3000007A67EE277AF0EE665AECEEA75AB1EEED
:104B4000467AF4EEC75AF1EE10FA08D4F4EEC65ADB
:104B5000F1EE10FA8CBFB0EE467AB0EE657A9BEDBE
:104B60004A6AF7EE007AB4EEE76AF1EE10FAACBFEB
:104B70000123002343B1F0EEE66AF0EEC77AF4EECB
:104B8000E67AF1EE10FA01D587ED007A022E04F0F4
:104B9000DF84974A974B52F826001B68B0EE4D0A07
:104BA0009847954A954B52F826001B6898479AF803
:104BB000373023B1924B1B88002B01F00F81B0EEF0
:104BC0004C8A904B38EE400A2B4493ED008A83EDDB
:104BD000000A9AF8483030EE480A20EE298A53B38A
:104BE000894B1B78D90741F17F80F7EE007AF4EE0C
:104BF000E7AAF1EE10FA9BF86431C1F2D187002BDD
:104C000001F09181DBF86831049AD31A7F4A126867
:104C10009A4210DD7E4BD3ED007AF0EEECCAF4EE52
:104C2000E7CAF1EE10FA42F1E882002318468BF849
:104C30006431F9F70FFC774B9BF874212B4493ED0B
:104C4000000A29EE000A20EE088A89ED008A32B9AE
:104C5000039B87ED00CA03ED01CA89ED00CA013646
:104C6000032E08F1040809F1040907F1040705F10E
:104C700004057FF4E3AD029B1B78072B01F09587B9
:104C8000012B02F04C82002307939BF87C31002B10
:104C900041F0BA83604BDFF8B4A11E68DAF8003047
:104CA00096F82C70DB0401F1B4805C4B5C4A0393F2
:104CB00019465C4B498B5C4D92ED006AD3ED005A6E
:104CC0005A4A5B4BD5ED036A93ED005AD2ED007A58
:104CD000D2ED013AD2ED024A8BED636A07EE101A6B
:104CE000B8EEC77A35EEC64A012336EEC77A8BEDA9
:104CF000616A8BED604ACBED645A8BF89431C7EE54
:104D0000055A338D5A4206EE102A4A4ADFED4A6AA6
:104D100092ED005A494A92ED004AB7EE007AF4EE5D
:104D2000C75A35EE045AF1EE10FA88BFF0EE475A32
:104D300035EE275AB8EEC66AF4EEE65AF1EE10FAEE
:104D400007EE903AB4EEC65AB8BFF0EE665AF1EEEE
:104D500010FACBED675AB8EE677A01F13785B4EEF9
:104D6000C75AF1EE10FA88BFB0EE475A314BDFED6B
:104D7000346AD3ED017A314B93ED014A77EE847AB0
:104D800025EE265A77EEA37AB4EEE76AF1EE10FA32
:104D900008DCB4EEE77AF1EE10FA8CBFB0EE676A89
:104DA000B0EE476A234A738DD2ED027A9FED247AE2
:104DB0005A4204EE102A74EEA77AB8EEC44A26EEE0
:104DC000076AF4EEC47AF1EE10FA4CD440E000BF6A
:104DD00088870020F83900201C810020C080002036
:104DE0008C3400209800002034810020CC800020EA
:104DF0009434002090340020E8340020E434002073
:104E0000483A00204C24002014390020188100204A
:104E100024810020D88000204C3A002054700020CB
:104E20005487002058870020503F0020A0AF00206A
:104E3000CC81002094AF002000000000ACAF002027
:104E40006F12833AEC80002014810020247A002025
:104E500007EE103AB8EE474AB4EEE74AF1EE10FA20
:104E600088BFB0EE674AEA4BDFEDEA7A5B7824EE62
:104E7000274A0BB9B1EE444A002F42F0F080B7EE5A
:104E8000003AE54F3A78002A03F08181E34BDFEDE9
:104E9000E47AD3ED024AD3ED016A93ED037A66EE2C
:104EA000244AE5EE264AE4EE074A63EE244AF4EE8D
:104EB000E74AF1EE10FAB4BFF0EE673AF0EE643A6A
:104EC00098BFF0EE647A012ACDED0C4A03F095818B
:104ED00093ED067AD3ED052AD3ED076A26EE077A1D
:104EE000A5EE227AA4EE267A23EE077AB4EEE77ACC
:104EF000F1EE10FAB4EEE37A8CBFF0EE676AF0EEF2
:104F0000476AF1EE10FA88BFF0EE676AB4BFF0EEC0
:104F1000637AF0EE477A022A8DED0D7A00F0DE809A
:104F200093ED0A7AD3ED092AD3ED0B3A26EE077AF0
:104F3000A5EE227AA4EE237A23EE077AB4EEE67A7F
:104F4000F1EE10FAB4EEE77A8CBFF0EE663AF0EECE
:104F5000473AF1EE10FA98BFF0EE636AA8BFF0EEA0
:104F6000477A032A8DED0E7A00F0B88093ED0E7A21
:104F7000D3ED0D2AD3ED0F3A26EE077AA5EE227A6D
:104F8000A4EE237A23EE077AB4EEE67AF1EE10FA75
:104F9000B4EEE77A8CBFF0EE663AF0EE473AF1EE07
:104FA00010FA98BFF0EE636AA8BFF0EE477A042AC1
:104FB0008DED0F7A00F09280D3ED123AD3ED112AE5
:104FC00093ED137A66EE233AE5EE223AE4EE073AE1
:104FD00063EE233AF4EEE63AF1EE10FAF4EEE73A35
:104FE0008CBFB0EE667AB0EE637AF1EE10FA98BF3D
:104FF000F0EE476AA8BFF0EE637A052ACDED103ACD
:105000006CD0D3ED163AD3ED152A93ED177A66EEF0
:10501000233AE5EE223AE4EE073A63EE233AF4EE61
:10502000E63AF1EE10FAF4EEE73A8CBFB0EE667AAB
:10503000B0EE637AF1EE10FA98BFF0EE476AA8BFBF
:10504000F0EE637A062ACDED113A47D0D3ED1A3A45
:10505000D3ED192A93ED1B7A66EE233AE5EE223A58
:10506000E4EE073A63EE233AF4EEE63AF1EE10FA94
:10507000F4EEE73A8CBFB0EE667AB0EE637AF1EE0A
:1050800010FA98BFF0EE476AA8BFF0EE637A072ADD
:10509000CDED123A22D093ED1E7AD3ED1D2AD3ED39
:1050A0001F3A26EE077AA5EE227AA3EE847A27EE3F
:1050B000037AB4EEE67AF1EE10FAB4EEE77A8CBF3A
:1050C000B0EE666AB0EE476AF1EE10FA8DED137A33
:1050D00098BFF0EE466AA8BFF0EE477A77EEE67A20
:1050E000F7EE006AF4EEE67AF1EE10FACBED4A7ACA
:1050F00044F39A8086EEA77A022ADDED0D7A64EEFB
:10510000874A67EE877ACDED0C4ACDED0D7A2DD02A
:10511000DDED0E7A67EE877A032ACDED0E7A25D083
:10512000DDED0F7A67EE877A042ACDED0F7A1DD078
:10513000DDED107A67EE877A052ACDED107A15D06D
:10514000DDED117A67EE877A062ACDED117A0DD062
:10515000DDED127A67EE877A072ACDED127A05D057
:10516000DDED137A27EE877A8DED137A2D4B1B68D0
:1051700013F0805901F0CB84F6EE005ACBED675A5C
:10518000002A02F0FC87284B28499BED646A0878C6
:10519000D978089126490591B1F906109BF9943107
:1051A00009910399DFF894E09BED635A214E498BF6
:1051B0009EF800800A91BDEEC66A07EE103ADAF852
:1051C00000300899D6ED004ADBED606ADBED617ACC
:1051D00016EE10EABDEEC56A00F0010C03F480562D
:1051E00003F0100003F480030B93B8EEC77A16EEB9
:1051F000103A002941F0B681002841F0F8850748AF
:105200009DED0C5A90ED006A0B4925EE866A17E079
:1052100088B100206F12833A0D3E00203C810020AF
:10522000000000008CAF00204C3200201439002018
:1052300048A6002038810020F8AF0020487C0020DC
:10524000A5EE076AB0EE675AA6EE265ABDEEC56A0D
:1052500016EE108A16EE106AF045A8BF7646434552
:10526000C8BF1E4606EE106AB8EEC66A012A81ED76
:10527000006A00F0DC8090ED046A9DED0D5A25EE89
:10528000866AA5EE076AB0EE675AA6EE265ABDEE0C
:10529000C56A16EE108A16EE106AF045A8BF76466B
:1052A0004345C8BF1E4606EE106AB8EEC66A022A1B
:1052B00081ED016A00F0BB8090ED086A9DED0E5A09
:1052C00025EE866AA5EE076AB0EE675AA6EE265A64
:1052D000BDEEC56A16EE108A16EE106AF045A8BF3C
:1052E00076464345C8BF1E4606EE106AB8EEC66A4B
:1052F000032A81ED026A00F09A8090ED0C6A9DED20
:105300000F5A25EE866AA5EE076AB0EE675AA6EE3A
:10531000265ABDEEC56A16EE108A16EE106AF045E2
:10532000A8BF76464345C8BF1E4606EE106AB8EED3
:10533000C66A042A81ED036A79D090ED106A9DED6A
:10534000105A25EE866AA5EE076AB0EE675AA6EEF9
:10535000265ABDEEC56A16EE108A16EE106AF045A2
:10536000A8BF76464345C8BF1E4606EE106AB8EE93
:10537000C66A052A81ED046A59D090ED146A9DED44
:10538000115A25EE866AA5EE076AB0EE675AA6EEB8
:10539000265ABDEEC56A16EE108A16EE106AF04562
:1053A000A8BF76464345C8BF1E4606EE106AB8EE53
:1053B000C66A062A81ED056A39D090ED186A9DED1E
:1053C000125A25EE866AA5EE076AB0EE675AA6EE77
:1053D000265ABDEEC56A16EE108A16EE106AF04522
:1053E000A8BF76464345C8BF1E4606EE106AB8EE13
:1053F000C66A072A81ED066A19D090ED1C6A9DEDF8
:10540000135A65EE865AE7EE055AE6EEA57AFDEEEA
:10541000E77A17EE900A8645A8BF86468342D8BF32
:10542000734607EE903AF8EEE77AC1ED077ABCF1E1
:10543000000F01F0A581E34B1B68002B41F0AD810B
:10544000E14B1B789BB1387870B1DFF8A483DFF8AB
:10545000A4930026F0B2D9F80030B8EC010A9847BE
:10546000387801368642F5DBD84B1B689847029B9B
:105470001B78072B01F0AE8300230893DAF8003085
:105480000793580501F1BE82D14BD3F8008018F084
:10549000080F41F05982CF4BDFF85CA31F88CE4B39
:1054A000059A1C68B2F906906289914580F262867D
:1054B0004FF07E53CBF82431039A9AF90430168BBF
:1054C000059A9AF80010B2F900009AF801E0002B52
:1054D000A0EB060383EAE37CACEBE37C14BF012280
:1054E0004FF0FF32BCF5FA7FA8BF4FF4FA7C61455C
:1054F00080F23C86ACEB010307EE903AF8EEE77AD7
:10550000B042C5ED007A03DAF1EE677AC5ED007AB4
:10551000059BB3F90200831B83EAE37CACEBE37CDD
:10552000BCF5FA7FA8BF4FF4FA7C614580F21A8679
:10553000ACEB010307EE903AF8EEE77AB042C5ED26
:10554000017A03DAF1EE677AC5ED017A059BB3F9CA
:1055500004108B1B83EAE370A0EBE370B0F5FA7FD5
:10556000A8BF4FF4FA707045CCBFA0EB0E0E4FF001
:10557000000E02FB0EFE07EE90EAF8EEE77AB1426B
:10558000079BC5ED027ABCBFF1EE677AC5ED027AE2
:1055900013F48053059300F0C085B9F5FA6F4A46BD
:1055A000A8BF4FF4FA62B2F57A7F9BF8A431B8BF76
:1055B0004FF47A72A2F57A72002B40F0C7858749C2
:1055C000DFF838E281FB0230D317C3EB6013581CBD
:1055D0006FF0630C3EF910003EF913E00CFB03235F
:1055E000A0EB0E0003FB00F381FB0321DB17C3EBF1
:1055F00061139E440FFA8EFE07EE90EA059BB8EE0B
:10560000E78A85ED038A002B41F03E8117F04003C5
:10561000099300F0FC80724B724993ED019A93ED6F
:10562000026A91ED020A91ED043AD3ED030AD3ED3B
:10563000003AD1ED038AD1ED015AD5ED011A95ED6D
:10564000002A694B30EE435A39EE467A73EEA07A5F
:1056500025EE077A75EEE84A73EEE09A35EEA8AAD1
:1056600024EEA71AB0EE474AAAEE294A17F0030221
:10567000B0EE415A79EE067A70EE036AAAEE295A24
:10568000A6EEA74AA6EEE75AF0EE474AD6EEA74A9C
:1056900034EE014AF6EE006A73EE89AA26EEC44A99
:1056A00035EE475A35EE807AF0EE647AEAEE694AD2
:1056B000A7EE2A4A77EEC17A36EE607A73EE68AAD0
:1056C00025EE265AEAEE297AAAEE875A74EE814A26
:1056D00024EE047A73EEC93A33EE283A64EEA64A11
:1056E00067EEA66AF0EE477AE3EE234A75EEC05AFB
:1056F00036EE206AD5EE057AA5EE057AE5EE866AE5
:10570000F1EE648AB0EE476AB0EE677AA8EEA47A4A
:10571000F1EE663A26EEA43AA3EEA66A64EE260AF5
:10572000F0EE665AB1EE450AA6EEA67AB0EE431A3E
:10573000F0EE606AE3EEA57A64EE243AE5EE246AC0
:10574000A0EE041AA8EEA46AF0EE638A71EEA19AA4
:10575000E0EE240AE5EE258A27EE217A32EE029A5F
:10576000A5EE043A61EE211A66EEA96AE4EEA47A87
:10577000E0EE253A0CBFD5ED022ADFED1C2A83EDC1
:10578000005AE2EE066AA0EE897AE2EE281A33EEBB
:10579000033A67EEA27A73EEA33AB0EE006AA2EE85
:1057A000837AE2EEA36AE1EE867A8BED6C7A85ED80
:1057B000017ACBED6B6AC5ED006ACBED6D7A83EDB6
:1057C000014A1DE088340020747F0020447C0020C2
:1057D000EC390020483A0020503A00201F85EB5158
:1057E0003C1C002098000020741C002000000000D9
:1057F000F8AF00203C7C002080870020E88100205A
:10580000C3ED025AC3ED034A0AB9C5ED027A18F096
:10581000140F03D017F4027F41F00981D94B1B7894
:105820009BB1039B5B8B4B450FDBD74B1B78012B4D
:1058300001F09884192B01F095840E2B05D0082BCC
:1058400003D00023AB60CBF838319BF8DA6116B196
:10585000BB0741F045849BF8E061002E40F0BA8719
:10586000039B9B7F002B00F05084022B01F02C84C3
:10587000032B41F02584039B93F82030C3EB4312A4
:1058800003EB8202D20092B2039BDB7F0233DBB2D6
:10589000002E00F0D185002A00F0CE85BB490968B2
:1058A000B2FBF1F20FFA82F9ABF81092ABB307EE4C
:1058B000909AF8EEE77AF7EE006A86EEA77A012B67
:1058C000D5ED007ADBED896A77EEE67A67EE877AC6
:1058D000CBED857A21D0D5ED017ADBED8A6A77EEC2
:1058E000E67A022B67EE877ACBED867A15D0D5ED76
:1058F000027ADBED8B6A77EEE67A032B67EE877A26
:10590000CBED877A09D0D5ED037ADBED8C6A77EEA3
:10591000E67A67EE877ACBED887A029A1278092ABE
:1059200003F0E082B9F1000F40F3F5839BB39BEDE8
:10593000897ADBED857A77EE877A012BCBED897A50
:10594000C5ED007A21D09BED8A7ADBED867A77EE81
:10595000877A022BCBED8A7AC5ED017A15D09BEDC3
:105960008B7ADBED877A77EE877A032BCBED8B7A18
:10597000C5ED027A09D0DBED8C7A9BED887A77EE63
:10598000877ACBED8C7AC5ED037A013B022BB8BF49
:105990000223DBB20693002E069818BF022023785C
:1059A000DFED7F6AA27807EE903AF8EEE77AB0EE84
:1059B000007A67EEA67A029BF4EEC77AF1EE10FA4F
:1059C000197840F3EE86DFED736A37EEC77AB0EEF2
:1059D000676AA7EE266AF0EE466A95ED007A9FEDBB
:1059E0006E6A27EE066AF0EEC65A8BED536ACBED6F
:1059F000565A9AB107EE102AB8EEC75A9FED687A48
:105A000066EE064A25EE075AB7EE007A37EE457A7B
:105A100064EEA54AA4EE857A26EE076A9FED5F7ACA
:105A2000637926EE877A27EE067ACBB1DFED5C6AE2
:105A30009FED5C6A65EEA65A06EE903AF8EEE66ACD
:105A400065EEA65AF4EEC65AF1EE10FA01F3D882CA
:105A5000B7EE006A76EE655AC6EE256A27EE267A1C
:105A60000C299FED518ADFED516A01F05780B4EEA9
:105A7000C87AF1EE10FA98BFB0EE478AB4EEE68A23
:105A8000F1EE10FAB8BFB0EE668A8BED4C8A0028B2
:105A900000F0F480B0EE007AF4EEC77AF1EE10FA7E
:105AA00005DD37EEC77ADFED3B6AE7EE267A95ED46
:105AB000017ADFED396A27EE267AF0EEC75A8BEDD0
:105AC000547ACBED575A9AB106EE902A9FED346A7C
:105AD000F8EEE66A27EE075A66EE866AB7EE006AC7
:105AE00036EE666A25EE255AA5EE266A27EE067A78
:105AF000DFED2A6AA37967EEA67A67EE877AABB103
:105B000007EE103AB8EEC77A9FED256ADFED256AF9
:105B100027EE257A27EE067AB4EEE67AF1EE10FA51
:105B200041F38682DFED1A6A67EEA67A0C2901F04E
:105B30001880DFED1D6A9FED1D7AF4EEE67AF1EE36
:105B400010FA88BFF0EE667AF4EEC77AF1EE10FA3A
:105B5000B8BFF0EE477A0128CBED4D7A40F38E8046
:105B60006378DFED0F6A07EE903AF8EEE77AB0EE71
:105B7000007A67EEA67A637AF4EEC77AF1EE10FA4D
:105B80001CDD15E0901C002088B1002084B10020AD
:105B90000000C842D7A368416F12033B000048438E
:105BA0000AD7233CA4707D3F00C0F94400C0F9C46B
:105BB00037EEC77A5FED096AE7EE267A95ED027A4D
:105BC0005FED0B6A27EE267AF0EEC75A8BED557A19
:105BD000CBED585A9BB106EE903A1FED0F6AF8EEE6
:105BE000E66A27EE075A66EE866AB7EE006A36EE78
:105BF000666A25EE255AA6EE856A27EE067A5FEDDF
:105C0000196AE37967EEA67A67EE877AFBB107EE49
:105C1000103AB8EEC77A1FED1E6A5FED1E6A27EED6
:105C2000257A27EE067AB4EEE67AF1EE10FA01F361
:105C3000EB81B5EEC07AF1EE10FA02F18084B7EE96
:105C4000006A36EE477AC6EE076A67EEA67A0C2936
:105C500000F07F875FED2C6A1FED2C7AF4EEE67A78
:105C6000F1EE10FA88BFF0EE667AF4EEC77AF1EE44
:105C700010FAB8BFF0EE477ACBED4E7A092900F062
:105C80003887039B93F82140002C40F0ED86BB4BF6
:105C9000D3F8008000238BF8E03118F0200F07D0F4
:105CA00017F0300F04D0B64B1B78DB0702F1CE8122
:105CB00016F08AFB002840F08183B24B1B7823B991
:105CC000B14B9B78002B41F02082029B1D78072D61
:105CD0007EF4B9AEF7F716FE029AAC4B1578089A27
:105CE000801AD880FEF7AFBE9BF86431002B3EF4DB
:105CF000A2AF002318468BF86431F8F7ABFBFEF730
:105D00009ABFB1F900209BED567AB1F90200DBEDA4
:105D1000576A9F4982EAE273A3EBE273F4EEC76A23
:105D200080EAE072F1EE10FAA2EBE072B4BFB0EEDE
:105D3000476AB0EE666A9342B8BF134607EE103A60
:105D40000B78B8EEC77A27EE0A7A002B40F0BC80B9
:105D5000904BD3ED005AF4EEEB5AF1EE10FA41F10C
:105D6000BA81B7EE005A75EE654ADFED8B6A9FED9A
:105D70008B5A8B4B36EEC77A24EE855AD3ED006AE8
:105D8000E7EE055A65EEA65AF5EEC05AF1EE10FAA6
:105D900040F2B986CBEE256AB7EE007AF0EE475AAC
:105DA000E6EE665AF0EE656AF4EEC76AF1EE10FAB6
:105DB00088BFF0EE476AF5EEC06AF1EE10FAB8BFA0
:105DC000F0EE4C6A774B93ED007A67EE877AA7EE98
:105DD000A68AFEF79ABD0123FEF7EEBC724B734A0A
:105DE0002B4493ED007AD2ED007A714B67EE277A5F
:105DF000F7EE006AF4EEE67AF1EE10FA93ED007A2F
:105E000088BFF0EE667A67EE877A27EE888AFEF71B
:105E1000D8BE684B684D1B78D5ED037A13F0010F9F
:105E2000664B039304BF1B8BABF88831644B1B8814
:105E300007EE103AB8EEC77AF4EEC77AF1EE10FA30
:105E400042F2AE805F4A128807EE102AB8EEC77A97
:105E5000F4EEC77AF1EE10FAC1F291815A4B5B4A27
:105E600093ED006AD2ED006A9BF99431CBED636A41
:105E700076EE665A012BCBED616ACBED605A8BED65
:105E8000646A01F0E386049BCBF89831002237EE78
:105E9000C77AFCEEE77A4E498BED677A17EE903AB7
:105EA000ABF88831012391ED005A8BF89431494BBE
:105EB0009A4242F26280484BD3ED007AD3ED013A28
:105EC000D3ED024AFEF71BBF354B93ED005AB5EEFA
:105ED000C05AF1EE10FA40F31686404BD3ED006A3B
:105EE000F5EEC06AF1EE10FA40F30D8636EEC77A91
:105EF00066EE4B5A87EE266AC5EE856AB7EE007AE3
:105F0000B4EEC76AF1EE10FA88BFB0EE476AB5EE9C
:105F1000C06AF1EE10FA76EE876AB8BFB0EE4C6A4E
:105F200066EE266A40E72E4AD2ED007AB0EEC87AD5
:105F3000B4EEE77AF1EE10FA7EF77DAE294AD2EDA3
:105F4000007AB0EEEC7AB4EEE77AF1EE10FA7EF772
:105F500072AE254AD8ED007A92ED007AF0EEE77A3B
:105F6000F4EEC77AF1EE10FA7EF565AE01220499DF
:105F7000CBF868118BF86421FEF748BEEC3900209D
:105F80004A3A0020243200205E420020303E0020A9
:105F9000F88000200081002000003443610BB63BF4
:105FA000F4800020F080002038240020E8800020C9
:105FB000E480002014390020503F0020547000205D
:105FC000D0810020D281002058870020BC81002091
:105FD000D88100208FD00300A0AF0020FC800020DB
:105FE00028810020248100202C810020DE4A02929A
:105FF00007EE103A1278DFF8B883CBF80C71B8EEE0
:10600000C77AF7EE006A132A86EE879AB8F9040079
:10601000BBF8105194ED070A01F0A485D34BD44A84
:1060200093ED001AD3ED053A93ED122A93ED173A4A
:10603000D3ED091AD3ED0E4A93ED016A93ED064AAA
:1060400093ED0A7AD3ED0F5AD3ED132AD3ED186AE4
:1060500093ED045AD3ED030A67EE897A69EE288A34
:1060600029EE088AE1EE273A02EB85060021A2EE2E
:10607000283ACBF80011CBF80411E1EE884AA6EEDD
:10608000274AE7EE085A93ED167A93ED0D6A93EDE1
:10609000021AD3ED0C1AC6ED003AE2EEA86A25EE1C
:1060A000635A27EE437A93ED0B2AD3ED152AC6EDFA
:1060B000204AA0EEE34A26EE646AD3ED143A83ED5B
:1060C000054AA1EE275AF0EE477AE1EEE45AA2EE35
:1060D000086AE2EEC36AE3EEA87A83ED065AC3EDDE
:1060E0000E5A83ED0F6A86ED403AC3ED176AC3ED91
:1060F000187ACBF808116B1C03F01F03ABF81031B2
:10610000A8F80400029BFEF75FBAABF8103299467C
:10611000002E3FF4C2AD022041E4039B5A8B91450F
:10612000C0F27D84B9F5FA6FD4BFC2EB0903C2F5A2
:10613000FA634FF47A7101FB03F19BF8A401C2F5F5
:10614000FA63B1FBF3F200283FF439AA9BF8A531BA
:10615000884902FB03F281FB0213D217C2EB6312E0
:10616000FFF72DBADFED847AFFF7E8B9DFED827A29
:10617000FFF7C6B9B9F5FA6F80F25484217AA9EB1A
:10618000020303FB01F3C2F5FA6293FBF2F3C3F1DE
:10619000640307EE903A9FED797AF8EEE77A67EEBE
:1061A000877ACBED497AFFF787B9754B1978DBF819
:1061B0001801744F9FED707AC600BB1983ED007A09
:1061C000002902F0AD83704AB0EE476AF0EE476AEC
:1061D0000023F2EC017A013367EEA77A05EE903ADC
:1061E000B4EEE77AF1EE10FAF8EEE55AB8BFB0EE89
:1061F000677A8B4276EEA76AA7EEA56AE9D1F5EE3B
:10620000C06ABB19F1EE10FA83ED007A42F388837D
:1062100086EE268A5D4BDFF89C81B8F80020F7EE09
:10622000007A38EE678AD3ED007A68EE277AFDEEC1
:10623000E77A17EE903A812B42F38E819342A8BF02
:10624000134607EE903AB8EEE70A514B304403EBA1
:106250008000F2F765F8FDEEC07AB8F8003017EE6E
:10626000902A812A42F37C819342A8BF134607EE0D
:10627000903AF8EEE77AFCEEE77ACDED037ABDF8D6
:106280000C30DBF81801C600BA199380029B1B780A
:1062900010B9132B02F0B487152B02F02B83142BAB
:1062A00001F0DB81DBF814213A4B013283FB02134E
:1062B0009918D317C3EBA103C3EBC303D21ACBF8CE
:1062C00014213549DBF81C21049D34480B68007803
:1062D000CBF81C51AA1A13440B60002840F0BC8074
:1062E00007EE902A2E4EDFF8D0902E4FB8EEE78AB8
:1062F00006F2447506F5F668F6EC017A94ED070AA5
:10630000D4F86C37F8EEE77A284627EE800A9847EB
:10631000A5F1E000D4F88C369847A5F17000D4F8C8
:10632000FC369847D6F85006D4F8AC309847D7EDED
:10633000007AA9EC010AE0EE087A2435A845E7ECDA
:10634000017AD9D1029B1D78FEF771BB164B174A13
:1063500019681288164BC96919805A8015B0BDECAE
:106360000C8BBDE8F08F00BF2C3E0020B44800200D
:10637000484600201F85EB51000000000AD7233C4F
:106380002A46002020490020E02200202C46002040
:106390004848002093244992648000201C46002035
:1063A0006472002068800020743D0020A62D00202B
:1063B000303E002028460020187A00205B4C15F063
:1063C000BFFE6378022B00F0BD86032B7FF475AC13
:1063D00041F2B813E35C002B41F09A8341F2A4032D
:1063E000E35C002B41F08F8341F2E803E35C002B78
:1063F00041F0848341F22C13E35C002B3FF45DAC4D
:106400004B481DF08CFB58E44A4B4B4F1B78DA0786
:1064100000F118843A78002A00F01886474B484962
:106420004848039392002AF07EFA474BDFF828A1F0
:10643000464D0593FEF7FFBFBBF8109209F1FF39F7
:106440000FFA89F9B9F1000FABF810923FF76EAA75
:10645000002E7FF460AE20E407EE902A3C4D3D4BC9
:10646000DFF8F880DFF8F890CDF80CB0F8EEE78AA6
:1064700005F2D4660027CDF818809B46029BD4ED28
:10648000077A1B78172B00F0958195ED007AB8EE0E
:10649000C78A082B28EE278A07D1B0EE480A059351
:1064A00029F0A0FA059BA8F80000DAF80020900077
:1064B0000BD5002F03F00281B0EE480AD4F86C37F8
:1064C00006F170009847B0EE408AB0EE480AD4F862
:1064D0008C36A6F170009847D4F8FC3630469847C1
:1064E000029B1B78032BB0EE408A00F05E81D5F84A
:1064F0005406D4F8AC30B0EE480A9847D9ED007A8B
:10650000ABEC010AE0EE287A0137032F06F12406EE
:1065100008F1020805F10405E9EC017AAED1029B0D
:10652000DDF80CB01D78FEF782BA00BF408800206D
:106530006C990020143900200D3E0020547000207A
:10654000F42D0020F8AF002048A60020503F002086
:1065500064720020187A0020247A0020303E002047
:1065600068800020002800F03787BCF1000F42F05F
:106570003F83CB48B8F1000F42F0E48190ED006A10
:106580009DED0C5AC74925EE866AFDEEE44AA5EE5C
:10659000076AB0EE675AA6EE265A14EE903ABDEEA0
:1065A000C56A16EE10CA16EE106AF445A8BF764604
:1065B0006345C8BF1E4606EE106AB8EEC66A012AD9
:1065C00081ED006A00F0DF8090ED046A9DED0D5AC8
:1065D00025EE866AA5EE076AB0EE675AA6EE265A41
:1065E000BDEEC56A16EE10CA16EE106AF445A8BFD5
:1065F00076469C45B8BF1E4606EE106AB8EEC66ADF
:10660000022A81ED016A00F0BE8090ED086A9DEDDE
:106610000E5A25EE866AA5EE076AB0EE675AA6EE18
:10662000265ABDEEC56A16EE10CA16EE106AF4457B
:10663000A8BF76469C45B8BF1E4606EE106AB8EE67
:10664000C66A032A81ED026A00F09D8090ED0C6A13
:106650009DED0F5A25EE866AA5EE076AB0EE675AE1
:10666000A6EE265ABDEEC56A16EE10CA16EE106AE0
:10667000F445A8BF76469C45B8BF1E4606EE106A94
:10668000B8EEC66A042A81ED036A7CD090ED106AE8
:106690009DED105A25EE866AA5EE076AB0EE675AA0
:1066A000A6EE265ABDEEC56A16EE10CA16EE106AA0
:1066B000F445A8BF76469C45B8BF1E4606EE106A54
:1066C000B8EEC66A052A81ED046A5CD090ED146AC2
:1066D0009DED115A25EE866AA5EE076AB0EE675A5F
:1066E000A6EE265ABDEEC56A16EE10CA16EE106A60
:1066F000F445A8BF76469C45B8BF1E4606EE106A14
:10670000B8EEC66A062A81ED056A3CD090ED186A9B
:106710009DED125A25EE866AA5EE076AB0EE675A1D
:10672000A6EE265ABDEEC56A16EE10CA16EE106A1F
:10673000F445A8BF76469C45B8BF1E4606EE106AD3
:10674000B8EEC66A072A81ED066A1CD090ED1C6A75
:106750009DED135A65EE865AE7EE055AE6EEA57AE8
:10676000FDEEE77A17EE900A8645A8BF864683427B
:10677000D8BF734607EE903AF8EEE77AC1ED077A94
:10678000002A3EF458AE9200474946482AF0CBF81A
:10679000464B1B68002B3EF453AE11F0A3F8FEF7F6
:1067A0004FBEF0EE676AFFF718B929F01BF9A8F899
:1067B00000009CE695ED007A04EB4702B8EEC78A2C
:1067C000128FA8F8002028EE278A6EE6B0EE465A0F
:1067D000FEF7CCBA364A374BD2F8EC201B6844F6A9
:1067E00020618A42A8BF0A46B2F57A7FB8BF4FF44B
:1067F0007A7292B2D806ABF8E22140F1BA84059BD6
:10680000002B01F0B0862C4B1868B0F832904FEA9C
:1068100059092A49DBF8E431D5ED037AA1FB0212CC
:106820009109642292FBF1F2142ABDEEE77A0BEB98
:10683000430EA8BF142201339342CBF8E43117EE84
:1068400010CAA4BF0023CBF8E4310BEB4303AEF82E
:10685000E8C1B3F9E83107EE103AB8EEC77A77EE3F
:10686000C77AFDEEE77ACDED057ABDF9142082EA0C
:10687000E273A3EBE2734B4502F32280104A4FF020
:106880007E531360FEF7ECBF1D210A48F3F704FCAA
:10689000002841F0B5830B4B03F1500218E000BF14
:1068A0003C810020F8AF0020F42D00208834002027
:1068B000AC0600208CAF00204C3A0020D34D621073
:1068C000980000202C29002004339A423EF49EAE0A
:1068D00019782629F8D193F802E0D8788645F3D2C2
:1068E000C44BDB78002B7EF491AEC348F3F7D4FBA6
:1068F000DFEDC27AC249002802F05E8438EE678A72
:10690000C6F57A72FDEEC87A12B2CDED097ABDF9FC
:1069100024301B0381FB0301DB17C3EBA11302FB34
:1069200003F343F30F33334407EE903AB8EEE78AAC
:10693000012385ED038A8BF8A031FEF767BEB14BCA
:106940000293DFF8F8B2BCE4D5ED027AAE4BB2EEBA
:106950000E7AF0EEE76AF4EEC76AF1EE10FA1F88DD
:10696000AA4B41D579073FD5B3F90430A84AA949C4
:10697000DFF8CCA2098882FB0302DB17C3EBA2037A
:106980005B1A9BB219B211F1B30FBCBF03F5B4731C
:1069900019B2B329C8BFA1F5B4739F4AC8BF19B2D1
:1069A0009AF804301278002B4FF6FF7318BF0123BA
:1069B00012077EF574AD994A126811FB03F3117E3C
:1069C000974A9BB211FB03F382FB03121A44DB17B5
:1069D000C3EB221307EE103AB8EEC77A77EEC77A08
:1069E000C5ED027AFEF75BBDB3F904308849894AE8
:1069F000DFF84CA281FB0301DB17C3EBA10313807B
:106A0000FEF74DBDA368002B3EF43EAD8549A1F1D4
:106A10004C009847DAF800300793FEF735BD05992A
:106A2000FFF78BBB237AC3F16403FFF7B2BB7A4B4A
:106A30001B7813F0100301F07E839BF8B821DBF87C
:106A4000BC3195ED017A002A0CBF01224FF0FF32D4
:106A500003FB02F307EE903AF8EEE77A77EE877AD7
:106A6000C5ED017AFEF7DABE1E216348F3F714FB89
:106A700000283FF40CA9099B002B7FF408A99BF880
:106A80003432A34242F04D82674B9BED8E0AD3ED28
:106A9000058ADBED4E5A9FED656ADFED656A20EEF3
:106AA000657A60EE087AA8EE887AE5EEA87AB4EE08
:106AB000C67AF1EE10FA88BFB0EE467AB4EEE67A06
:106AC000F1EE10FAF4EEC67AB8BFB0EE667AF1EEE7
:106AD00010FA88BFF0EE467AF4EEE67AF1EE10FA9C
:106AE000B8BFF0EE667A8BED4C7ACBED4E7AFFF7BD
:106AF000CEB8FDEEC87A4F4A17EE903AA2F804904D
:106B0000D380FFF7BEB8DFED4C6AFFF75BB9DAF868
:106B100000305E023EF530ABFEF732BBB4EEC87A11
:106B2000F1EE10FA98BFB0EE478ABDEEC77AB4EE28
:106B3000E68A404EF1EE10FA17EE103AB8BFB0EE0A
:106B4000668A8BED4C8A338000287EF4A3AFFFF772
:106B500098B8BDEEE77A374B17EE102A9A80FFF708
:106B600079B89FED327ADFED326A324AF4EEC77AB5
:106B7000F1EE10FA98BFB0EE677AFDEEE77AB4EE68
:106B8000E67AF1EE10FA17EE903AB8BFB0EE667AF8
:106B900001288BED4D7A53803EF7E2AFFFF771B8D5
:106BA000002B3EF448A8FEF72DB8F6F7ABFE029B8B
:106BB000089A1B78DFF87C80801A012BA8F8020065
:106BC00000F0AF82072B7EF45EA8F6F79BFE0790DD
:106BD000FEF75BB8F6F796FE029B07991B78154AFD
:106BE000401A072B90807EF447ACF6F78BFE089096
:106BF000FEF744BC4C3200208CAF002000007A44E9
:106C0000D34D62102C3E0020483A0020F839002075
:106C100067666666343D00204A3A00204C3A002000
:106C200089888888847200209800002000C0F94478
:106C300000C0F9C4303E002000000000E022002027
:106C4000808700203B78002B00F00082DBED573A74
:106C50009BED566ADBED617AED4A9BED607AD2EDF1
:106C6000005A9BED544ADBED534AEA48EA49F4EEF8
:106C7000C63AF3EE046AF1EE10FA37EEA65A00F1C6
:106C8000CB8290ED026A26EE446AF0EE674AE6EEA9
:106C9000074AF4EEC54A34EEE66AF1EE10FA48BF50
:106CA000B0EE656A012B81ED006A00F0CF8190EDB6
:106CB000066A26EE446AF0EE674AE6EE074AF4EE0C
:106CC000C54A34EEE66AF1EE10FA48BFB0EE656AE6
:106CD000022B81ED016A00F0B98190ED0A6A26EE7F
:106CE000446AF0EE674AE6EE074AF4EEC54A34EE2F
:106CF000E66AF1EE10FA48BFB0EE656A032B81ED4B
:106D0000026A00F0A38190ED0E6A26EE446AF0EE6E
:106D1000674AE6EE074AF4EEC54A34EEE66AF1EE5B
:106D200010FA48BFB0EE656A042B81ED036A00F0EB
:106D30008D8190ED126A26EE446AF0EE674AE6EE27
:106D4000074AF4EEC54A34EEE66AF1EE10FA48BF9F
:106D5000B0EE656A052B81ED046A00F0778190ED55
:106D6000166A26EE446AF0EE674AE6EE074AF4EE4B
:106D7000C54A74EEE66AF1EE10FA48BFF0EE656AB5
:106D8000062BC1ED056A00F06181D0ED1A6A66EE4E
:106D9000C46AF0EE674AE6EE874AB3EE046AF4EEA0
:106DA000C54A74EEC66AF1EE10FA48BFF0EE656AA5
:106DB000072BC1ED066A00F04981D0ED1E6A974BA2
:106DC000039326EEC44A964BDFF860A2954D0593D7
:106DD000E4EE077AF4EEC57A77EEC67AF1EE10FAB1
:106DE00048BFF0EE657AC1ED077AFEF724BB89480B
:106DF0009DED0C5A90ED006ABCF1000F41F040820D
:106E000025EE866A8449A5EE076AB0EE675AA6EEBB
:106E1000265ABDEEC56A16EE10CA16EE106AF44583
:106E2000A8BF76466345C8BF1E4606EE106AB8EE98
:106E3000C66A012A81ED006A3FF4A5AC90ED046AB0
:106E40009DED0D5A25EE866AA5EE076AB0EE675AEB
:106E5000A6EE265ABDEEC56A16EE10CA16EE106AE8
:106E6000F445A8BF76466345C8BF1E4606EE106AC5
:106E7000B8EEC66A022A81ED016A3FF484AC90ED57
:106E8000086A9DED0E5A25EE866AA5EE076AB0EEF9
:106E9000675AA6EE265ABDEEC56A16EE10CA16EE61
:106EA000106AF445A8BF76466345C8BF1E4606EE85
:106EB000106AB8EEC66A032A81ED026A3FF463AC39
:106EC00090ED0C6A9DED0F5A25EE866AA5EE076AD5
:106ED000B0EE675AA6EE265ABDEEC56A16EE10CA87
:106EE00016EE106AF445A8BF76466345C8BF1E4635
:106EF00006EE106AB8EEC66A042A81ED036A3FF412
:106F000042AC90ED106A9DED105A25EE866AA5EE12
:106F1000076AB0EE675AA6EE265ABDEEC56A16EEAF
:106F200010CA16EE106AF445A8BF76466345C8BF7E
:106F30001E4606EE106AB8EEC66A052A81ED046A9E
:106F40003FF421AC90ED146A9DED115A25EE866A4E
:106F5000A5EE076AB0EE675AA6EE265ABDEEC56AE0
:106F600016EE10CA16EE106AF445A8BF76466345C1
:106F7000C8BF1E4606EE106AB8EEC66A062A81ED44
:106F8000056A3FF400AC90ED186A9DED125A25EEAB
:106F9000866AA5EE076AB0EE675AA6EE265ABDEEDF
:106FA000C56A16EE10CA16EE106AF445A8BF7646FA
:106FB0006345C8BF1E4606EE106AB8EEC66A072AC9
:106FC00081ED066A3FF4DFAB90ED1C6A9DED135A2C
:106FD00065EE865AE7EE055AE5EEA67AFDEEE77A0B
:106FE00017EE900A8645A8BF86468342C8BF9E46D4
:106FF00007EE90EAF8EEE77AC1ED077AFFF7C0BB3B
:10700000DFED096AFEF72ABDDFED076AFEF71DBE58
:10701000388100203C810020F8AF0020547000200F
:1070200048A60020503F00200000C842247A0020DB
:10703000B5EEC07AF1EE10FA01F18582B7EE006A82
:1070400036EE477AC6EE076AFEF76EBDCD4B039368
:10705000CD4BDFF87CA3CD4D0593FEF7ECB9CC4AC0
:107060005379002B3DF40BAFCA4B1B78002B3DF43A
:1070700006AF1278DFEDC84A07EE902AC74AB8EE8D
:10708000677A128807EE903A06EE902AF8EEE77AD1
:10709000F8EE666A67EE277AB7EE007A87EEA63AD0
:1070A000B4EEE43AF1EE10FA88BFB0EE643AB4EE12
:1070B000C73AF1EE10FAB8BFB0EE473AFDF7E1BEBD
:1070C000B74B5A88FEF7E0BBBBF8E22102F57A72B3
:1070D00092B2FEF7D9BBB34BD3ED005AFEF754BEC4
:1070E000B14B9FEDB27AD3ED087AF4EEC77AF1EEA8
:1070F00010FA00F28F849FEDAE7AD5ED037A77EE29
:10710000877AC5ED037AFEF7A6BB049823F090FAC0
:10711000FEF7DBBDF6F7F6FB0890FDF754BBDFF892
:10712000B482F6F7EFFBA34ADBF8783112680790D8
:10713000C31A9A1ACBF87801A8F80430A8F80620E8
:10714000FDF7A3BDA3784FF00109072B3EF6B5ADBF
:10715000DFE813F0CC06F006E406A80645062E0686
:107160003806FC05944B9B7B002B3EF46AABFEF784
:107170006CBB079BD9003FF542ABFEF771BBBBF878
:1071800088219A4200F29184262021F073FE002883
:1071900040F08B84894B8A4AD3ED007A894B92ED7B
:1071A000007A1B78CBED637A8BED647A002B01F0CB
:1071B000818377EE676A9BF99431CBED606A013386
:1071C000CBED617A01F04986049BCBF8983100221F
:1071D0009FED777A7C498BED677AFF2391ED005A1A
:1071E0008BF89431FEF763BE0120F7F733F9DBF833
:1071F0006821049B9A1AFDF7A1BB744BD8ED007A65
:1072000093ED007AF0EEE77AF4EEC77AF1EE10FA39
:107210007DF711ADFDF709BD90ED016A26EE646AB8
:10722000B0EE674AA6EE074AB4EEC54A34EE666A87
:10723000F1EE10FA48BFB0EE656A012B81ED006AED
:107240003FF404AF90ED056A26EE646AB0EE674A3B
:10725000A6EE074AB4EEC54A34EE666AF1EE10FABD
:1072600048BFB0EE656A022B81ED016A3FF4EEAED5
:1072700090ED096A26EE646AB0EE674AA6EE074A08
:10728000B4EEC54A34EE666AF1EE10FA48BFB0EECD
:10729000656A032B81ED026A3FF4D8AE90ED0D6A6A
:1072A00026EE646AB0EE674AA6EE074AB4EEC54A17
:1072B00034EE666AF1EE10FA48BFB0EE656A042B50
:1072C00081ED036A3FF4C2AE90ED116A26EE646A66
:1072D000B0EE674AA6EE074AB4EEC54A34EE666AD7
:1072E000F1EE10FA48BFB0EE656A052B81ED046A35
:1072F0003FF4ACAE90ED156A26EE646AB0EE674AD4
:10730000A6EE074AB4EEC54A74EE666AF1EE10FACC
:1073100048BFF0EE656A062BC1ED056A3FF496AEF4
:10732000D0ED196A66EEE46AB0EE674AA6EE874AC7
:10733000B3EE046AB4EEC54A74EE466AF1EE10FA92
:1073400048BFF0EE656A072BC1ED066A3FF47EAEDA
:10735000D0ED1D6A0B4B039366EEE44A0A4BDFF84F
:1073600070A00A4D0593E4EE877AF4EEC57A77EEC5
:10737000C67AF1EE10FAB8BFF0EE657AC1ED077A81
:10738000FEF759B85470002048A60020503F002056
:10739000DC3900204E3F0020713DAA3F383F0020DD
:1073A000DC2F0020F48000203C8000208FC2753C40
:1073B0000000000084B10020C87000205487002025
:1073C000C0810020487C0020D48100202C81002036
:1073D000247A0020303E0020E348B8F1000F41F04D
:1073E000D98090ED006A9DED0C5AE04925EE866A41
:1073F000FDEEE44AA5EE076AB0EE675AA6EE265AFD
:1074000014EE903ABDEEC56A16EE108A16EE106ABA
:10741000F045A8BF76464345C8BF1E4606EE106A33
:10742000B8EEC66A012A81ED006A3EF400A890ED2C
:10743000046A9DED0D5A25EE866AA5EE076AB0EE48
:10744000675AA6EE265ABDEEC56A16EE108A16EEEB
:10745000106AF045A8BF76469845B8BF1E4606EEAE
:10746000106AB8EEC66A022A81ED016A3DF4DFAF08
:1074700090ED086A9DED0E5A25EE866AA5EE076A24
:10748000B0EE675AA6EE265ABDEEC56A16EE108A11
:1074900016EE106AF045A8BF76469845B8BF1E465E
:1074A00006EE106AB8EEC66A032A81ED026A3DF460
:1074B000BEAF90ED0C6A9DED0F5A25EE866AA5EEE3
:1074C000076AB0EE675AA6EE265ABDEEC56A16EEFA
:1074D000108A16EE106AF045A8BF76469845B8BFE8
:1074E0001E4606EE106AB8EEC66A042A81ED036AEB
:1074F0003DF49DAF90ED106A9DED105A25EE866A21
:10750000A5EE076AB0EE675AA6EE265ABDEEC56A2A
:1075100016EE108A16EE106AF045A8BF764698451A
:10752000B8BF1E4606EE106AB8EEC66A052A81ED9F
:10753000046A3DF47CAF90ED146A9DED115A25EE7E
:10754000866AA5EE076AB0EE675AA6EE265ABDEE29
:10755000C56A16EE108A16EE106AF045A8BF764688
:107560009845B8BF1E4606EE106AB8EEC66A062AEF
:1075700081ED056A3DF45BAF90ED186A9DED125AFE
:1075800025EE866AA5EE076AB0EE675AA6EE265A81
:10759000BDEEC56A16EE108A16EE106AF045A8BF59
:1075A00076469845B8BF1E46FDF71FBF704EDBED0F
:1075B000017A9BED006A3188736977EEA77AF0EE65
:1075C000006AB0EE677AA6EE267A4E1E0BEBC60175
:1075D000D6EE267A08391033F6EE003A27EE237AF3
:1075E00067EEA37A8BED207ACBED217ADFF888B1B4
:1075F0005F460BF1800091ED027A91ED036AD7EDC1
:10760000036AD7ED027A53ED014A13ED025A37EEC1
:10761000674A76EEC65A77EE277AE4EE845A013E40
:10762000A1F10801E5EE047A07F1080703F1080368
:1076300036EE267A00F10800E4EE877AE5EE475A46
:1076400067EEA37A25EEA37AC0ED007A80ED017A89
:10765000D1D1BEF1140F7EF427AEF6F753F9DFF85F
:107660002C81DBF81421401BA8F80200FEF71CBE99
:10767000DBF81801BBF810313E4FDFF814813E4AA9
